:0C00000094EF03F000F000F004EF08F0B3
:04100000F9EF08F00C
:101008004D82FACF15F0FBCF16F0E9CF17F0EACFF3
:1010180018F0E1CF19F0E2CF1AF0D9CF1BF0DACFF0
:101028001CF0F3CF1DF0F4CF1EF0F6CF1FF0F7CF72
:1010380020F0F8CF21F0F5CF22F04DC023F04EC0BC
:1010480024F04FC025F050C026F0F2A473D0000E53
:101058000101FB27000EFC23FF0EFD23FF0EFE23DC
:10106800FEBF05D0FE5165E1FD05D8B062D02D0E5A
:10107800FB27310EFC23010EFD23000EFE23334A0D
:10108800342A010E0827000E09230A230B230F0E0A
:10109800345CD8A006D0264B272B000E346E000EE9
:1010A800336E52515311D8B403D05207D8A0530706
:1010B80050515111D8B403D05007D8A051074E5100
:1010C8004F11D8B403D04E07D8A04F074C514D113B
:1010D800D8B403D04C07D8A04D074A514B11D8B407
:1010E80003D04A07D8A04B0748514911D8B403D0B8
:1010F8004807D8A0490746514711D8B403D0460736
:10110800D8A0470744514511D8B403D04407D8A004
:10111800450740514111D8B403D04007D8A0410732
:101128003E513F11D8B403D03E07D8A03F07EFEC9B
:1011380061F0F29477A00BD026C107F027C108F020
:1011480033C009F034C00AF05CEC50F0779077A215
:101158000BD026C107F027C108F033C009F034C00E
:101168000AF095EC4FF0779277AE04D00101244B4A
:10117800252B779E77AA04D00101244B252B779A3B
:101188009EAA03D08DEC67F09E9AA4AA03D08DEC9A
:1011980067F0A49A77A403D008EC3AF0779426C0B5
:1011A80050F025C04FF024C04EF023C04DF022C0AF
:1011B800F5FF21C0F8FF20C0F7FF1FC0F6FF1EC0D3
:1011C800F4FF1DC0F3FF1CC0DAFF1BC0D9FF1AC013
:1011D800E2FF19C0E1FF18C0EAFF17C0E9FF16C017
:1011E800FBFF15C0FAFF4D92110014EF63F00000E9
:1011F8000099C5ABCE320BCFD8561D6416FDD30768
:10120800F49E31AC3A35FFC82C51E963E2FA2797CE
:10121800AD0E683C63A5A65875C1B0F3BB6A7E9055
:1012280059099C3B97A2525F81C644F44F6D8A2EA0
:101238005BB79E85951C50E18378464A4DD3882933
:10124800AFB06A82611BA4E6777FB24DB9D47CB98E
:10125800F6203312388BFD762EEFEBDDE04425BE09
:101268000227C715CC8C0971DAE81FDA1443D1C5F7
:10127800F35C366E3DF7F80A2B93EEA1E53820C2F1
:10128800075BC269C9F00C0DDF941AA6113FD4524E
:101298005ECB9BF99060559D8604433648AF8D55CB
:1012A800AACC6FFE6467A19A7203B731BCA879EB28
:1012B800A8726D4066D9A32470BDB58FBE167BECAD
:1012C8005C75994792DE572384BA41884A118F7C0E
:1012D80005E5C0D7CB4E0EB3DD2A18181381D67B8F
:1012E800F1E234D03F49FAB4292DEC1FE7862213E6
:1012F800A28A67B86C21A9DC7A45BF77B4EE71146D
:10130800568D93BF98265DDB8E424B7040E98584ED
:101318000F1DCA2FC1B6044BD7D212E01979DC834E
:10132800FB1A3E2835B1F04C23D5E6E7ED7E283D83
:10133800F9A43C96370FF2F2216BE459EFC02A3A30
:101348000DA3C891C30806F5D56C105E1BC7DEAAAD
:10135800543391019A985F658CFC49CE425787AD0A
:10136800A03465066E9FAB6278FBBDC9B65073D6D4
:10137800514F947D9FE45A1989804CB2472B82D1F2
:10138800A548607A6BE3AE1E7D87B8B5B32C76416D
:10139800FCD839EA3273F78E2417E125EABC2F46C8
:1013A80008DFCDEDC6740389D01015221EBBDBF80B
:1013B8000A61CF53C4CA0137D2AE179C1C05D9FFA6
:1013C800FE663B5430CDF53026A9E39BE8022D6F2D
:1013D800A7F662C4695DACA07F39BA0BB192746894
:1013E80053F196C39D5A58A78B3E4E0C45958020C5
:1013F8002053457420205B3C3E7C49447C43414E4D
:1014080042527C4C56437C4856437C4C5643437C62
:10141800485643437C4256437C42564D494E7C5481
:10142800484D41587C4C564344454C41597C48569C
:101438004344454C41597C4D41505D0D0A202020C4
:1014480020202020203C3E20202020202020202D4D
:101458002073686F7720636F6E6669670D0A2020B6
:1014680020202020202069642020202020202020E7
:101478002D20626D73632049442028312E2E342993
:101488000D0A202020202020202063616E62722017
:10149800202020202D2043414E2062617564207257
:1014A80061746520283132357C3235307C353030F6
:1014B800290D0A20202020202020206D6170203C4A
:1014C8006C74633E203C7061636B3E203C677270B5
:1014D8003E202D204D617020616E204C54432074B5
:1014E8006F2061205061636B2F43656C6C204772DD
:1014F8006F75700D0A202020202020202068766338
:10150800202020202020202D204869676820566F41
:101518006C74616765204375746F66660D0A2020D8
:101528002020202020206C766320202020202020CE
:101538002D204C6F7720566F6C746167652043755A
:10154800746F66660D0A20202020202020206876EF
:101558006364656C617920202D2044656C61792075
:1015680028696E207365636F6E64732920626566EF
:101578006F7265207265706F7274696E6720485665
:101588004320616C6572740D0A20202020202020E1
:10159800206C766364656C617920202D2044656C2D
:1015A80061792028696E207365636F6E64732920E2
:1015B8006265666F7265207265706F7274696E67B6
:1015C800204C564320616C6572740D0A202020203F
:1015D80020202020687663632020202020202D20D2
:1015E8004869676820566F6C746167652043757435
:1015F8006F666620436C6561722054687265736813
:101608006F6C640D0A20202020202020206C766337
:10161800632020202020202D204C6F7720566F6CCF
:1016280074616765204375746F666620436C6561F5
:1016380072205468726573686F6C640D0A202020EC
:101648002020202020627663202020202020202DAA
:10165800204368617267652042616C616E63696EE0
:101668006720566F6C74616765204375746F666692
:101678000D0A202020202020202062766D696E200F
:10168800202020202D2043656C6C204469736368FA
:10169800617267652042616C616E63696E6720568E
:1016A8006F6C74616765204D696E696D756D0D0AA3
:1016B800202020202020202074686D6178202020A0
:1016C80020202D20546865726D6973746F72204DE7
:1016D80061782054656D70657261747572650D0A64
:1016E800002020454E61626C65207C20444953618E
:1016F800626C65205B42414C414E43457C43414E00
:101708005445524D7C4333313030527C54486572D5
:101718006D6973746F72730D0A20202020202020B9
:10172800202020202020202020202020207C4C4FFA
:101738004F504F437C4C4F4F50434C4F5345444FB1
:101748004E464C547C53504545444855545D0D0A0B
:10175800202020202020202062616C616E6365209B
:1017680020202D20656E61626C652F64697361624B
:101778006C652043656C6C204469736368617267AB
:10178800652042616C616E63696E670D0A202020D6
:10179800202020202063616E7465726D2020202D2A
:1017A80020656E61626C652F64697361626C652087
:1017B80043414E207465726D696E6174696F6E2065
:1017C8007265736973746F720D0A202020202020BF
:1017D8002020333130307220202020202D20656ECB
:1017E80061626C652F64697361626C652043757210
:1017F80074697320333130305220646973706C61BE
:10180800790D0A2020202020202020746865726D20
:101818006973746F7273203C6C74633E203C6E7500
:101828006D3E202D20656E61626C652F6469736161
:10183800626C6520746865726D6973746F72287361
:10184800290D0A00202053486F77205B3C3E7C56C8
:10185800657273696F6E7C434F6E6669677C4D4134
:10186800507C43454C4C537C4C54437C535441541A
:10187800537C544865726D6973746F72735D0D0A99
:1018880020202020202020203C3E20202020202016
:1018980020202D207374617475730D0A2020202078
:1018A8002020202076657273696F6E2020202D20FD
:1018B8006669726D776172652076657273696F6E9D
:1018C8000D0A2020202020202020636F6E66696783
:1018D800202020202D20636F6E6669677572617401
:1018E800696F6E0D0A20202020202020206D617055
:1018F800202020202020202D2063656C6C2067721A
:101908006F7570206D61700D0A2020202020202026
:101918002063656C6C7320202020202D2063656C6B
:101928006C2076616C7565730D0A202020202020BC
:1019380020206C7463202020202020202D206D651D
:1019480061737572656D656E742063686970730D77
:101958000A20202020202020207374617473202006
:101968002020202D2063656C6C207374617469736A
:10197800746963730D0A20202020202020207468B9
:1019880065726D6973746F7273202D207468657247
:101998006D6973746F722072656164696E67730D27
:1019A8000A000D0A202A2A2A0D0A202A2A2A20207B
:1019B800202020202020202020202020202020201F
:1019C800205374617274696E6720424D53432055E9
:1019D800706772616465202020202020202020204C
:1019E800202020202020202020202020202A2A2AD1
:1019F8000D0A202A2A2A2031292045786974206670
:101A0800726F6D20746865207465726D696E616CA3
:101A1800206170706C69636174696F6E202020208A
:101A280020202020202020202020202020202020AE
:101A380020202020202A2A2A0D0A202A2A2A203279
:101A4800292053746172742074686520626F6F7402
:101A58006C6F6164657220616E6420646F776E6C70
:101A68006F61642061206E6577202E686578206636
:101A7800696C65202020202020202020202A2A2A66
:101A88000D0A202A2A2A203329205265737461728C
:101A9800742074686520424D534320202020202064
:101AA800202020202020202020202020202020202E
:101AB800202020202020202020202020202020201E
:101AC80020202020202A2A2A0D0A0D0A0020205230
:101AD80045736574205B434F4E4649477C535441D8
:101AE80054535D0D0A2020202020202020636F6E93
:101AF800666967202020202D207265736574206335
:101B08006F6E66696775726174696F6E20746F2095
:101B180064656661756C74730D0A2020202020208E
:101B28002020737461747320202020202D2072657A
:101B38007365742063656C6C207374617469737465
:101B48006963730D0A00687C68656C707C736574E2
:101B58007C73657C73686F777C73687C747261636F
:101B6800657C74727C656E7C656E61626C657C6494
:101B780069737C64697361626C657C6469736368AA
:101B8800617267657C73656E647C72657365747C6D
:101B9800757067726164657C6C6F636B7C676900E4
:101BA80062616C616E63657C63616E7465726D7C85
:101BB80033313030727C74687C746865726D697317
:101BC800746F727C746865726D6973746F72737CFC
:101BD8006C6F6F706F637C6C6F6F70636C6F736525
:101BE800646F6E666C747C736D70307C7370656541
:101BF80064687574002D2D2D2D7C2D2D2D2D2D2DEA
:101C08002D2D7C2D2D2D7C2D2D2D2D2D2D2D2D2D5E
:101C18002D2D2D2D2D2D2D2D2D2D2D2D2D2D2D2DEC
:101C28002D2D2D2D2D2D2D2D2D2D2D2D2D2D2D2DDC
:101C38002D2D2D2D2D2D2D2D2D2D2D2D2D2D2D2DCC
:101C48002D2D2D2D2D2D0D0A00206C74637C2073F5
:101C58007461747573207C7265767C202056616E81
:101C680020207C202056646967207C2020567265DD
:101C780066207C20544D50207C202020534F432048
:101C8800207C20202053554D20207C2020636F6E1F
:101C980066207C2020646973630D0A0069647C6D8A
:101CA80061707C6C76637C6C7663637C6876637C3D
:101CB800687663637C6276637C62766D696E7C7439
:101CC800686D61787C74686D696E7C6362727C6330
:101CD8006272727C6C766364656C61797C68766329
:101CE80064656C61797C63616E62720020202020DB
:101CF800202020206C6F6F706F63202020202D2003
:101D08006C6F6F7020697320636F6E666967757298
:101D18006564206173206F70656E20636F6C6C65FD
:101D280063746F722028485643206C70312C204C05
:101D38005643206C7032290D0A00746F74616C7CF4
:101D48002D6D65616E2063656C6C20766F6C7461B7
:101D580067652D2D2D2D2D2D7C2D7374616E64617D
:101D6800726420646576696174696F6E2D2D2D2DFE
:101D78002D2D2D2D2D2D2D2D2D2D2D2D0D0A002008
:101D8800202020202020206C6F6F70636C6F73659B
:101D9800646F6E666C74202D206C6F6F70206C6F92
:101DA8006769632072657665727365643A20636C4F
:101DB8006F736564206F6E206661756C740D0A0020
:101DC8007C2D766F6C746167652D2D2D2D6D696E78
:101DD8002D2D2D2D6D61782D2D7C2D2D2D2D6465AE
:101DE80076696174696F6E2D2D2D2D2D6D696E2D9F
:101DF8002D2D6D61782D2D64656C74612D0D0A0093
:101E08002A202020202020202020202020202020C0
:101E1800202020202044696C69746869756D20440D
:101E2800657369676E202020202020202020202034
:101E38002020202020202A0D0A002A2A2A2A2A2A9D
:101E48002A2A2A2A2A2A2A2A2A2A2A2A2A2A2A2AEA
:101E58002A2A2A2A2A2A2A2A2A2A2A2A2A2A2A2ADA
:101E68002A2A2A2A2A2A2A2A2A2A2A2A2A2A2A2ACA
:101E78002A0D0A004348414E47494E472043414EE8
:101E8800204241554452415445202D205359535422
:101E9800454D204D4159204245434F4D4520554E13
:101EA800555341424C452021210D0A006C6F6F703B
:101EB800636C6F7365646F6E666C7420286C6F6FEB
:101EC80070206C6F676963207265766572736564EC
:101ED8003A20636C6F736564206F6E20666C74299A
:101EE8000D0A00767C76657273696F6E7C636F7C11
:101EF800636F6E6669677C6C74637C74687C7468F5
:101F080065726D6973746F72737C63656C6C737CD6
:101F180073746174737C6D6170002D2D2D2D7C2D73
:101F28002D2D2D7C2D2D2D2D2D7C2D2D2D2D2D2D3B
:101F38002D2D2D2D2D2D2D2D2D2D2D2D2D2D2D2DC9
:101F48002D2D2D2D2D2D2D2D2D2D2D2D0D0A006CEA
:101F58006F6F706F6320284C6F6F70206F7574708F
:101F680075747320617265206F70656E20636F6C85
:101F78006C6563746F72204856432C204C56432975
:101F88000D0A00202055504752414445202020206A
:101F980020202020202D20706572666F726D7320BE
:101FA80061206669726D776172652075706772610C
:101FB80064650D0A0062616C616E63652028636563
:101FC8006C6C206469736368617267652062616C18
:101FD800616E63696E6720697320656E61626C6506
:101FE80064290D0A00636F6E6669677572617469AA
:101FF8006F6E204E4F54206C6F636B65643B206E90
:102008006F2063656C6C7320646973636F766572A7
:1020180065640D0A0063616E7465726D2028434122
:102028004E207465726D696E6174696F6E20726599
:10203800736973746F7220656E61626C6564290DD3
:102048000A00202020202020202073706565646805
:10205800697420202D205350454544485554204349
:10206800414E206D657373616765730D0A00737067
:10207800656564687574202873706565646875742F
:102088002043414E206D6573736167657320656EEB
:1020980061626C6564290D0A002D2D2D2D7C2D2D76
:1020A8002D2D2D2D2D2D2D2D2D2D2D2D2D2D2D2D58
:1020B8002D2D2D2D2D2D2D2D2D2D2D2D2D2D2D2D48
:1020C8002D0D0A0020204C4F434B2020202020209B
:1020D8002020202020202D206C6F636B20636F6EE2
:1020E80066696775726174696F6E0D0A00206C7499
:1020F800637C2020543120207C2020543220207CF6
:102108002020543320207C2020543420207C202080
:1021180054350D0A0053657474696E6773207769C6
:102128006C6C20626520696E20706C616365207537
:102138006E74696C2072657365740D0A003A206EBE
:102148006F7420616C6C20636F6E66696775726569
:10215800642063656C6C732064657465637465647E
:102168002021006572726F723A20546865726D6939
:1021780073746F72204944206F7574206F662072E3
:10218800616E67650D0A002A20202020202020206B
:1021980020202020202020202020424D5320436F43
:1021A8006E74726F6C6C657220006368616E67692B
:1021B8006E67204333313030722043414E206261D4
:1021C80075642072617465210D0A003331303072F4
:1021D800202843757274697320646973706C61791F
:1021E80020656E61626C6564290D0A00547970651A
:1021F80020616E79206B657920746F20636F6E742F
:10220800696E7565202E2E2E0D0A006572726F722A
:102218003A207061636B202F2063656C6C206E6FB1
:102228007420666F756E640D0A006D616E75616C61
:1022380020646973636861726765207475726E657E
:1022480064206F66660D0A006572726F723A206EBE
:102258006F20686172647761726520737570706F42
:1022680072740D0A00766572626F7365207472610C
:1022780063696E67206973206E6F77204F4E0D0A71
:102288000063616E20626175642072617465206EFE
:102298006F74206368616E6765640D0A0065727209
:1022A8006F723A204F7074696F6E2069732072657F
:1022B8007175697265640D0A0063616E62757320D9
:1022C80074726163696E67206973206E6F77204F3F
:1022D8004E0D0A00636F6E66696775726174696F87
:1022E8006E206E6F74206C6F636B65640D0A0063FB
:1022F80068616E67696E672043414E20626175644C
:102308002072617465210D0A006572726F723A203D
:102318004C5443206F7574206F662072616E676538
:102328000D0A00616C6C2074726163696E672069C4
:1023380073206E6F77204F46460D0A006572726FE4
:10234800723A20556E6B6E6F776E20436F6D6D61BC
:102358006E640D0A00206C74637C7061636B7C672B
:10236800726F75707C2063656C6C730D0A00202099
:10237800736D70302020202020203A20656E616225
:102388006C65640D0A006572726F723A20556E6B47
:102398006E6F776E204F7074696F6E0D0A006572EC
:1023A800726F723A20756E6B6E6F776E206F7074F5
:1023B800696F6E0D0A00636F6E6669677572617486
:1023C800696F6E206C6F636B65640D0A00746865D5
:1023D800726D6973746F72732064697361626C657E
:1023E800640D0A006572726F723A2062616420702F
:1023F8006172616D657465720D0A0063616E7C635C
:10240800616E6275737C6F66667C766572626F73E7
:102418006500746865726D6973746F727320656E98
:1024280061626C65640D0A00746865726D69737425
:102438006F72206F76657274656D700D0A002C20BE
:10244800646961676E6F73746963206661696C752E
:1024580072653D006E6F2063656C6C7320646574F3
:1024680065637465640D0A00746865726D697374D8
:102478006F722063656E7375730D0A00202020202B
:10248800202020202020202020202020207C200008
:10249800202076657273696F6E2020203A202020F4
:1024A8002000204E4F542044455445435445442170
:1024B8000D0A00206D75737420626520626574775B
:1024C80065656E00432C204F56455254454D5021AA
:1024D8000D0A00202020202020202020202020203D
:1024E80020002020203F3F202020202020202020C6
:1024F80000202D2D2D2D2D2D2020202020202000C6
:102508002020202020202020202020203A200020C9
:1025180020696420202020202020203A200020202C
:1025280063616E627220202020203A2000202074EF
:10253800686D617820202020203A200020206F70CC
:1025480074696F6E732020203A200020206876631B
:1025580064656C617920203A200020206C766364E1
:10256800656C617920203A20002C204C5443206F60
:1025780076657274656D7000202D2D2D2D2D2D2DF5
:102588002D2D2D0D0A006469736368617267696E89
:10259800670D0A0063656C6C2063656E7375730D57
:1025A8000A0020203331303072202020203A2000C9
:1025B80020207363616E73202020203A20002020A1
:1025C80049736F5350492020203A2000202075700D
:1025D80074696D652020203A20002020616C6572A6
:1025E80074732020203A20002020202063656C6C22
:1025F8007320203A200020202020766F6C746167B9
:10260800653A2000762C2064697363686172676597
:1026180020002020627663202020202020203A00FD
:102628002020687663202020202020203A002020C7
:102638006C7663202020202020203A002020687615
:1026480063632020202020203A0020206C766363DA
:102658002020202020203A00202062766D696E20FC
:10266800202020203A00207365636F6E6428732948
:102678000D0A00432C2074656D70204F4B0D0A0025
:10268800206D696E7574652873292C200020202020
:10269800206D65616E2020203A0020202020737470
:1026A80064206465763A006E6F74206465746563AF
:1026B8007465640073746174737C636F6E666967B4
:1026C800002C204C544320616273656E74002069AD
:1026D8006E2048564320210D0A0020696E204C5672
:1026E8004320210D0A003132357C3235307C3530BB
:1026F80030004D6179203133203230323200646449
:102708005F696E64202020203A0064645F726571FE
:10271800202020203A0020504543206572726F72B5
:102728003D006F7065726174696F6E616C0020683E
:102738006F75722873292C2000756E6B6E6F776E1B
:1027480020203A00206E6F207265706C793D002061
:1027580020746F74616C0D0A00207265747269656B
:10276800733D002020202020206C746300202070FE
:1027780061636B0D0A00206661756C742028003057
:10278800383A35353A31350020636F6E6669673DF2
:102798000067726F75702069640068766364656CA1
:1027A8006179006C766364656C6179002073656398
:1027B800730D0A0073686F72740D0A00203E42564A
:1027C80043202000203E485643202000203C4C5601
:1027D800432020006572726F723A20003A6469657E
:1027E800203D2000203E485643432000203C4C56C4
:1027F80043432000203E3E444953200076322E3287
:102808002E3134002070726F62653D002073746150
:1028180072743D007061636B20696400206E2F61E3
:102828000D0A006E6F6E650D0A006B6270730D0AFB
:10283800002020202E20200020204E432020002091
:10284800206F6B20200020203C30432000203A20BD
:1028580052583D0020727472763D002053484F5202
:1028680054006C74632069640020207061636B00FD
:1028780020202020207C004256430D0A0048564361
:102888000D0A004C56430D0A00203F3F3F200070C0
:1028980061636B200077616B653D0062766D696EE0
:1028A8000074686D6178000D0A0A0A006E630D0AEB
:1028B80000202B202000202D202000207C2020001C
:1028C800202B2B2000202D2D200076207C2000207E
:1028D800207C280068766363006C76636300626D11
:1028E80073630020616E640020666C7400760D0AC4
:1028F8000073202000762020003235300031323538
:102908000028633D00206D3D004C5443004F46466F
:102918000062766300687663006C7663006F6666B3
:1029280000616C6C003B20003E2000732000202ECC
:1029380000203F004F4E003A5400205800767C009B
:0D29480029002B002D002F007600770000E5
:10295600ECC095F0EDC096F0EEC097F0EFC098F0A1
:10296600A40E0001996F1C0E9A6FB80E9B6F010E94
:102976009C6FDFEC70F00009D8A405EF1AF03BEF6E
:102986001AF0F0EC34F01200ECC095F0EDC096F0C1
:10299600EEC097F0EFC098F0BD0E0001996F010EE2
:1029A6009A6F8DEC71F00009D8B434D0000E010195
:1029B600AB6FBD51BE11D8B408D0BE5106E1050EAD
:1029C600BD5DD8B002D0010EAB6F6E0E0001E46F94
:1029D600280EE56F000EE66FABC1E7F0000EE96F5B
:1029E600010EE86F000EEB6F040EEA6F23EC61F048
:1029F6000009D8B41200000E0001A26F020EA16FEA
:102A0600BDC1A3F0BEC1A4F055EC6FF00001A15109
:102A16004C6E1200EC0E0001916F230E926F8EEC3D
:102A26006EF01200ECC095F0EDC096F0EEC097F097
:102A3600EFC098F0B60E0001996F010E9A6F8DECFB
:102A460071F00009D8B4F1D0000E0101AC6FB65197
:102A5600B711D8B408D0B75106E1090EB65DD8B0A3
:102A660002D0010EAC6F6A0E0001E46F280EE56F0E
:102A7600000EE66FACC1E7F0000EE96F010EE86FDD
:102A8600000EEB6F080EEA6F23EC61F00009D8B474
:102A96001200ECC095F0EDC096F0EEC097F0EFC0D6
:102AA60098F0B20E0001996F010E9A6F8DEC71F0DD
:102AB6000009D8B4B2D0000E0101AD6FB251B31106
:102AC600D8B408D0B35106E1090EB25DD8B002D031
:102AD600010EAD6F1C0E0001E46F280EE56F000EAF
:102AE600E66FADC1E7F0000EE96F010EE86F000E6C
:102AF600EB6F080EEA6F23EC61F00009D8B4120000
:102B0600ECC095F0EDC096F0EEC097F0EFC098F0EF
:102B1600B40E0001996F010E9A6F8DEC71F00009E9
:102B2600D8B473D0000E0101AE6FB451B511D8B44C
:102B360008D0B55106E10D0EB45DD8B002D0010E35
:102B4600AE6F990E0001E46F270EE56F000EE66F7B
:102B5600AEC1E7F0000EE96F010EE86F000EEB6FF5
:102B66000C0EEA6F23EC61F00009D8B41200B4C170
:102B7600F0F0FF0E0001F0270101AA510001F01943
:102B8600F00BF0190101AA6FB2C1F0F00001F03BA1
:102B96000101AA510001F0190F0BF0190101AA6FEA
:102BA600FF0EB6250001976FFF0E0101B721000148
:102BB600986F000E9A6F030E996F30EC71F06B0EE2
:102BC60000019725D96E010E9821DA6EFF0E0101DC
:102BD600B6250001976FFF0E0101B7210001986F1E
:102BE600000E9A6F030E996F30EC71F00C0E000117
:102BF60097259D6F000E98219E6FAAC19FF017EC36
:102C06006FF0DF6EB2EC6BF01200EC0E0001916F0C
:102C1600230E926F8EEC6EF01200EC0E0001916F97
:102C2600230E926F8EEC6EF01200EC0E0001916F87
:102C3600230E926F8EEC6EF01200ECC099F0EDC090
:102C46009AF0EEC09BF0EFC09CF0030E00019D6F62
:102C5600B90E9E6F010E9F6F44EC71F00009D8B457
:102C660052D00101BD69BE69BCBF07D0BC51BB11C2
:102C760013E1190EBA5DD8B00FD0B9C197F0BAC139
:102C860098F0000E00019A6F0A0E996F30EC71F001
:102C960097C0BDF198C0BEF1000E0101AF6F980E4E
:102CA600BD5D3A0EBE59D8A008D0110EBD5DA40E6A
:102CB600BE59D8B002D0010EAF6F210E0001E46FED
:102CC600290EE56F010EE66FAFC1E7F03A0EE96F28
:102CD600980EE86FA40EEB6F100EEA6F23EC61F00E
:102CE6000009D8B41200000E0001A26F040EA16FF5
:102CF600BDC1A3F0BEC1A4F055EC6FF0A1C03DF07C
:102D0600A2C03EF01200EC0E0001916F230E926FEE
:102D16008EEC6EF01200ECC099F0EDC09AF0EEC0A9
:102D26009BF0EFC09CF0030E00019D6FB90E9E6FE5
:102D3600010E9F6F44EC71F00009D8B44BD001012D
:102D4600BD69BE69BCBF07D0BC51BB1113E1190EEA
:102D5600BA5DD8B00FD0B9C197F0BAC198F0000EDD
:102D660000019A6F0A0E996F30EC71F097C0BDF1B1
:102D760098C0BEF1E10E0001E46F280EE56F010E6A
:102D8600E66F110E0101BD5DA40EBE59D8B002D08A
:102D9600010E01D0000E0001E76F000EE96F000E74
:102DA600E86FA40EEB6F100EEA6F23EC61F00009DA
:102DB600D8B41200000E0001A26F300EA16FBDC183
:102DC600A3F0BEC1A4F055EC6FF0A1C037F0A2C0CD
:102DD60038F01200EC0E0001916F230E926F8EEC0C
:102DE6006EF01200ECC099F0EDC09AF0EEC09BF0C8
:102DF600EFC09CF0030E00019D6FB90E9E6F010E91
:102E06009F6F44EC71F00009D8B452D00101BD693E
:102E1600BE69BCBF07D0BC51BB1113E1190EBA5D28
:102E2600D8B00FD0B9C197F0BAC198F0000E000122
:102E36009A6F0A0E996F30EC71F097C0BDF198C089
:102E4600BEF1000E0101B06F200EBD5D4E0EBE59E3
:102E5600D8A008D0210EBD5DCB0EBE59D8B002D089
:102E6600010EB06F1D0E0001E46F290EE56F010E15
:102E7600E66FB0C1E7F04E0EE96F200EE86FCB0E9D
:102E8600EB6F200EEA6F23EC61F00009D8B4120054
:102E9600000E0001A26F060EA16FBDC1A3F0BEC158
:102EA600A4F055EC6FF0A1C03BF0A2C03CF01200BC
:102EB600EC0E0001916F230E926F8EEC6EF01200F5
:102EC600ECC099F0EDC09AF0EEC09BF0EFC09CF01C
:102ED600030E00019D6FB90E9E6F010E9F6F44ECAD
:102EE60071F00009D8B44BD00101BD69BE69BCBF01
:102EF60007D0BC51BB1113E1190EBA5DD8B00FD083
:102F0600B9C197F0BAC198F0000E00019A6F0A0E87
:102F1600996F30EC71F097C0BDF198C0BEF1DC0E30
:102F26000001E46F280EE56F010EE66F210E010128
:102F3600BD5DCB0EBE59D8B002D0010E01D0000E39
:102F46000001E76F000EE96F000EE86FCB0EEB6F26
:102F5600200EEA6F23EC61F00009D8B41200000ECF
:102F66000001A26F2E0EA16FBDC1A3F0BEC1A4F0D9
:102F760055EC6FF0A1C039F0A2C03AF01200EC0E89
:102F86000001916F230E926F8EEC6EF01200ECC072
:102F960099F0EDC09AF0EEC09BF0EFC09CF0030EE6
:102FA60000019D6FB90E9E6F010E9F6F44EC71F08C
:102FB6000009D8B44BD00101BD69BE69BCBF07D0BA
:102FC600BC51BB1113E1190EBA5DD8B00FD0B9C10F
:102FD60097F0BAC198F0000E00019A6F0A0E996F29
:102FE60030EC71F097C0BDF198C0BEF1190E00012A
:102FF600E46F290EE56F010EE66FB10E0101BD5DAE
:10300600B30EBE59D8B002D0010E01D0000E000199
:10301600E76F4E0EE96F200EE86FB30EEB6FB00E42
:10302600EA6F23EC61F00009D8B41200000E00012B
:10303600A26F080EA16FBDC1A3F0BEC1A4F055ECEE
:103046006FF0A1C035F0A2C036F01200EC0E000100
:10305600916F230E926F8EEC6EF01200ECC099F019
:10306600EDC09AF0EEC09BF0EFC09CF0030E00019D
:103076009D6FB90E9E6F010E9F6F44EC71F00009B3
:10308600D8B44BD00101BD69BE69BCBF07D0BC51E5
:10309600BB1113E1190EBA5DD8B00FD0B9C197F0C4
:1030A600BAC198F0000E00019A6F0A0E996F30ECC3
:1030B60071F097C0BDF198C0BEF1A30E0001E46F98
:1030C600280EE56F010EE66FB10E0101BD5DB30E70
:1030D600BE59D8B002D0010E01D0000E0001E76F34
:1030E600000EE96F000EE86FB30EEB6FB00EEA6FDD
:1030F60023EC61F00009D8B41200000E0001A26FA3
:103106000A0EA16FBDC1A3F0BEC1A4F055EC6FF0CD
:10311600A1C03AF1A2C03BF11200EC0E0001916F82
:10312600230E926F8EEC6EF01200ECC095F0EDC09F
:1031360096F0EEC097F0EFC098F0BD0E0001996FC3
:10314600010E9A6F8DEC71F00009D8B42BD0A90E40
:103156000001E46F280EE56F000EE66F0101BE5117
:1031660006E1650EBD5DD8B002D0010E01D0000E9D
:103176000001E76F000EE96F000EE86F000EEB6FBF
:10318600640EEA6F23EC61F00009D8B41200000E59
:1031960000019E6F2C0E9D6FBDC19FF017EC6FF066
:1031A600446E1200EC0E0001916F230E926F8EECAE
:1031B6006EF01200EC0E0001916F230E926F8EECF2
:1031C6006EF01200ECC095F0EDC096F0EEC097F0F0
:1031D600EFC098F0EE0E0001996F260E9A6FB80EAA
:1031E6009B6F010E9C6FDFEC70F00009D8B41CD009
:1031F600B20E0001916F210E926F8EEC6EF00101FE
:10320600B805D8A404D0040E58EC72F01200030ED0
:103216000101B819D8A404D0060E58EC72F01200B9
:10322600050E58EC72F012008E0E0001916F230EFF
:10323600926F8EEC6EF01200040E58EC72F01200D3
:10324600ECC095F0EDC096F0EEC097F0EFC098F0A8
:10325600BD0E0001996F010E9A6F8DEC71F0000999
:10326600D8B427D0AB0E0001E46F270EE56F000E31
:10327600E66F0101BE05D8B002D0010E01D0000EE6
:103286000001E76F000EE96F000EE86F000EEB6FAE
:10329600EA6923EC61F00009D8B41200000E0001BF
:1032A6009E6F320E9D6FBDC19FF017EC6FF0476E9B
:1032B6001200EC0E0001916F230E926F8EEC6EF0F1
:1032C6001200ECC095F0EDC096F0EEC097F0EFC09E
:1032D60098F0BD0E0001996F010E9A6F8DEC71F09A
:1032E6000009D8B427D0A20E0001E46F270EE56FBF
:1032F600000EE66F0101BE05D8B002D0010E01D066
:10330600000E0001E76F000EE96F000EE86F000E79
:10331600EB6FEA6923EC61F00009D8B41200000EE5
:1033260000019E6F330E9D6FBDC19FF017EC6FF0CD
:10333600466E1200EC0E0001916F230E926F8EEC1A
:103346006EF01200ECC095F0EDC096F0EEC097F06E
:10335600EFC098F0EE0E0001996F260E9A6FB80E28
:103366009B6F010E9C6FDFEC70F00009D8B442D061
:10337600000E0101B16FB805D8A402D0020EB16FDC
:10338600020EB819D8A402D0030EB16F030EB819F5
:10339600D8A402D0040EB16FB1514818D8A408D0F1
:1033A600890E0001916F220E926F8EEC6EF0120064
:1033B600F70E0001916F220E926F8EEC6EF0000EEA
:1033C60000019E6F340E9D6FB1C19FF017EC6FF038
:1033D600486E000E0001916F000E906F000E936F05
:1033E600000E926F000E956F000E946F485023ECFE
:1033F60051F012008E0E0001916F230E926F8EEC2B
:103406006EF012000101B851000AD8B4C4EF14F0EE
:10341600010AD8B4C7EF14F0030AD8B415EF15F0B3
:10342600010AD8B40AD4070AD8B475D4010AD8B4A4
:10343600D9D4030AD8B444D5010AD8B4A8D50F0AFA
:10344600D8B40CD6010AD8B470D6030AD8B4B2D60A
:10345600010AD8B4B7D6070AD8B4EED6010AD8B44A
:10346600EFD6030AD8B42DD7010AD8A412006AD71A
:103476008E0E0001916F230E926F8EEC6EF012008D
:1034860055EC70F0010E0101B66F020E6419D8B446
:1034960006D0030E6419D8B402D0000EB66FB6C1BA
:1034A60095F04B50D2EC64F055EC70F055EC70F0A2
:1034B60055EC70F055EC70F0000E90EC6FF055EC9A
:1034C60070F055EC70F055EC70F055EC70F0000EA5
:1034D6000101BD6F060EBE6FBDC1BCF0BEC1BDF021
:1034E600D20E0001BE6F010EBF6F4B508BEC58F031
:1034F6004BC0DFF0010E0001E06FDF2B02D0D89049
:10350600E037DF2FFCD7FF0E0001E027E051010175
:10351600B76FB86BD251B7150001DF6FE06B0101D1
:10352600B7510001DF1906E10101B8510001E019A8
:10353600D8B43FD026C1BBF027C1BCF033C0BDF024
:1035460034C0BEF060EC53F06EEC72F090C0ACF19B
:1035560091C0ADF1060E01013C250001966F000EEB
:1035660001013D210001976F000E996F010E986FC2
:10357600BCEC68F0D20E0001966F010E976F000E3C
:10358600996F010E986F1BEC6EF0ACC196F0ADC151
:1035960097F0000E0001996F050E986FBCEC68F06D
:1035A600D20E0001916F1A0E926F8EEC6EF064EFE0
:1035B6001FF0000E0101DE6F050EDF6F000EDD6FDE
:1035C60063D0DEC1D9FFDFC1DAFFDECFE1F1DDCFA7
:1035D600E2F1BDC1D9FFBEC1DAFFDECFCFF1DDCF4B
:1035E600D0F1E151E211D8A404D0CFC1E1F1D0C1AC
:1035F600E2F12F0EE15DF80EE259D8B007D0D00EF9
:10360600E125B96F070EE221BA6F02D0B969BA692E
:10361600D10EE15D070EE259D8A007D0300EE125A4
:10362600BB6FF80EE221BC6F04D0000EBC6F000E1B
:10363600BB6FCF51B95DD051BA59D8B005D0B9C119
:10364600E1F1BAC1E2F10FD0BB51CF5DBC51D05907
:10365600D8B005D0BBC1E1F1BCC1E2F104D0CFC105
:10366600E1F1D0C1E2F1DEC1D9FFDFC1DAFFE1C18C
:10367600DEFFE2C1DDFF020EDE27000EDF23020EB3
:10368600BD27000EBE23DD2B4350DD5DD8A099D7A4
:1036960074EC72F0A90E0001BE6F010EBF6FA70E8B
:1036A600C06F010EC16F86EC3BF0BEC0BFF1BFC05C
:1036B600C0F1C0C0C1F1C1C0C2F1BFC130F1C0C1CB
:1036C60031F1000E0101DE6F050EDF6F600ED36F64
:1036D600070ED46F000EDD6F0AD1DEC1D9FFDFC140
:1036E600DAFFDECFDFF0DDCFE0F0A7C1E1F0A8C161
:1036F600E2F00001E11FE21FE14BE22BDF51E1277F
:10370600E051E223E1C0D6F1E2C0D7F10101000E9B
:10371600D7BFFF0ED86FD96F020EDE27000EDF234C
:10372600D9BF07D0D951D811D7111EE1D605D8B0C7
:103736001BD0D6C1DFF0D7C1E0F0D8C1E1F0D9C1C6
:10374600E2F00001DF1FE01FE11FE21FDF2B000E8A
:10375600E023E123E223DFC0AEF1E0C0AFF1E1C038
:10376600B0F1E2C0B1F108D0D6C1AEF1D7C1AFF128
:10377600D8C1B0F1D9C1B1F10101B1BF5CD0B1512D
:10378600B011AF1104E10A0EAE5DD8A054D0D9BF76
:1037960007D0D951D811D7111EE1D605D8B01BD004
:1037A600D6C1DFF0D7C1E0F0D8C1E1F0D9C1E2F06F
:1037B6000001DF1FE01FE11FE21FDF2B000EE023E9
:1037C600E123E223DFC0B2F1E0C0B3F1E1C0B4F11E
:1037D600E2C0B5F108D0D6C1B2F1D7C1B3F1D8C1B4
:1037E600B4F1D9C1B5F1BFC1B0F0C0C1B1F0C1C12A
:1037F600B2F0C2C1B3F00A0E0001B46F000EB56F8D
:10380600000EB66F000EB76FBCEC60F00001B05151
:103816000101B25D0001B1510101B3590001B2517C
:103826000101B459B551800A0001DF6FB351800A16
:10383600DF59D8B006D0000E0101CE6F000ECD6F55
:1038460029D0D6C1A4F0D7C1A5F0D8C1A6F0D9C158
:10385600A7F00A0E0001A86F000EA96F000EAA6F4E
:10386600000EAB6FC6EC6CF0A4C0B0F0A5C0B1F012
:10387600A6C0B2F0A7C0B3F0BFC1B4F0C0C1B5F0E6
:10388600C1C1B6F0C2C1B7F0BCEC60F0B0C0CDF1BA
:10389600B1C0CEF10101CEBF0AD0CE5104E1640E13
:1038A600CD5DD8A004D0000ECE6F630ECD6FCDC116
:1038B600DFF0CEC1E0F00001DF1FE01FDF4BE02BA1
:1038C600E0BF0BD0E05104E1640EDF5DD8A005D067
:1038D600FF0E0101CE6F9D0ECD6FD3C1D9FFD4C1AE
:1038E600DAFFCDC1DFFF0101D34BD42BDD2B4350D3
:1038F600DD5DD8A0F2D62A512B11D8B471D030C1D3
:103906002EF131C12FF130C12CF131C12DF1A7C1FA
:1039160034F1A8C135F1A7C132F1A8C133F1000EC7
:10392600DE6F050EDF6F000EC56F090EC66F000E47
:10393600C76F0A0EC86F600ED36F070ED46F000EE6
:10394600C96F070ECA6F000ECB6F080ECC6F000E44
:10395600DD6F3FD0DEC1D9FFDFC1DAFFC5C1E1FFB0
:10396600C6C1E2FFDECFE6FFDDCFE5FF020EC527CB
:10397600000EC623DEC1D9FFDFC1DAFFC7C1E1FFF2
:10398600C8C1E2FFDECFE6FFDDCFE5FF020EDE2790
:10399600000EDF23020EC727000EC823D3C1D9FFAE
:1039A600D4C1DAFFC9C1E1FFCAC1E2FFDFCFE7FF39
:1039B600C94BCA2BD3C1D9FFD4C1DAFFCBC1E1FFB2
:1039C600CCC1E2FFDFCFE7FFD34BD42BCB4BCC2BC5
:1039D600DD2B4350DD5DD8A0BDD72A07D8A02B0725
:1039E6002A512B11D8A46DD23451A75D3551A8594F
:1039F600D8B004D0A7C134F1A8C135F1A751325DC2
:103A0600A8513359D8B004D0A7C132F1A8C133F1B7
:103A16002E51305D2F513159D8B004D030C12EF11E
:103A260031C12FF130512C5D31512D59D8B004D010
:103A360030C12CF131C12DF1000EDE6F050EDF6FA6
:103A4600000EC56F090EC66F000EC76F0A0EC86F4F
:103A5600600ED36F070ED46F000EC96F070ECA6FC4
:103A6600000ECB6F080ECC6F000EDD6F6FD0DEC17F
:103A7600D9FFDFC1DAFFDECFE1F1DDCFE2F1020EE1
:103A8600DE27000EDF23C5C1D9FFC6C1DAFFDE502F
:103A9600E15DDE50E259D8B008D0C5C1D9FFC6C134
:103AA600DAFFE1C1DEFFE2C1DDFFC7C1D9FFC8C150
:103AB600DAFFE151DE5CE251DE58D8B008D0C7C16A
:103AC600D9FFC8C1DAFFE1C1DEFFE2C1DDFF020EA8
:103AD600C527000EC623020EC727000EC823D3C172
:103AE600D9FFD4C1DAFFDF50D16FD34BD42BC9C174
:103AF600D9FFCAC1DAFFDE50800A0001E06F01017A
:103B0600D151800A0001E05DD8B006D0C9C1D9FF05
:103B1600CAC1DAFFD1C1DFFFCBC1D9FFCCC1DAFF01
:103B26000101D151800A0001E06FDE50800AE05D9C
:103B3600D8B006D0CBC1D9FFCCC1DAFFD1C1DFFFE7
:103B46000101C94BCA2BCB4BCC2BDD2B4350DD5D82
:103B5600D8A08DD7000EDC6F000EDE6F050EDF6F6E
:103B6600000ED56F000EE06F000EDD6F80D1D551CF
:103B76000D0D4C0EF324DA6F020EF420DB6FD551D7
:103B8600030D010EF326000EF4226B0EF324D96EFC
:103B9600010EF420DA6EDF50AA6F20EE02F0DA5141
:103BA600D926DB51DA22DECFDFF0DDCFE0F0E0C14F
:103BB600E1F0010E0001E26F000EE36FE12B03D08E
:103BC600D890E237E337E12FFBD70001DF51E21748
:103BD600E051E317E251E311D8B402D0010E01D04F
:103BE600000E0101AB6F20EE06F0DA51D926DB514B
:103BF600DA22DECFDFF0DDCFE0F0E0C1E1F0010E4A
:103C06000001E26F000EE36FE12B03D0D890E2379C
:103C1600E337E12FFBD70001DF51E217E051E3174D
:103C2600E251E311D8B402D0010E01D0000E010119
:103C3600C36F20EE08F0DA51D926DB51DA22DECF47
:103C4600DFF0DDCFE0F0E0C1E1F0010E0001E26F50
:103C5600000EE36FE12B03D0D890E237E337E12F74
:103C6600FBD70001DF51E217E051E317E251E31100
:103C7600D8B402D0010E01D0000E0101C46FDEC11E
:103C8600D9FFDFC1DAFFDECFE1F1DDCFE2F1020ECF
:103C9600DE27000EDF23E25104E1C90EE15DD8A064
:103CA600DCD03D50E15D3E50E259D8B02CD0C45135
:103CB600D8A40CD0E0C1BEF0D55146EC68F0E20EB7
:103CC6000001916F260E926F8EEC6EF0E0C1DFF070
:103CD600010E0001E06F000EE16FDF2B03D0D890DC
:103CE600E037E137DF2FFBD7010120EE08F0DA518C
:103CF600D926DB51DA220001E051DE12E151DD1254
:103D06000101DC83AAD0E1513B5CE2513C58D8B0BA
:103D16002CD0C351D8A40CD0E0C1BEF0D55146EC8E
:103D260068F0D60E0001916F260E926F8EEC6EF043
:103D3600E0C1DFF0010E0001E06F000EE16FDF2B46
:103D460003D0D890E037E137DF2FFBD7010120EE13
:103D560006F0DA51D926DB51DA220001E051DE12F3
:103D6600E151DD120101DC8178D0C351D8B40CD009
:103D760039503A10D8B408D0E151395CE2513A587A
:103D8600D8B002D0DC815ED0C451D8B40CD0375044
:103D96003810D8B408D03750E15D3850E259D8B061
:103DA60002D0DC834FD0C351D8A403D0C451D8B4B9
:103DB60049D0E0C1BEF0D55146EC68F0820E000154
:103DC600916F260E926F8EEC6EF0E0C1DFF0010E61
:103DD6000001E06F000EE16FDF2B03D0D890E037D3
:103DE600E137DF2FFBD70001E01DE26FE11DE36F36
:103DF600010120EE06F0DA51D926DB51DA22000164
:103E0600E251DE16E351DD16E0C1DFF0010EE06F90
:103E1600000EE16FDF2B03D0D890E037E137DF2FBC
:103E2600FBD70001E01DE26FE11DE36F010120EE0B
:103E360008F0DA51D926DB51DA220001E251DE160A
:103E4600E351DD1635503610D8B407D00101E151E3
:103E5600355CE2513658D8A0DC850101E02B0C0E0A
:103E6600E019D8A403D0D52B000EE06FDD2B43500C
:103E7600DD5DD8A07CD6DC516519D8B422D065A109
:103E8600DCA106D04650400DF3CF3EF1F4CF3FF112
:103E960065B1DCB104D0000E3F6F000E3E6F65A326
:103EA600DCA306D04750400DF3CF40F1F4CF41F1EB
:103EB60065B3DCB304D0000E416F000E406FDCC169
:103EC60065F10101284B292B12004B505FEC25F0C0
:103ED600010E90EC6FF00D0E0001986FAC0E976F0F
:103EE6003BEC70F0000E0001BC6F060EBD6FF00ECD
:103EF600BE6F000EBF6F4B508BEC58F013EC56F0B4
:103F060001016151D8B434D0750E0001916F270EAE
:103F1600926F8EEC6EF0FE0E0001916F250E926F81
:103F26008EEC6EF000C2DEF001C2DFF002C2E0F0FD
:103F360003C2E1F0F50E0001E26F280EE36F66ECB6
:103F460069F0F00E0001916F250E926F8EEC6EF007
:103F560034C2B8F00001B96B010EBA6FADEC6FF068
:103F6600D20E0001916F1A0E926F8EEC6EF08AD00F
:103F7600000E0001F26F070EF26501D067D0F25114
:103F8600040D000EF324D96E020EF420DA6EDE5014
:103F9600DE10DE10DE10D8B456D0710E916F280EEA
:103FA600926F8EEC6EF0010E0001F225B86FB96BC0
:103FB600000EB923010EBA6FADEC6FF0D20E000100
:103FC600916F1A0E926F8EEC6EF0FE0E0001916FDD
:103FD600250E926F8EEC6EF00001F251040D000E6C
:103FE600F324D96E020EF420DA6EDECFDEF0DECFD9
:103FF600DFF0DECFE0F0DECFE1F0F50EE26F280E67
:10400600E36F66EC69F0F00E0001916F250E926F7A
:104016008EEC6EF00001F251010D340EF324D96ED0
:10402600020EF420DA6EDF50E46FE451B86FB96B1C
:10403600010EBA6FADEC6FF0D20E0001916F1A0E41
:10404600926F8EEC6EF00001F22B95D7570E916FA2
:10405600270E926F8EEC6EF0F00E0001916F250E1A
:10406600926F8EEC6EF062C1B8F00001B96B010E72
:10407600BA6FADEC6FF0D20E0001916F1A0E926F0F
:104086008EEC6EF0950E0001916F260E926F8EECFF
:104096006EF0A7C1DEF0A8C1DFF0F50E0001E06FFB
:1040A600280EE16F80EC6BF0A20E0001916F260ED8
:1040B600926F8EEC6EF030C1DEF031C1DFF0F50E9E
:1040C6000001E06F280EE16F80EC6BF04AA43DD151
:1040D600B80E0001916F250E926F8EEC6EF028C11E
:1040E600B8F029C1B9F0010E0001BA6FADEC6FF05E
:1040F600D20E0001916F1A0E926F8EEC6EF0C60E04
:104106000001916F250E926F8EEC6EF09D0E0001F0
:10411600916F280E926F8EEC6EF03CC1D9FF3DC1B7
:10412600DAFFDF500001E46FE451B86FB96B010E9E
:10413600BA6FADEC6FF0900E0001916F270E926F83
:104146008EEC6EF0010120EE01F03C51D9263D5176
:10415600DA22DF500001E46FE451B86FB96B010E4B
:10416600BA6FADEC6FF0140E0001916F280E926FCE
:104176008EEC6EF0010120EE02F03C51D9263D5145
:10418600DA22DF500001E46FE451B86FB96B010E1B
:10419600BA6FADEC6FF00C0E0001916F280E926FA6
:1041A6008EEC6EF0010120EE03F03C51D9263D5114
:1041B600DA22DF500001E46FE451B86FB96B010EEB
:1041C600BA6FADEC6FF05C0E0001916F280E926F26
:1041D6008EEC6EF0010120EE04F03C51D9263D51E3
:1041E600DA22DF500001E46FE451B86FB96B010EBB
:1041F600BA6FADEC6FF0610E0001916F270E926FF2
:104206008EEC6EF0010120EE05F03C51D9263D51B1
:10421600DA22DF500001E46FE451B86FB96B010E8A
:10422600BA6FADEC6FF0D20E0001916F1A0E926F5D
:104236008EEC6EF0000E0001F16F83D06B0E916F65
:10424600270E926F8EEC6EF0010E0001F125B86F0D
:10425600B96B000EB923010EBA6FADEC6FF0550EB7
:104266000001916F280E926F8EEC6EF00001F151F5
:10427600030D080EF326000EF422F35001013C252F
:10428600D96EF4503D21DA6EDF500001E46FE4513F
:10429600B86FB96B010EBA6FADEC6FF01E0E000170
:1042A600916F270E926F8EEC6EF00001F151030DA7
:1042B600080EF326000EF4223CC1E4F03DC1E5F001
:1042C600F350E427F450E523020EE425D96E000EE0
:1042D600E521DA6EDF50E66FE651B86FB96B010E75
:1042E600BA6FADEC6FF04C0E0001916F270E926F16
:1042F6008EEC6EF00001F151030D080EF326000E50
:10430600F4223CC1E4F03DC1E5F0F350E427F4505B
:10431600E523010EE425D96E000EE521DA6EDF50A5
:10432600E66FE651B86FB96B010EBA6FADEC6FF080
:10433600D20E0001916F1A0E926F8EEC6EF0000194
:10434600F12B4B50F15DD8A079D7E20E0001916FA9
:10435600250E926F8EEC6EF0000E0101606F000E5E
:104366000001F16F52D0F1510D0D0B0EF326000E28
:10437600F4224C0EF324D96E020EF420DA6EDE50CF
:10438600DE10D8B440D09EEC71F0110E0001916F92
:10439600290E926F8EEC6EF0010E0001F125B86FBA
:1043A600B96B000EB923010EBA6FADEC6FF07E0E3D
:1043B6000001916F270E926F8EEC6EF00001F151A5
:1043C6000D0D0B0EF326000EF4224C0EF324D96EBF
:1043D600020EF420DA6EDECF90F0DDCF91F0E80E1B
:1043E600926F000E936FB5EC62F0E80E0001916FCC
:1043F600000E926F8EEC6EF03E0E0001916F1D0E58
:10440600926F8EEC6EF00001F12B4B50F15DD8A04F
:10441600AAD742A209D09EEC71F09C0E0001916FC2
:10442600250E926F8EEC6EF042A609D09EEC71F0CE
:10443600700E0001916F240E926F8EEC6EF042A406
:1044460009D09EEC71F0300E0001916F240E926F30
:104456008EEC6EF0010165A109D09EEC71F0850E1F
:104466000001916F280E926F8EEC6EF0010165A32C
:1044760009D09EEC71F08B0E0001916F280E926FA1
:104486008EEC6EF0010165A509D09EEC71F07F0EF1
:104496000001916F280E926F8EEC6EF0020E0101F4
:1044A6006419D8B404D0030E6419D8A409D09EECBC
:1044B60071F08E0E0001916F250E926F8EEC6EF0EC
:1044C60042A009D09EEC71F0DC0E0001916F220E25
:1044D600926F8EEC6EF001016051D8A407D02B0EBE
:1044E6000001916F280E926F8EEC6EF049A433D0C6
:1044F600AA0E0001916F250E926F8EEC6EF08FEC76
:1045060072F00001F26FF251D8B403D0F229D8A4A8
:1045160007D0AF0E916F260E926F8EEC6EF014D010
:10452600050E0001F219D8A407D02A0E916F270EA6
:10453600926F8EEC6EF008D0F2C0B8F00001B96B45
:10454600010EBA6FADEC6FF0D20E0001916F1A0E2C
:10455600926F8EEC6EF0D40E0001916F250E926F65
:104566008EEC6EF0F4EC57F012000001AC6F000E0A
:104576000001916F020E906F28EC72F04C6E0001F4
:10458600AC51D8A406D04C50D8B403D0040E4C6419
:1045960009D0000E9E6F020E9D6F010E9F6F17ECE5
:1045A6006FF04C6E000E0001916F000E906F28ECBC
:1045B60072F04A6E0001AC51D8A403D04A28D8A4A0
:1045C6000AD0000E4A6E000E9E6F000E9D6F000E02
:1045D6009F6F17EC6FF0000E0001916F010E906F48
:1045E60028EC72F0496E0001AC51D8A403D04928DA
:1045F600D8A40AD0000E496E000E9E6F010E9D6F64
:1046060049C09FF017EC6FF0000E0001916F2C0E61
:10461600906F28EC72F0446E0001AC51D8A403D020
:10462600640E446409D0000E9E6F2C0E9D6F320EF0
:104636009F6F17EC6FF0446E000E0001916F2D0E08
:10464600906F28EC72F00101676F0001AC51D8B48D
:104656000AD0000E9E6F2D0E9D6F000E9F6F17ECF9
:104666006FF00101676F000E0001916F320E906FBF
:1046760028EC72F0476E0001AC51D8A403D047284D
:10468600D8A409D0000E9E6F320E9D6F000E9F6F4C
:1046960017EC6FF0476E000E0001916F330E906FAE
:1046A60028EC72F0466E0001AC51D8A403D046281F
:1046B600D8A409D0000E9E6F330E9D6F000E9F6F1B
:1046C60017EC6FF0466E000E0001916F340E906F7E
:1046D60028EC72F00001AB6FAC51D8A40CD0020EDE
:1046E600AB19D8B412D0030EAB19D8B40ED0040E41
:1046F600AB19D8B40AD0000E9E6F340E9D6F030E10
:104706009F6F17EC6FF00001AB6FABC048F0000E67
:10471600936F040E926FCAEC6FF092C03DF093C097
:104726003EF00001AC51D8A40CD0980E3D5C3A0E78
:104736003E58D8A006D0110E3D5CA40E3E58D8A017
:104746000ED0000EA26F040EA16F5D0EA46FC00EF8
:10475600A36F55EC6FF0A1C03DF0A2C03EF0000E75
:104766000001936F060E926FCAEC6FF092C03BF099
:1047760093C03CF00001AC51D8A40CD0200E3B5C99
:104786004E0E3C58D8A006D0210E3B5CCB0E3C58B2
:10479600D8A00ED0000EA26F060EA16F840EA46FD5
:1047A600D00EA36F55EC6FF0A1C03BF0A2C03CF059
:1047B600000E0001936F2E0E926FCAEC6FF092C03E
:1047C60039F093C03AF00001AC51D8A406D0210EBE
:1047D600395CCB0E3A58D8A00ED0000EA26F2E0E22
:1047E600A16F000EA46F000EA36F55EC6FF0A1C071
:1047F60039F0A2C03AF0000E0001936F300E926FAE
:10480600CAEC6FF092C037F093C038F00001AC519B
:10481600D8A406D0110E375CA40E3858D8A00ED0F6
:10482600000EA26F300EA16F000EA46F000EA36FD4
:1048360055EC6FF0A1C037F0A2C038F0000E0001B1
:10484600936F080E926FCAEC6FF092C035F093C06A
:1048560036F00001AC51D8A406D0B10E355CB30ECB
:104866003658D8A00ED0000EA26F080EA16F000E0B
:10487600A46F000EA36F55EC6FF0A1C035F0A2C077
:1048860036F0000E0001936F0A0E926FCAEC6FF0BD
:1048960092C03AF193C03BF10001AC51D8A407D0C5
:1048A600B10E01013A5DB30E3B59D8A00FD0000EF0
:1048B6000001A26F0A0EA16F750EA46F300EA36FD2
:1048C60055EC6FF0A1C03AF1A2C03BF1000E000119
:1048D600A76F6B0EA86F010EA96F0C0EAA6F000EC4
:1048E600AD6F070EAD6501D034D0AAC090F0916BC4
:1048F60028EC72F00001A66FA629D8A403D0010EF9
:10490600A76F25D0A8C0D9FFA9C0DAFFA6C0DFFFD0
:10491600A84BA92BAA2BAAC090F0916B28EC72F099
:10492600A8C0D9FFA9C0DAFFDF6E0001AA2BA84BE9
:10493600A92BAAC090F0916B28EC72F0A8C0D9FF01
:10494600A9C0DAFFDF6E0001AA2BA84BA92BAD2B5D
:10495600C8D7AC51D8A403D0A751D8B454D0000EB0
:10496600AD6F070EAD6501D031D0AD51030D6B0EA5
:10497600F324D96E010EF420DA6E0101DF500F0B1D
:104986001009DF6E0001AD51030D6B0EF324D96ED5
:10499600010EF420DA6E0101DF500001AD19F00BB3
:1049A600AD190101DF6E0001AD51030D010EF326B5
:1049B600000EF4226B0EF324D96E010EF420DA6E8B
:1049C600000EDE6E000EDD6EAD2BCBD76B0EA86F24
:1049D600010EA96F0C0EAA6F000EAD6F170EAD6516
:1049E60001D011D0AAC09DF09E6BA8C0D9FFA9C066
:1049F600DAFFDF509F6F17EC6FF00001AA2BA84B70
:104A0600A92BAD2BEBD7240EAA6F000EAD6F070EA8
:104A1600AD6501D01ED0240EAD25906F916B000EB2
:104A2600912328EC72F00001AB6FABC0A5F0E00E4D
:104A3600A517D8B402D0010EA76FAD51010D000E17
:104A4600F324D96E010EF420DA6EABC0DFFFAD2B76
:104A5600DED7AC51D8A403D0A751D8B41CD0000ED1
:104A6600AD6F070EAD6501D016D0AD51010D000E2C
:104A7600F324D96E010EF420DA6E240EAD259D6F57
:104A86009E6B000E9E23000E9F6F17EC6FF0DF6E7D
:104A96000001AD2BE6D7B2EC6BF001016C516D1144
:104AA600D8B4428049A604D0938292909292120082
:104AB60092809282939212000001D26F55EC70F0B0
:104AC60055EC70F055EC70F055EC70F0ECEC71F0C4
:104AD60055EC70F055EC70F055EC70F055EC70F04C
:104AE600400E0001BC6F040EBD6FD2514EEC67F054
:104AF600000E0001D36F34D0D3510D0D0B0EF326EB
:104B0600000EF4224C0EF324D96E020EF420DA6E57
:104B1600000EDE6E000EDD6ED351060D710EF3240F
:104B2600CC6F040EF420CD6F20EE05F0CC51D926C3
:104B3600CD51DA22DF50C46FD890C433C4A10ED051
:104B4600D3510D0D0B0EF326000EF4224C0EF3245A
:104B5600D96E020EF420DA6E0201DF800001D32B3B
:104B6600D251D35DD8A0C8D7D4EC71F055EC70F013
:104B760055EC70F055EC70F055EC70F0400E0001FD
:104B8600BC6F040EBD6FD2514EEC67F010EC72F0A4
:104B960055EC70F055EC70F055EC70F055EC70F08B
:104BA600280E0001BC6F030EBD6FD25145EC6AF0B2
:104BB600000E0001D36FC3D0D351060D410EF3246E
:104BC600D06F040EF420D16FD351060D710EF3246D
:104BD600CC6F040EF420CD6FD351060D590EF3247D
:104BE600C96F030EF420CA6FD0C0D9FFD1C0DAFF57
:104BF600550EDE1804E1950EDE18D8B40ED0D3514A
:104C06000D0D0B0EF326000EF4224C0EF324D96E76
:104C1600020EF420DA6E0201DF84000120EE02F0BB
:104C2600D051D926D151DA22550EDE1804E1950E5F
:104C3600DE18D8B40ED0D3510D0D0B0EF326000E90
:104C4600F4224C0EF324D96E020EF420DA6E020121
:104C5600DF86000120EE04F0D051D926D151DA22A8
:104C6600550EDE1804E1950EDE18D8B40ED0D351D9
:104C76000D0D0B0EF326000EF4224C0EF324D96E06
:104C8600020EF420DA6E0201DF88CCC0D9FFCDC057
:104C9600DAFF550EDE1804E1950EDE18D8B40FD0F3
:104CA6000001D3510D0D0B0EF326000EF4224C0E0F
:104CB600F324D96E020EF420DA6E0201DF8A0001B7
:104CC60020EE05F0CC51D926CD51DA22DFA00ED048
:104CD600D3510D0D0B0EF326000EF4224C0EF324C9
:104CE600D96E020EF420DA6E0201DF82000120EE98
:104CF60004F0C951D926CA51DA22C70EDE5C750EF8
:104D0600DE58D8B00CD020EE04F0C951D926CA51CD
:104D1600DA229A0EDE5C740EDE58D8B00ED0D3516D
:104D26000D0D0C0EF326000EF4224C0EF324D96E54
:104D3600020EF420DA6E0201DF880001D32BD25175
:104D4600D35DD8A039D7C8EC71F055EC70F055ECAE
:104D560070F055EC70F055EC70F0400E0001BC6F31
:104D6600040EBD6FD2514EEC67F0000E0001D36FFA
:104D76007DD0D351060D410EF324D06F040EF420DE
:104D8600D16FD351060D710EF324CC6F040EF420AF
:104D9600CD6FD0C0D9FFD1C0DAFFAA0EDE1804E16C
:104DA6006A0EDE18D8B40ED0D3510D0D0B0EF326B5
:104DB600000EF4224C0EF324D96E020EF420DA6EA5
:104DC6000201DF8E000120EE02F0D051D926D1512A
:104DD600DA22AA0EDE1804E16A0EDE18D8B40ED066
:104DE600D3510D0D0C0EF326000EF4224C0EF324B7
:104DF600D96E020EF420DA6E0201DF80000120EE89
:104E060004F0D051D926D151DA22AA0EDE1804E1D7
:104E16006A0EDE18D8B40ED0D3510D0D0C0EF32643
:104E2600000EF4224C0EF324D96E020EF420DA6E34
:104E36000201DF82CCC0D9FFCDC0DAFFAA0EDE1890
:104E460004E16A0EDE18D8B40FD00001D3510D0D5F
:104E56000C0EF326000EF4224C0EF324D96E020E2D
:104E6600F420DA6E0201DF840001D32BD251D35D28
:104E7600D8A07FD704EC72F055EC70F055EC70F0CA
:104E860055EC70F055EC70F0000E0001BC6F060E8C
:104E9600BD6FCB0EBE6F000EBF6FD2518BEC58F0BC
:104EA600000E0001CE6F000ED36F39D0CEC0CFF00A
:104EB6001FD0CF51020D000EF324D96E060EF4203A
:104EC600DA6E550EDE1804E1950EDE18D8B40ED053
:104ED600D3510D0D0B0EF326000EF4224C0EF324C7
:104EE600D96E020EF420DA6E0201DF8C0001CF2BA0
:104EF600CE51C46FC56B0C0EC427000EC523CF510F
:104F0600C66FC76BC451C65DC751800AC86FC5510D
:104F1600800AC859D8A0CDD70C0ECE27D32BD25194
:104F2600D35DD8A0C3D7F8EC71F055EC70F055EC12
:104F360070F055EC70F055EC70F0000E0001BC6F8F
:104F4600060EBD6FCB0EBE6F000EBF6FD2518BEC3F
:104F560058F0000E0001CE6F000ED36F39D0CEC0D0
:104F6600CFF01FD0CF51020D000EF324D96E060EDE
:104F7600F420DA6EAA0EDE1804E16A0EDE18D8B442
:104F86000ED0D3510D0D0C0EF326000EF4224C0E4E
:104F9600F324D96E020EF420DA6E0201DF860001D8
:104FA600CF2BCE51C46FC56B0C0EC427000EC52384
:104FB600CF51C66FC76BC451C65DC751800AC86F53
:104FC600C551800AC859D8A0CDD70C0ECE27D32BF1
:104FD600D251D35DD8A0C3D7D251CAEC70F012001B
:104FE60002014CB10DD001016C516D11D8A408D04D
:104FF6005C0E0001916F240E926F8EEC6EF0120023
:10500600000E0101AD6F6B390F0BB46F010EB86F57
:10501600070EB86501D02ED0B8510D0D4C0EF324F5
:10502600D96E020EF420DA6E0201DFB011D0010152
:10503600B851030D010EF326000EF4226B0EF32475
:10504600D96E010EF420DA6EDE50DE10D8B410D020
:105056000101B851030D6B0EF324D96E010EF42035
:10506600DA6EDF380F0BB419D8B402D0010EAD6F6B
:10507600B82BCED7000E3BD2AF69B069B169B26921
:10508600000EBA6F030EBA6501D06CD0000EB36F76
:1050960056D0B551010D3C0EF324D96E020EF42004
:1050A600DA6EDF50BB6F080EBB6146D0BB510D0DEB
:1050B6004C0EF324D96E020EF420DA6E0201DFB034
:1050C60011D00101BB51030D010EF326000EF4228F
:1050D6006B0EF324D96E010EF420DA6EDE50DE106C
:1050E600D8B42AD00101BA51D8A40CD0BB51030DB3
:1050F6006B0EF324D96E010EF420DA6EDF380F0B37
:10510600B46F0DD0BB51030D6B0EF324D96E010E97
:10511600F420DA6EDF380F0BB419D8A40BD0BA51CD
:10512600010DAF0EF324D96E010EF420DA6EBBC169
:10513600DFFF02D0010EB36FB351D8B4B52BBA510D
:10514600010DAF0EF324D96E010EF420DA6EDE28BF
:10515600D8A406D0080EB56103D0B351D8B499D7F8
:10516600BA2B90D7AF29D8B4C1D1AD51D8B417D086
:10517600970E0001916F280E926F8EEC6EF0B4C1FF
:10518600B8F00001B96B010EBA6FADEC6FF0800E8E
:105196000001916F250E926F8EEC6EF00CD04B5085
:1051A6000101B55DD8B007D03D0E0001916F1C0E10
:1051B600926F8EEC6EF0000E0101B96F0B0EB965A1
:1051C60001D096D1000EBA6F030EBA6501D082D116
:1051D600BA51010DAF0EF324D96E010EF420DA6E2A
:1051E600DF50BB6FBB29D8B472D1BB51030D6B0E18
:1051F600F324D96E010EF420DA6EDF380F0BB46F8C
:10520600BB51030D6B0EF324D96E010EF420DA6E3A
:10521600DF500F0BAA6FAA510C0DF350B9250001F0
:10522600F46FF4290101AB6FBB510C0DF350B92596
:10523600AE6FB929AC6FAE51020D000EF324D96ED4
:10524600050EF420DA6EDECFB6F1DDCFB7F1E80E4B
:105256000001916F240E926F8EEC6EF04C0E0001E1
:10526600BB6F290EBC6F0101AB51D4EC6EF001018E
:10527600BB510D0D4C0EF324D96E020EF420DA6EDE
:105286000201DFA0ECD00101B7510CE1C80EB65DFA
:10529600D8B008D0F90E0001916F240E926F8EECF3
:1052A6006EF015D1B6C1DEF0B7C1DFF0500E0001C9
:1052B600E06F290EE16F80EC6BF00101BB510D0D23
:1052C600040EF326000EF4224C0EF324D96E020EC1
:1052D600F420DA6EDECFF4F0DDCFF5F0B9C1F6F0EA
:1052E600010E0001F76F000EF86FF62B03D0D89071
:1052F600F737F837F62FFBD70001F451F717F551BA
:10530600F817F751F811D8B407D0FC0E916F270E95
:10531600926F8EEC6EF0DBD03B500101B65D3C50D7
:10532600B759D8A008D0CC0E0001916F270E926F06
:105336008EEC6EF0CCD00101BB510D0D060EF3269E
:10534600000EF4224C0EF324D96E020EF420DA6E0F
:10535600DECFF4F0DDCFF5F0B9C1F6F0010E0001B5
:10536600F76F000EF86FF62B03D0D890F737F837A3
:10537600F62FFBD70001F451F717F551F817F7513F
:10538600F811D8B407D0EC0E916F270E926F8EEC01
:105396006EF09DD035503610D8B40FD0355001017F
:1053A600B65D3650B759D8A008D0C40E0001916F2B
:1053B600270E926F8EEC6EF08AD00101B6513D5CDD
:1053C600B7513E58D8A008D0D40E0001916F270ED1
:1053D600926F8EEC6EF07BD00101BB510D0D080E65
:1053E600F326000EF4224C0EF324D96E020EF4209E
:1053F600DA6EDECFF4F0DDCFF5F0B9C1F6F0010ECE
:105406000001F76F000EF86FF62B03D0D890F73730
:10541600F837F62FFBD70001F451F717F551F817B7
:10542600F751F811D8B407D0F40E916F270E926F8A
:105436008EEC6EF04CD00101AE51010D600EF324DE
:10544600D96E070EF420DA6EDF5053EC62F0E60EEA
:105456000001916F240E926F8EEC6EF038D0010130
:10546600BB51030D010EF326000EF4226B0EF3243E
:10547600D96E010EF420DA6EDECFF4F0DDCFF5F052
:10548600ACC1F6F0FF0E0001F627010EF76F000E15
:10549600F86FF62B03D0D890F737F837F62FFBD7EF
:1054A6000001F451F717F551F817F751F811D8B470
:1054B60007D0EA0E916F240E926F8EEC6EF007D035
:1054C600DB0E0001916F240E926F8EEC6EF00101DF
:1054D600BA2B7AD6D20E0001916F1A0E926F8EEC0D
:1054E6006EF07CEC6AF00101B92B68D6080EB56F38
:1054F600070EB565C1D51200000E00019B6F080EA0
:105506009EEC69F04B505FEC25F0010E90EC6FF0CD
:10551600070E0001986FD00E976F3BEC70F0000EEF
:105526000001BC6F060EBD6FCE0EBE6F010EBF6FC3
:105536004B508BEC58F010EC72F0070E0001986F90
:10554600D00E976F3BEC70F0280E0001BC6F030E77
:10555600BD6F4B5045EC6AF0510E0001916F1C0E69
:10556600926F8EEC6EF0FD0E0001916F1B0E926F26
:105576008EEC6EF0000E0101D16F070ED16501D0E1
:1055860012004B50D15DD8A010D0D151030D010EA1
:10559600F326000EF4226B0EF324D96E010EF420CE
:1055A600DA6EDE50DE10D8B416D2D151060D410E99
:1055B600F324CF6F040EF420D06FD151060D710E77
:1055C600F324C86F040EF420C96FD151060D290EBD
:1055D600F324BE6F030EF420BF6FD151060D590E92
:1055E600F324CA6F030EF420CB6FE70E0001916F10
:1055F600240E926F8EEC6EF0010E0101D125000192
:10560600B86FB96B000EB923010EBA6FADEC6FF02F
:10561600940E0001916F240E926F8EEC6EF04B503B
:105626000101D15DD8B0C9D1D1510D0D0B0EF326B4
:10563600000EF4224C0EF324D96E020EF420DA6E1C
:10564600DE50DE10D8A408D0470E0001916F280E58
:10565600926F8EEC6EF01FD00101D1510D0D0B0E25
:10566600F326000EF4224C0EF324D96E020EF4201B
:10567600DA6EDECF90F0DDCF91F0AA0E0001926FC8
:10568600010E936FB5EC62F0AA0E0001916F010E48
:10569600926F8EEC6EF00101D151060D410EF3248E
:1056A600CF6F040EF420D06FD151060D710EF32486
:1056B600C86F040EF420C96FD151060D290EF324CC
:1056C600BE6F030EF420BF6FD151060D590EF324A1
:1056D600CA6F030EF420CB6FD1510D0D010EF326C8
:1056E600000EF4224C0EF324D96E020EF420DA6E6C
:1056F600DF50CC6F940E0001916F240E926F8EECEA
:105706006EF0CCC1B8F00001B96B010EBA6FADEC0A
:105716006FF07C0E0001916F280E926F8EEC6EF08A
:10572600010120EE04F0CF51D926D051DA22DECF86
:10573600DEF0DDCFDFF0450E0001E06F290EE16FF0
:1057460080EC6BF0C8C1D9FFC9C1DAFFDECFDEF04D
:10575600DDCFDFF0450E0001E06F290EE16F80EC32
:105766006BF0010120EE04F0CA51D926CB51DA22A2
:10577600DECFDEF0DDCFDFF0450E0001E06F290E53
:10578600E16F80EC6BF0040E0101CC6102D04AA4FB
:1057960017D020EE02F0CF51D926D051DA22DECF33
:1057A60097F0DDCF98F0F3EC6DF097C0C0F198C09C
:1057B600C1F1C0C1BBF0C1C1BCF0E3EC6BF007D0D6
:1057C600E50E0001916F240E926F8EEC6EF0C30E03
:1057D6000001916F280E926F8EEC6EF0CFC1D9FF4B
:1057E600D0C1DAFFDECFF0F0DDCFF1F0020E00011E
:1057F600F025906F000EF121916F000E936F050E4C
:10580600926FA0EC6DF090C0C2F191C0C3F1C2C11D
:10581600DEF0C3C1DFF0000E0001E16F640EE06F41
:10582600020EE26F020EE36F20EC70F0FD0E000137
:10583600916F280E926F8EEC6EF0000E0101C46F10
:10584600000EC56F000EC66F000EC76FD1510C0D4E
:10585600F3CFCDF11AD00101CD51020D000EF32484
:10586600D96E060EF420DA6EDECFF0F0DDCFF1F061
:105876000001F0510101C4270001F1510101C523C6
:10588600000EC623000EC723CD2B010ED125000125
:10589600976F986B000E9823000E9A6F0C0E996FF7
:1058A60030EC71F00101CD510001F06FF16B9751B1
:1058B600F05DF151800AF26F9851800AF259D8A032
:1058C600CAD7320E0101C4250001B06F000E0101D6
:1058D600C5210001B16F000E0101C6210001B26FA2
:1058E600000E0101C7210001B36F640EB46F000EF4
:1058F600B56F000EB66F000EB76FBCEC60F0B0C0AF
:10590600DEF0B1C0DFF0000E0001E16F640EE06F63
:10591600020EE26F020EE36F20EC70F0D20E000171
:10592600916F280E926F8EEC6EF00101D151030D2E
:10593600010EF326000EF4226B0EF324D96E010E2F
:10594600F420DA6EDECF90F0DDCF91F0AA0E0001E2
:10595600926F010E936FB5EC62F0AA0E0001916F83
:10596600010E926F8EEC6EF0E70E0001916F240E21
:10597600926F8EEC6EF00101D1510D0D020EF326E1
:10598600000EF4224C0EF324D96E020EF420DA6EC9
:10599600DECF90F0DDCF91F0AA0E0001926F010EDE
:1059A600936FB5EC62F0AA0E0001916F010E926F33
:1059B6008EEC6EF07CEC6AF007D0910E0001916FD0
:1059C600280E926F8EEC6EF0D20E0001916F1A0EB9
:1059D600926F8EEC6EF00101D12BCFD5000E000137
:1059E600EF150101AA6F000E0001F0150101AB6F62
:1059F600FF0E0001F1150101AC6FFF0E0001F2155B
:105A06000101AD6FDE0EAC1904E1AD05AA11AB11B3
:105A1600D8A45AD1000E0001EF150101AE6FFF0E9A
:105A26000001F0150101AF6FEFC0AAF1F0C0ABF1B4
:105A3600040EAC6FD890AB33AA33AC2FFBD7AA5168
:105A4600030BB06F0001EF51070B0101B16F15D1C8
:105A5600F3C0B7F1F4C0B8F120EE02F0B751D92681
:105A6600B851DA22DECF18F1DDCF19F1B7C1D9FF6F
:105A7600B8C1DAFFDE50DE10D8B40ED0B7C1D9FFF8
:105A8600B8C1DAFFDECFE1F0DDCFE2F018C1E3F016
:105A960019C1E4F0B3EC6AF0020E0101496F800E01
:105AA600486F4AD14C50AA6FAB6BB051AC6FAD6B1F
:105AB600010EAC27000EAD23AA51AC1903E1AB5180
:105AC600AD19D8A439D1B15156EC57F035D1F3C040
:105AD600B9F1F4C0BAF1B9C1D9FFBAC1DAFFDECF64
:105AE600BBF1DDCFBCF1200E0101BB5D4E0EBC59F2
:105AF600D8A015D0210EBB5DCB0EBC59D8B00FD0A7
:105B0600000E0001A26F060EA16FBBC1A3F0BCC1BF
:105B1600A4F055EC6FF0A1C03BF0A2C03CF001012F
:105B260020EE02F0B951D926BA51DA22DECFBBF106
:105B3600DDCFBCF1980EBB5D3A0EBC59D8A015D08E
:105B4600110EBB5DA40EBC59D8B00FD0000E0001DB
:105B5600A26F040EA16FBBC1A3F0BCC1A4F055ECAB
:105B66006FF0A1C03DF0A2C03EF0010120EE04F0AE
:105B7600B951D926BA51DA22DECFBBF1DDCFBCF15D
:105B8600B10EBB5DB30EBC59D8B00FD0000E0001EC
:105B9600A26F0A0EA16FBBC1A3F0BCC1A4F055EC65
:105BA6006FF0A1C03AF1A2C03BF1010120EE06F070
:105BB600B951D926BA51DA22DECFBBF1DDCFBCF11D
:105BC600B10EBB5DB30EBC59D8B00FD0000E0001AC
:105BD600A26F080EA16FBBC1A3F0BCC1A4F055EC27
:105BE6006FF0A1C035F0A2C036F009EC68F0A4D081
:105BF600F3C0B4F1F4C0B5F1B4C1D9FFB5C1DAFF51
:105C0600DECFBBF1DDCFBCF1210E0101BB5DCB0EBA
:105C1600BC59D8B00FD0000E0001A26F2E0EA16F96
:105C2600BBC1A3F0BCC1A4F055EC6FF0A1C039F024
:105C3600A2C03AF0010120EE02F0B451D926B551C6
:105C4600DA22DECFBBF1DDCFBCF1110EBB5DA40EB7
:105C5600BC59D8B00FD0000E0001A26F300EA16F54
:105C6600BBC1A3F0BCC1A4F055EC6FF0A1C037F0E6
:105C7600A2C038F009EC5FF05FD0AEC1AAF1AFC1A7
:105C8600ABF10101AB51010AD8B40AD0020AD8B46B
:105C96000CD00B0AD8B40ED0040AD8B410D04CD00D
:105CA600AA51000AD8B4D4D647D0AA51000AD8B40B
:105CB6000ED742D0AA51000AD8B4F4D63DD0AA5184
:105CC600000AD8B495D738D049A436D07B0E000147
:105CD600EF190DE1070EF019F111F211D8A407D052
:105CE600F3C0CBF0F4C0CCF0B1EC6EF020D0FB0EDC
:105CF6000001EF190DE1050EF019F111F211D8A40A
:105D060007D0F3C0C5F0F4C0C6F04FEC72F00FD068
:105D1600FB0E0001EF1910E1F005F111F211D8A404
:105D26000BD0F3C090F0F4C091F00DEC67F0000ECC
:105D36000101476F800E466F4AA01200B60E0001A1
:105D4600906F010E916FB20E926F010E936FE5EC9C
:105D56005FF00009D8B41200F6C0BBF0F7C0BCF083
:105D6600F8C0BDF0F9C0BEF060EC53F0000E0001C3
:105D7600EF150101AA6F000E0001F0150101AB6FCE
:105D8600FF0E0001F1150101AC6FFF0E0001F215C7
:105D96000101AD6FDD0EAC190DE1AD05AA11AB1118
:105DA600D8A408D0060E0001916F270E926F8EECD4
:105DB6006EF02BD0000E0001EF150101AA6F000E48
:105DC6000001F0150101AB6FFF0E0001F115010195
:105DD600AC6FFF0E0001F2150101AD6FDE0EAC19BE
:105DE6000DE1AD05AA11AB11D8A408D0120E000121
:105DF600916F270E926F8EEC6EF007D0410E000168
:105E0600916F270E926F8EEC6EF0EF0E0001966F7B
:105E1600000E976F000E996F010E986F89EC61F076
:105E2600F3C096F0F4C097F0F5C098F00001996BB6
:105E36001BEC6EF0D20E0001916F1A0E926F8EEC73
:105E46006EF0120002014CB10DD001016C516D11C2
:105E5600D8A408D05C0E0001916F240E926F8EECD0
:105E66006EF01200420E0001916F1D0E926F8EECC5
:105E76006EF0780E0001916F280E926F8EEC6EF028
:105E8600A7C1DEF0A8C1DFF0500E0001E06F290EB9
:105E9600E16F80EC6BF0840E0001916F240E926F1F
:105EA6008EEC6EF030C1DEF031C1DFF0F50E000190
:105EB600E06F280EE16F80EC6BF0000E0101AF6F12
:105EC600000EB66F070EB66501D01200B651010D71
:105ED6003C0EF324D96E020EF420DA6EDF50BB6F4F
:105EE600BB29D8B4BED1BB51030D6B0EF324D96EBA
:105EF600010EF420DA6EDF380F0BB46FAF51B41910
:105F0600D8B418D0730E0001916F280E926F8EECE4
:105F16006EF0B4C1B8F00001B96B010EBA6FADEC0A
:105F26006FF0C80E0001916F1D0E926F8EEC6EF031
:105F3600B4C1AFF10101BB510D0D4C0EF324D96E66
:105F4600020EF420DA6E0201DFA08BD10101BB51F3
:105F56000C0DF3CFBCF1BB51030D6B0EF324D96EC0
:105F6600010EF420DA6EDF500F0B0C0DF328AA6F2A
:105F7600000EB56F0B0EB56501D073D1BC51020D85
:105F8600000EF324D96E050EF420DA6EDECFBDF1D5
:105F9600DDCFBEF1BC51020D000EF324D96E090E01
:105FA600F420DA6EDECFB7F1DDCFB8F1BC51020DC9
:105FB600000EF324D96E0A0EF420DA6EDECFB9F1A4
:105FC600DDCFBAF1000E0001936F0A0E926FB7C1D2
:105FD60090F0B8C191F0A0EC6DF090C097F091C030
:105FE60098F0000E00019A6F0A0E996F30EC71F06E
:105FF60097C0B7F198C0B8F1000E0001936F0A0E72
:10600600926FB9C190F0BAC191F0A0EC6DF090C05A
:1060160097F091C098F0000E00019A6F0A0E996FE2
:1060260030EC71F097C0B9F198C0BAF10101B751DF
:10603600BD5DB851BE59D8B004D0BDC1B7F1BEC11F
:10604600B8F1BD51B95DBE51BA59D8B004D0BDC181
:10605600B9F1BEC1BAF1BE5104E1C90EBD5DD8A009
:10606600F9D0E80E0001916F240E926F8EEC6EF05F
:106076007C0E0001BB6F280EBC6F0101AA51B5252D
:10608600D4EC6EF0BDC1DEF0BEC1DFF0FD0E000146
:10609600E06F280EE16F80EC6BF0B7C1DEF0B8C19F
:1060A600DFF0500E0001E06F290EE16F80EC6BF01F
:1060B600B9C1DEF0BAC1DFF0D20E0001E06F280EE2
:1060C600E16F80EC6BF00101BD51A75DBE51A8598F
:1060D600D8B018D0E80E0001916F240E926F8EECA6
:1060E6006EF0A7C1F4F0A8C1F5F00001F41FF51F8A
:1060F600F44BF52B0101BD510001F4250101AB6FF5
:10610600BE5117D04C0E0001916F290E926F8EEC86
:106116006EF0BDC1F4F0BEC1F5F00001F41FF51F2D
:10612600F44BF52B0101A7510001F4250101AB6FDA
:10613600A8510001F5210101AC6FABC1DEF0ACC185
:10614600DFF0FD0E0001E06F280EE16F4EEC6BF004
:106156000101BC51010D000EF324D96E080EF42086
:10616600DA6EDF50B06FBC51010D000EF324D96E0C
:10617600070EF420DA6EDF50B16FB0C1F4F0000103
:10618600F56BF4BFF507F41FF51FF44BF52BF4512F
:106196000101B125B26F000EB1BFFF0E0001F5215E
:1061A6000101B36FBC51010D600EF324D96E070EC9
:1061B600F420DA6EDF5072EC65F0F90E0001916F93
:1061C600280E926F8EEC6EF00101B05172EC65F004
:1061D600330E0001916F290E926F8EEC6EF0010165
:1061E600B15172EC65F0F90E0001916F280E926FB5
:1061F6008EEC6EF00101B3BF05D0B35111E1B205CB
:10620600D8B00ED0B2C1F4F0B3C1F5F00001F41F5E
:10621600F51FF44BF52BF4C0ADF1F5C0AEF104D08B
:10622600B2C1ADF1B3C1AEF1ADC1DEF0AEC1DFF0CA
:10623600000E0001E16F0A0EE06F010EE26F010E23
:10624600E36F20EC70F0B80E0001916F270E926F8D
:106256008EEC6EF00101BC2B7CEC6AF00101B52BD3
:1062660089D60101B62B2ED60001D66F0001D65174
:10627600080DA10EF324DD6F040EF420DE6FCBC0F3
:10628600D7F0DDC0D9FFDEC0DAFF43C0DFFF20EE66
:1062960001F0DD51D926DE51DA22A9C1DFFF4B50CC
:1062A600D65DD8A003D0D751D8B41200D6510C0D64
:1062B600D890F336F436000EF324DF6F050EF42083
:1062C600E06FDFC0D9FFE0C0DAFFDECFD8F0DDCF68
:1062D600D9F0020EDF27000EE023DFC0D9FFE0C0B1
:1062E600DAFFDECFDAF0DDCFDBF0020EDF27000EBD
:1062F600E023DAC097F0DBC098F0D6EC69F0000135
:10630600CC6FCC3BF00ECC17D8C097F0D9C098F024
:10631600D6EC69F00001CC25DC6F20EE02F0DD51F1
:10632600D926DE51DA22DC51DE18D8B40AD0010EA5
:10633600D76F20EE02F0DD51D926DE51DA22DCC01D
:10634600DFFFDFC0D9FFE0C0DAFFDECFD8F0DDCF58
:10635600D9F0020EDF27000EE023DFC0D9FFE0C030
:10636600DAFFDECFDAF0DDCFDBF0020EDF27000E3C
:10637600E023DAC097F0DBC098F0D6EC69F00001B4
:10638600CC6FCC3BF00ECC17D8C097F0D9C098F0A4
:10639600D6EC69F00001CC25DC6F20EE03F0DD5170
:1063A600D926DE51DA22DC51DE18D8B40AD0010E25
:1063B600D76F20EE03F0DD51D926DE51DA22DCC09C
:1063C600DFFFDFC0D9FFE0C0DAFFDECFD8F0DDCFD8
:1063D600D9F0020EDF27000EE023DFC0D9FFE0C0B0
:1063E600DAFFDECFDAF0DDCFDBF0020EDF27000EBC
:1063F600E023DAC097F0DBC098F0D6EC69F0000134
:10640600CC6FCC3BF00ECC17D8C097F0D9C098F023
:10641600D6EC69F00001CC25DC6F20EE04F0DD51EE
:10642600D926DE51DA22DC51DE18D8B40AD0010EA4
:10643600D76F20EE04F0DD51D926DE51DA22DCC01A
:10644600DFFFDFC0D9FFE0C0DAFFDECFD8F0DDCF57
:10645600D9F0020EDF27000EE023DFC0D9FFE0C02F
:10646600DAFFDECFDAF0DDCFDBF0020EDF27000E3B
:10647600E023DAC097F0DBC098F0D6EC69F00001B3
:10648600CC6FCC3BF00ECC17D8C097F0D9C098F0A3
:10649600D6EC69F00001CC25DC6F20EE05F0DD516D
:1064A600D926DE51DA22DC51DE18D8B40AD0010E24
:1064B600D76F20EE05F0DD51D926DE51DA22DCC099
:1064C600DFFFDFC0D9FFE0C0DAFFDECFD8F0DDCFD7
:1064D600D9F0020EDF27000EE023DFC0D9FFE0C0AF
:1064E600DAFFDECFDAF0DDCFDBF0020EDF27000EBB
:1064F600E023DAC097F0DBC098F0D6EC69F0000133
:10650600CC6FCC3BF00ECC17D8C097F0D9C098F022
:10651600D6EC69F00001CC25DC6F20EE06F0DD51EB
:10652600D926DE51DA22DC51DE18D8B40AD0010EA3
:10653600D76F20EE06F0DD51D926DE51DA22DCC017
:10654600DFFFDFC0D9FFE0C0DAFFDECFD8F0DDCF56
:10655600D9F0020EDF27000EE023DFC0D9FFE0C02E
:10656600DAFFDECFDAF0DDCFDBF0020EDF27000E3A
:10657600E023DAC097F0DBC098F0D6EC69F00001B2
:10658600CC6FCC3BF00ECC17D8C097F0D9C098F0A2
:10659600D6EC69F00001CC25DC6F20EE07F0DD516A
:1065A600D926DE51DA22DC51DE18D8B40AD0010E23
:1065B600D76F20EE07F0DD51D926DE51DA22DCC096
:1065C600DFFFD751D8B412004C50CC6FCD6BCC3B0B
:1065D600CD3BF00ECD17CC510F0BCD13F00ECC17D3
:1065E600F00ECC25CE6FFF0ECD21CF6FD06BCFBF77
:1065F600D007D051D16FD651CE25D26F000ECF2104
:10660600D36F000ED021D46F000ED121D56F000EAE
:10661600D225B96F050ED321BA6FDF0ED421BB6F19
:10662600010ED521BC6FDDC0BDF0DEC0BEF0080E88
:10663600BF6F81EC68F01200000E0001BC6F2B509A
:106646002D1804E12C502E18D8B4C5D12BC097F0C4
:106656002CC098F0000E9A6F110E996F30EC71F005
:10666600100E00019725CB6F0D0E9821CC6FCBC075
:10667600D9FFCCC0DAFFA3C0E1FFA4C0E2FFDECFA2
:10668600E6FFDDCFE5FF20EE02F0CB51D926CC5157
:10669600DA22A5C0E1FFA6C0E2FFDECFE6FFDDCF2E
:1066A600E5FF20EE07F0CB51D926CC51DA22DFA642
:1066B6009AD020EE04F0CB51D926CC51DA22DF5005
:1066C600A76FA751B46FB56BB66BB76B20EE05F02D
:1066D600CB51D926CC51DA22DF50A76FA751B86F1C
:1066E600B96BBA6BBB6B20EE06F0CB51D926CC51F9
:1066F600DA22DF50A76FA751BD6FBE6BBF6BC06BB1
:1067060020EE07F0CB51D926CC51DA22DF50A76F05
:10671600A751C16FC26BC36BC46BBDC0A7F0BEC02F
:10672600A8F0BFC0A9F0C0C0AAF0150ED890A73730
:10673600A837A937AA37E82EF9D7A7C0C5F0A8C049
:10674600C6F0A9C0C7F0AAC0C8F0E00EC115A76F71
:10675600000EC215A86F000EC315A96F000EC41552
:10676600AA6F0D0ED890A737A837A937AA37E82EF3
:10677600F9D7A751C527A851C623A951C723AA519E
:10678600C823030EC115A76F000EC215A86F000E11
:10679600C315A96F000EC415AA6FA8C0AAF0A7C09A
:1067A600A9F0A86BA76BA751C527A851C623A95165
:1067B600C723AA51C823B4C0A8F0B5C0A9F0B6C073
:1067C600AAF0A76BA751C527A851C623A951C7236D
:1067D600AA51C823B851C527B951C623BA51C723F0
:1067E600BB51C82357D020EE06F0CB51D926CC5149
:1067F600DA22DF50A76FA751BD6FBE6BBF6BC06BB0
:1068060020EE07F0CB51D926CC51DA22DF50A76F04
:10681600A751C16FC26BC36BC46B050EA76FC1C016
:10682600A8F0C2C0A9F0C3C0AAF0C4C0ABF0A76765
:1068360001D007D0AB35AB33AA33A933A833A72F82
:10684600F6D7070E0001A815AC6F000EA915AD6F9F
:10685600000EAA15AE6F000EAB15AF6FBDC0B0F03F
:10686600BEC0B1F0BFC0B2F0C0C0B3F0030ED89046
:10687600B037B137B237B337E82EF9D7AC51B025B8
:10688600C56FAD51B121C66FAE51B221C76FAF51C1
:10689600B321C86F9DC0D9FF9EC0DAFFC5C0DEFF19
:1068A600C6C0DEFFC7C0DEFFC8C0DEFF090ECB25AF
:1068B600C96F000ECC21CA6FC9C0D9FFCAC0DAFFA2
:1068C6009FC0E1FFA0C0E2FFDFCFE7FFC94BCA2BA5
:1068D6009F4BA02BC9C0D9FFCAC0DAFF9FC0E1FFFA
:1068E600A0C0E2FFDFCFE7FFC94BCA2B9F4BA02B0F
:1068F600C9C0D9FFCAC0DAFF9FC0E1FFA0C0E2FF4E
:10690600DFCFE7FFC94BCA2B9F4BA02BC9C0D9FFCE
:10691600CAC0DAFF9FC0E1FFA0C0E2FFDFCFE7FFFA
:10692600C94BCA2B9F4BA02BC9C0D9FFCAC0DAFFDF
:106936009FC0E1FFA0C0E2FFDFCFE7FFC94BCA2B34
:106946009F4BA02BC9C0D9FFCAC0DAFF9FC0E1FF89
:10695600A0C0E2FFDFCFE7FFC94BCA2B9F4BA02B9E
:10696600C9C0D9FFCAC0DAFF9FC0E1FFA0C0E2FFDD
:10697600DFCFE7FFC94BCA2B9F4BA02BC9C0D9FF5E
:10698600CAC0DAFF9FC0E1FFA0C0E2FFDFCFE7FF8A
:10699600C94BCA2B9F4BA02B20EE08F0CB51D92612
:1069A600CC51DA22A1C0E1FFA2C0E2FFDFCFE7FFB0
:1069B6002C500BE10F0E2B5CD8B007D0010E2B2408
:1069C6002B6E000E2C202C6E04D0000E2C6E000EAA
:1069D6002B6E010EBC6FBC511200170E0001916F99
:1069E600250E926F8EEC6EF0000E0001936F020E74
:1069F600926FCAEC6FF0000192514C6E4CC0B8F029
:106A0600B96B010EBA6FADEC6FF0D20E0001916F4B
:106A16001A0E926F8EEC6EF0260E0001916F250E07
:106A2600926F8EEC6EF0020E4818D8A407D0050EB1
:106A36000001916F290E926F8EEC6EF0030E4818CE
:106A4600D8A407D0010E0001916F290E926F8EEC2B
:106A56006EF0040E4818D8A407D0F60E0001916F08
:106A6600260E926F8EEC6EF0320E0001916F280E9C
:106A7600926F8EEC6EF0360E0001916F260E926FBD
:106A86008EEC6EF0000E0001936F040E926FCAEC4E
:106A96006FF092C03DF093C03EF03DC0DEF03EC0C8
:106AA600DFF0F50E0001E06F280EE16F80EC6BF071
:106AB600280E0001916F260E926F8EEC6EF0000E7E
:106AC6000001936F060E926FCAEC6FF092C03BF016
:106AD60093C03CF03BC0DEF03CC0DFF0F50E000199
:106AE600E06F280EE16F80EC6BF04750D8B416D0FB
:106AF600620E0001916F250E926F8EEC6EF047C00C
:106B0600B8F00001B96B010EBA6FADEC6FF0B40EC0
:106B16000001916F270E926F8EEC6EF04650D8B43E
:106B260016D0530E0001916F250E926F8EEC6EF00B
:106B360046C0B8F00001B96B010EBA6FADEC6FF04C
:106B4600B40E0001916F270E926F8EEC6EF0520E0E
:106B56000001916F260E926F8EEC6EF0000E000112
:106B6600936F300E926FCAEC6FF092C037F093C0FD
:106B760038F037C0E4F038C0E5F06EEC70F0440E43
:106B86000001916F260E926F8EEC6EF0000E0001E2
:106B9600936F2E0E926FCAEC6FF092C039F093C0CD
:106BA6003AF039C0E4F03AC0E5F06EEC70F01A0E37
:106BB6000001916F260E926F8EEC6EF0000E0001B2
:106BC600936F080E926FCAEC6FF092C035F093C0C7
:106BD60036F035C0E4F036C0E5F06EEC70F0600ECD
:106BE6000001916F260E926F8EEC6EF0000E000182
:106BF600936F0A0E926FCAEC6FF092C03AF193C08F
:106C06003BF13AC1E4F03BC1E5F06EEC70F0350EB5
:106C16000001916F250E926F8EEC6EF044C0B8F0B5
:106C26000001B96B010EBA6FADEC6FF0810E000179
:106C3600916F280E926F8EEC6EF0000E0001916F30
:106C4600010E906F28EC72F0496E000E0001E76F9E
:106C560049C0E6F07F0EE617D8B480D0440E916F97
:106C6600250E926F8EEC6EF049A00AD0BD0E000183
:106C7600916F1F0E926F8EEC6EF0010E0001E76FA2
:106C860049A214D00001E751D8B406D0080E916F7E
:106C9600250E926F8EEC6EF01D0E0001916F200E88
:106CA600926F8EEC6EF0010E0001E76F49A414D0CE
:106CB6000001E751D8B406D0080E916F250E926FE9
:106CC6008EEC6EF0D30E0001916F210E926F8EEC5A
:106CD6006EF0010E0001E76F49A614D00001E751DE
:106CE600D8B406D0080E916F250E926F8EEC6EF01A
:106CF600570E0001916F1F0E926F8EEC6EF0010E13
:106D06000001E76F49A814D00001E751D8B406D0B6
:106D1600080E916F250E926F8EEC6EF0B40E000188
:106D2600916F1E0E926F8EEC6EF0010E0001E76FF2
:106D360049AA14D00001E751D8B406D0080E916FC5
:106D4600250E926F8EEC6EF0760E0001916F200E7E
:106D5600926F8EEC6EF0010E0001E76F4AA41200EE
:106D660049AE1200760E0001916F230E926F8EECE3
:106D76006EF0120010EC72F00B0E0001986FB80E58
:106D8600976F3BEC70F0280E0001BC6F030EBD6FD1
:106D96004B5045EC6AF0000E0001C66F000EC76F3F
:106DA600000E456E000ED86F070ED86501D087D14C
:106DB600D8510D0D4C0EF324D26F020EF420D36F72
:106DC600D851060D290EF324CE6F030EF420CF6F93
:106DD600D851060D590EF324C86F030EF420C96F5F
:106DE600000EC56F4B50D85DD8B055D1D851010DA6
:106DF600000EF324D96E010EF420DA6EDF5020095E
:106E0600D06F000ED46F040ED46501D04CD1D4C01F
:106E1600C0F0010EC16FC02B02D0D890C137C02F71
:106E2600FCD70001C151D76F000ECC6F050ED4619F
:106E3600CCD0D451D8A405D0CEC0D9FFCFC0DAFF6C
:106E46001FD0D405D8A403D020EE02F006D0020E3F
:106E5600D419D8A406D020EE04F0CE51D926CF51AD
:106E66000ED0030ED419D8A405D0C8C0D9FFC9C006
:106E7600DAFF06D020EE02F0C851D926C951DA222F
:106E8600DECFCAF0DDCFCBF0CAC098F0CBC099F008
:106E9600ACEC59F098C0D5F099C0D6F00001D6AF49
:106EA60005D0000EC46F000EC36F03D0D5C0C3F06B
:106EB600C46BD851050D000EC06F030EC16FF350A1
:106EC600C027F450C123D451010DF350C025D96E0B
:106ED600F450C121DA6EC3C0DFFFD52903E1D629FC
:106EE600D8B406D0FD0ED51916E1D629D8A413D0EC
:106EF600D051D7150009D8B402D0010EC76FD851AA
:106F0600010D440EF324D96E020EF420DA6EDF5022
:106F1600D7150009A6D0D751C513D051D7150009EA
:106F2600D8B405D0D551455CD8A0D5C045F0D851C8
:106F3600010D440EF324D96E020EF420DA6EDF50F2
:106F4600D7150009D8A402D0010ECC6F20EE0AF0A6
:106F5600D251D926D351DA22DF50D7150009D8B439
:106F660002D0010E01D0000ECD6F4450C06FC16B30
:106F7600D551C05DC151800AC26FD651800AC2592F
:106F8600D8B002D0010E01D0000ED16FD151D8B4C5
:106F960010D020EE0AF0D251D926D351DA22D75199
:106FA600DF12D051D7150009D8B459D0010EC66FDB
:106FB60056D0D751FF0AC06F20EE0AF0D251D9261B
:106FC600D351DA22C051DF164AD0D851060D400EF1
:106FD600C06F040EC16F010EC027000EC123F3500F
:106FE600C027F450C123020EC025D96E000EC12160
:106FF600DA6EDECF97F0DDCF98F0F3EC6DF097C048
:10700600D5F098C0D6F00001D551455CD8A0D5C0C2
:1070160045F020EE0AF0D251D926D351DA22DF50BC
:10702600D7150009D8B402D0010E01D0000ECD6FDD
:10703600D6BF08D0D65104E1650ED55DD8A002D0E2
:10704600010E01D0000ED16FD151D8B408D020EE78
:107056000AF0D251D926D351DA22D751DF12D151B3
:10706600CD19D8B402D0010ECC6FD051D715000976
:10707600D8B40ED0CC51D8B40BD0D4C0BBF0D1C04C
:10708600BCF0D5C0BDF0D6C0BEF0D8512AEC5EF03B
:107096000001D42BB8D620EE0AF0D251D926D3510E
:1070A600DA22000EDF6ED851010D440EF324D96E9C
:1070B600020EF420DA6EC5C0DFFFD82B75D6C65196
:1070C600D8B402D0428401D04294C751D8B402D079
:1070D6004286120042961200000EF2BC010E00011A
:1070E6009D6FF29CB40EA76F020EA86F0F0120AD24
:1070F6000DD0000120EE0EF0A751D926A851DA22B4
:10710600DE2A000EDD220F01209D209720AB0AD03B
:10711600000120EE10F0A751D926A851DA22DE2A66
:10712600000EDD220F0120A90DD0000120EE12F085
:10713600A751D926A851DA22DE2A000EDD220F0138
:10714600209920972750291804E128502A18D8B4E6
:1071560055D127C097F028C098F0000E00019A6F0D
:10716600110E996F30EC71F0000E00019725A36F98
:107176000C0E9821A46F20EE04F0A351D926A45139
:10718600DA22DF509F6F20EE05F0A351D926A451D5
:10719600DA22DF50A06F20EE06F0A351D926A451C3
:1071A600DA22DF50A16F20EE07F0A351D926A451B1
:1071B600DA22DF50A26F20EE08F0A351D926A4519F
:1071C600DA22DF509E6F090EA325A96F000EA421B7
:1071D600AA6F0F0120B712D19FC023FFA0C024FFC2
:1071E600A1C021FFA2C022FF9EC025FFA9C0D9FFD2
:1071F600AAC0DAFFDF50266F0001A94BAA2BA9C04F
:10720600D9FFAAC0DAFFDF500F01276F0001A94B93
:10721600AA2BA9C0D9FFAAC0DAFFDF500F01286F39
:107226000001A94BAA2BA9C0D9FFAAC0DAFFDF50DB
:107236000F01296F0001A94BAA2BA9C0D9FFAAC02B
:10724600DAFFDF500F012A6F0001A94BAA2BA9C054
:10725600D9FFAAC0DAFFDF500F012B6F0001A94B3F
:10726600AA2BA9C0D9FFAAC0DAFFDF500F012C6FE5
:107276000001A94BAA2BA9C0D9FFAAC0DAFFDF508B
:107286000F012D6F0001A94BAA2B0F012087285053
:107296000BE10F0E275CD8B007D0010E2724276E0E
:1072A600000E2820286E04D0000E286E000E276ED1
:1072B600B40E0001A76F020EA86FA7C0D9FFA8C021
:1072C600DAFFDE2A000EDD2220EE02F0A751D926D3
:1072D600A851DA22A1C0DFFF20EE03F0A751D9267C
:1072E600A851DA22A2C0DFFF20EE04F0A751D9266A
:1072F600A851DA229FC0DFFF20EE05F0A751D9265C
:10730600A851DA22A0C0DFFF080EA95F000EAA5B13
:10731600060EA725A56F000EA821A66FA9C0D9FF46
:10732600AAC0DAFFA5C0E1FFA6C0E2FFDFCFE7FFF4
:10733600A94BAA2BA54BA62BA9C0D9FFAAC0DAFF39
:10734600A5C0E1FFA6C0E2FFDFCFE7FFA94BAA2B4E
:10735600A54BA62BA9C0D9FFAAC0DAFFA5C0E1FF9D
:10736600A6C0E2FFDFCFE7FFA94BAA2BA54BA62BB2
:10737600A9C0D9FFAAC0DAFFA5C0E1FFA6C0E2FFF7
:10738600DFCFE7FFA94BAA2BA54BA62BA9C0D9FF98
:10739600AAC0DAFFA5C0E1FFA6C0E2FFDFCFE7FF84
:1073A600A94BAA2BA54BA62BA9C0D9FFAAC0DAFFC9
:1073B600A5C0E1FFA6C0E2FFDFCFE7FFA94BAA2BDE
:1073C600A54BA62BA9C0D9FFAAC0DAFFA5C0E1FF2D
:1073D600A6C0E2FFDFCFE7FFA94BAA2BA54BA62B42
:1073E600A9C0D9FFAAC0DAFFA5C0E1FFA6C0E2FF87
:1073F600DFCFE7FFA94BAA2BA54BA62B00019DA12A
:1074060002D0F28C1200F29C1200000EF2BC010EA9
:10741600076EF29CB40E0F6E020E106E0F0120ADB9
:107426000BD020EE0EF00F50D9261050DA22DE2AAD
:10743600000EDD22209D209720AB09D020EE10F013
:107446000F50D9261050DA22DE2A000EDD2220A99E
:107456000BD020EE12F00F50D9261050DA22DE2A79
:10746600000EDD22209920972750291804E1285084
:107476002A18D8B442D127C001F028C002F0000E65
:10748600046E110E036E57EC71F0000E01240D6EA2
:107496000C0E02200E6E20EE04F00D50D9260E5072
:1074A600DA22DF50096E20EE05F00D50D9260E5077
:1074B600DA22DF500A6E20EE06F00D50D9260E5065
:1074C600DA22DF500B6E20EE07F00D50D9260E5053
:1074D600DA22DF500C6E20EE08F00D50D9260E5041
:1074E600DA22DF50086E090E0D24136E000E0E20F0
:1074F600146E0F0120B701D109C023FF0AC024FF73
:107506000BC021FF0CC022FF08C025FF13C0D9FF06
:1075160014C0DAFFDF50266F134A142A13C0D9FFAE
:1075260014C0DAFFDF50276F134A142A13C0D9FF9D
:1075360014C0DAFFDF50286F134A142A13C0D9FF8C
:1075460014C0DAFFDF50296F134A142A13C0D9FF7B
:1075560014C0DAFFDF502A6F134A142A13C0D9FF6A
:1075660014C0DAFFDF502B6F134A142A13C0D9FF59
:1075760014C0DAFFDF502C6F134A142A13C0D9FF48
:1075860014C0DAFFDF502D6F134A142A20872850C3
:107596000BE10F0E275CD8B007D0010E2724276E0B
:1075A600000E2820286E04D0000E286E000E276ECE
:1075B600B40E0F6E020E106E0FC0D9FF10C0DAFFA8
:1075C600DE2A000EDD2220EE02F00F50D9261050E2
:1075D600DA220BC0DFFF20EE03F00F50D926105041
:1075E600DA220CC0DFFF20EE04F00F50D92610502F
:1075F600DA2209C0DFFF20EE05F00F50D926105021
:10760600DA220AC0DFFF080E135E000E145A060EB9
:107616000F24116E000E1020126E13C0D9FF14C075
:10762600DAFF11C0E1FF12C0E2FFDFCFE7FF134A26
:10763600142A114A122A13C0D9FF14C0DAFF11C046
:10764600E1FF12C0E2FFDFCFE7FF134A142A114A17
:10765600122A13C0D9FF14C0DAFF11C0E1FF12C00D
:10766600E2FFDFCFE7FF134A142A114A122A13C09A
:10767600D9FF14C0DAFF11C0E1FF12C0E2FFDFCF6D
:10768600E7FF134A142A114A122A13C0D9FF14C05D
:10769600DAFF11C0E1FF12C0E2FFDFCFE7FF134AB6
:1076A600142A114A122A13C0D9FF14C0DAFF11C0D6
:1076B600E1FF12C0E2FFDFCFE7FF134A142A114AA7
:1076C600122A13C0D9FF14C0DAFF11C0E1FF12C09D
:1076D600E2FFDFCFE7FF134A142A114A122A13C02A
:1076E600D9FF14C0DAFF11C0E1FF12C0E2FFDFCFFD
:1076F600E7FF134A142A114A122A07A002D0F28C75
:107706001200F29C1200000E0001DD6F000ED76F12
:10771600000ED86F000ED96F000EDA6F000ECB6F19
:10772600000ECC6F000ECD6F000ECE6F000EC66F32
:10773600000EC76F000EC86F000EC96F000ED36F24
:10774600000ED46F000ED56F000ED66F010EDE6FE1
:10775600D2D00001DD2BD7C0C2F0D8C0C3F0D9C04B
:10776600C4F0DAC0C5F0C21FC31FC41FC51FC22B99
:10777600000EC323C423C523DB51C225CF6FDC51C2
:10778600C321D06F000EC421D16F000EC521D26F68
:10779600CFC0B0F0D0C0B1F0D1C0B2F0D2C0B3F01B
:1077A600DD51B46FB56BB66BB76BBCEC60F0000126
:1077B600B051D727B151D823B251D923B351DA23C7
:1077C600DE05D8A430D0D7C0C2F0D8C0C3F0D9C027
:1077D600C4F0DAC0C5F0C21FC31FC41FC51FC22B29
:1077E600000EC323C423C523DB51C225A46FDC517D
:1077F600C321A56F000EC421A66F000EC521A76F79
:10780600CFC0A8F0D0C0A9F0D1C0AAF0D2C0ABF0CA
:10781600C6EC6CF00001A451D327A551D423A65180
:10782600D523A7513FD0D7C0C2F0D8C0C3F0D9C026
:10783600C4F0DAC0C5F0C21FC31FC41FC51FC22BC8
:10784600000EC323C423C523DB51C225A46FDC511C
:10785600C321A56F000EC421A66F000EC521A76F18
:10786600CFC0A8F0D0C0A9F0D1C0AAF0D2C0ABF06A
:10787600C6EC6CF0A4C0B0F0A5C0B1F0A6C0B2F0E2
:10788600A7C0B3F00001CA51B46FB56BB66BB76B46
:10789600BCEC60F00001B051D327B151D423B251F2
:1078A600D523B351D623D6BF26D0040ED65DD8A095
:1078B60022D0DE51020DF3CFDEF0DE51DE03F3CF30
:1078C600CAF0D3C0B0F0D4C0B1F0D5C0B2F0D6C0C3
:1078D600B3F0040EB46F000EB56F000EB66F000E57
:1078E600B76FBCEC60F0B0C0D3F0B1C0D4F0B2C09A
:1078F600D5F0B3C0D6F0DB0E0001906F000E916F8D
:10790600CCEC67F00009D8A424D7020E0001DD6193
:1079160009D0000ECB6F000ECC6F000ECD6F000E9F
:10792600CE6F26D0D3C0B0F0D4C0B1F0D5C0B2F07F
:10793600D6C0B3F0FF0EC26FFF0EC36FDD51C46F2A
:10794600C56BC251C427C351C523C4C0B4F0C5C05A
:10795600B5F0000EB5BFFF0EB66FB76FBCEC60F0AA
:10796600B0C0CBF0B1C0CCF0B2C0CDF0B3C0CEF059
:10797600BEC0D9FFBFC0DAFFDDC0DFFFC0C0D9FF80
:10798600C1C0DAFFD7C0DEFFD8C0DDFFCBC090F0A4
:10799600CCC091F0CDC092F0CEC093F0BCEC5AF0C2
:1079A60090C0A4F091C0A5F092C0A6F093C0A7F035
:1079B6000001DE51A86FA96BAA6BAB6BC6EC6CF02D
:1079C600A4C0C6F0A5C0C7F0A6C0C8F0A7C0C9F03D
:1079D600C6C0BEF0C7C0BFF0C8C0C0F0C9C0C1F0C5
:1079E600120073EC6FF037EC6FF004EC70F0000EE1
:1079F6000101656F000E426E000E416F000E406F72
:107A0600000E3F6F000E3E6F000E666F000EB8EC64
:107A160022F0000E0001916F000E906F000E936F22
:107A2600000E926F000E956F000E946F485023EC77
:107A360051F07AEC72F0C8EC5BF068EC72F090C032
:107A46003CF191C03DF13DEC72F033EC72F0B4ECD8
:107A560070F0000E0101516F080E506F46EC72F087
:107A6600000ECEEC5CF049A202D08A8001D08A904A
:107A7600000E0101476F000E466F43EC5DF0000EED
:107A860001014D6F200E4C6FF28CF28E1CEC6BF0E8
:107A9600FA0E0001D46F010ED56F62EC43F0000EB2
:107AA6000101536F000E526F4B505FEC25F088ECCE
:107AB60047F086EC70F049A40CD0010146514711FD
:107AC600D8A407D0BBEC71F0000E0101476F800E01
:107AD600466F49AA0BD0010144514511D8A406D0DE
:107AE600000E456F100E446F0EEC6AF07CEC6AF0E7
:107AF60071EC63F001016651D8A440D05051511188
:107B0600D8A407D043EC1AF0000E0101516F080EFD
:107B1600506F52515311D8A415D0FA0E0001D46FEC
:107B2600010ED56F62EC43F00101FA51D8A433EC93
:107B360072F088EC47F0BDEC36F0010E0101536F90
:107B4600400E526F000EED6F000EF56F13D0F5511B
:107B56000D0D0B0EF326000EF4224C0EF324D96EF7
:107B6600020EF420DA6EDE50DE10D8B402D0010E1A
:107B7600ED6FF52B4B50F55DD8A0E9D7000EEE6FF3
:107B8600000EEF6F65A106D03E513F11D8A402D07A
:107B9600010EEE6F65A306D040514111D8A402D064
:107BA600010EEF6FED51D8B404D0080EB7EC56F0C5
:107BB60038D042A204D0060EB7EC56F032D042A618
:107BC60004D0070EB7EC56F02CD042A404D0050E14
:107BD600B7EC56F026D00101EE51D8B404D0030E0E
:107BE600B7EC56F01ED00101EF51D8B404D0040E04
:107BF600B7EC56F016D042A004D0020EB7EC56F001
:107C060010D0020E01016419D8B404D0030E641911
:107C1600D8A404D0010EB7EC56F003D0000EB7EC92
:107C260056F001014E514F11D8B4B8EC65F0F60E7E
:107C360000019D6F010E9E6FE50E9F6F010EA06FF6
:107C4600F40EA16F010EA26FF00EA36F010EA46FCA
:107C5600F20EA56F010EA66F1FEC33F00009D8B423
:107C66002AD7F6C1EFF0F7C1F0F0F8C1F1F0F9C18B
:107C7600F2F0E50E0001F36F010EF46FF4C1F5F0BA
:107C8600F0C1F6F0F1C1F7F0F2C1F8F0F3C1F9F086
:107C9600F1EC2CF010D7F2C095F0F3C096F0F4C0DA
:107CA60097F0F5C098F0A80E0001996F1B0E9A6F19
:107CB600FA0E9B6F000E9C6FDFEC70F00009D8A4E3
:107CC60011D134D1A50E0001916F220E926F8EEC68
:107CD6006EF0120043EC5DF0000E00019E6F010E87
:107CE6009D6F4950FE0B9F6F17EC6FF0496E000EAB
:107CF6000101646F000E4F6F000E4E6F12008A90E6
:107D0600000E9E6F010E9D6F4950FD0B9F6F17EC85
:107D16006FF0496E1200BBEC71F0000E00019E6F11
:107D2600010E9D6F4950FB0B9F6F17EC6FF0496E6C
:107D36001200F2C095F0F3C096F0F4C097F0F5C0CB
:107D460098F0290E0001996F290E9A6FFA0E9B6F13
:107D5600000E9C6FDFEC70F00009D8B432D0000E34
:107D66000001FB6F070EFB6501D024D0FB51010D0E
:107D7600000EF324D96E010EF420DA6E240EFB25D4
:107D86009D6F9E6B000E9E23000E9F6F17EC6FF08B
:107D9600DF6E0001FB510D0D0A0EF326000EF422D4
:107DA6004C0EF324D96E020EF420DA6E000EDF6E4E
:107DB600FB2BD8D7D50E916F230E926F8EEC6EF0FB
:107DC6001200F2C09BF0F3C09CF0F4C09DF0F5C029
:107DD6009EF0FC0E00019F6F000EA06FF90EA16FC2
:107DE600000EA26F51EC60F00009D8B41200000139
:107DF600FC51010D000EF324D96E010EF420DA6E4B
:107E0600240EFC259D6F9E6B000E9E23FC51010DDA
:107E1600000EF324E16E010EF420E26EE750F66FD9
:107E2600F9C0F7F0010EF86FF72B02D0D890F837AB
:107E3600F72FFCD70001F851FF0AF6159F6F17ECD4
:107E46006FF0DF6EF9C0F6F0010E0001F76FF62B4A
:107E560002D0D890F737F62FFCD70001F751FF0A6A
:107E6600F86FFC510D0D0A0EF326000EF4224C0E8F
:107E7600F324D96E020EF420DA6EF851DF161200E2
:107E8600928092829392000E9E6F010E9D6F4950D2
:107E9600F70B9F6F17EC6FF0496E1200000E000192
:107EA6009E6F010E9D6F4950EF0B9F6F17EC6FF0A1
:107EB600496E1200000E00019E6F010E9D6F495023
:107EC6007F0B9F6F17EC6FF0496E1200000E0001DA
:107ED6009E6F010E9D6F4950DF0B9F6F17EC6FF081
:107EE600496E12000001FA51000AD8B4EBD6010A15
:107EF600D8B4F0D6030AD8B402D7010AD8B40BD73F
:107F0600070AD8B416D7010AD8B413D7030AD8B4C7
:107F160010D7010AD8B4B4D70F0AD8B4BFD7010A0C
:107F2600D8B4C8D7030AD8A41200D0D78E0E000141
:107F3600916F230E926F8EEC6EF01200F2C095F0E8
:107F4600F3C096F0F4C097F0F5C098F0A80E0001C3
:107F5600996F1B0E9A6FFA0E9B6F000E9C6FDFECEB
:107F660070F00009D8A40CD12FD1F0EC34F0120037
:107F760043EC5DF0000E00019E6F010E9D6F4950AF
:107F860001099F6F17EC6FF0496E12008A80000E90
:107F96009E6F010E9D6F495002099F6F17EC6FF09F
:107FA600496E120049B41200000E9E6F010E9D6FBD
:107FB600495004099F6F17EC6FF0496EBBEC71F0E6
:107FC6001200F2C095F0F3C096F0F4C097F0F5C039
:107FD60098F0290E0001996F290E9A6FFA0E9B6F81
:107FE600000E9C6FDFEC70F00009D8B43AD0000E9A
:107FF6000001FC6F070EFC6501D02CD0FC51010D71
:10800600000EF324D96E010EF420DA6E240EFC2540
:108016009D6F9E6B000E9E23FC51010D440EF324B2
:10802600E16E020EF420E26EE7509F6F17EC6FF0E0
:10803600DF6E0001FC510D0D0A0EF326000EF42230
:108046004C0EF324D96E020EF420DA6E000EDF6EAB
:10805600FC2BD0D71A0E916F240E926F8EEC6EF019
:108066001200F2C09BF0F3C09CF0F4C09DF0F5C086
:108076009EF0FB0E00019F6F000EA06FF90EA16F20
:10808600000EA26F51EC60F00009D8B41200000196
:10809600FB51010D000EF324D96E010EF420DA6EA9
:1080A600240EFB259D6F9E6B000E9E23FB51010D3A
:1080B600000EF324E16E010EF420E26EE750F66F37
:1080C600F9C0F7F0010EF86FF72B02D0D890F83709
:1080D600F72FFCD70001F851F6119F6F17EC6FF0E0
:1080E600DF6E0001FB510D0D0A0EF326000EF42281
:1080F6004C0EF324D96E020EF420DA6E000EDF6EFB
:1081060012000101FFA308D0500E0001916F220E4C
:10811600926F8EEC6EF01200938292909292000E05
:1081260000019E6F010E9D6F495008099F6F17EC65
:108136006FF0496E120049B81200000E9E6F010ED4
:108146009D6F495010099F6F17EC6FF0496E120032
:10815600000E00019E6F010E9D6F495080099F6FB2
:1081660017EC6FF0496E1200000E00019E6F010EB3
:108176009D6F495020099F6F17EC6FF0496E1200F2
:108186000001FA51000AD8B4F0D6010AD8B4F0D6E4
:10819600030AD8B4FBD6010AD8B404D7070AD8B460
:1081A60010D7010AD8B40DD7030AD8B40AD7010AE2
:1081B600D8B4A7D70F0AD8B4BED7010AD8B4C8D73F
:1081C600030AD8A41200D0D78E0E0001916F230E99
:1081D600926F8EEC6EF012004B50CAEC70F0000EEF
:1081E6000101BE6F32D1000EBD6F000EBC6FBE51D5
:1081F6000D0D040EF326000EF4224C0EF324D96E58
:10820600020EF420DA6EDECFAAF1DDCFABF1BE515D
:108216000D0D4C0EF324D96E020EF420DA6E020117
:10822600000EDFB0010E0101BA6FBA51D8B482D088
:10823600000EBB6FBB51D8A47DD0BE510C0DF3CF41
:10824600B0F1000EB16F000EB76F010EB76501D029
:1082560071D0000EB26F000EB66F000EB56F000E35
:10826600BF6F050EBF6501D049D0B051020D000E9B
:10827600F324D96E050EF420DA6EDECFB8F1DDCF29
:10828600B9F1B8513A5DB9513B59D8B032D0190E4F
:10829600A7250001EB6F000E0101A8210001EC6F7C
:1082A6000101B8510001EB5D0101B9510001EC5922
:1082B600D8B01FD0A7C1EBF0A8C1ECF0EB1FEC1FA4
:1082C600EB4BEC2B0101B8510001EB250101B36F1B
:1082D600B9510001EC210101B46FB351B55DB45140
:1082E600B659D8B006D0B3C1B5F1B4C1B6F1B1C173
:1082F600B2F10101B12BB02BBF2BB3D7B551B611DB
:10830600D8B416D0B2C1EBF0010E0001EC6F000E2E
:10831600ED6FEB2B03D0D890EC37ED37EB2FFBD777
:108326000001EC510101BC130001ED510101BD1327
:10833600B72B8BD7BC1D0001EB6F0101BD1D0001E2
:10834600EC6F0101AA510001EB150101AC6FAB51B5
:108356000001EC150101AD6FBCC1AEF1BDC1AFF1BD
:108366004AA456D0000EBF6F0B0EBF6501D050D089
:10837600BFC1EBF0010E0001EC6F000EED6FEB2BB1
:1083860003D0D890EC37ED37EB2FFBD70101AE5178
:108396000001EC170101AF510001ED17EC51ED1191
:1083A600D8B40DD0BFC1E4F0010EE56FBAC1E6F056
:1083B600BBC1E7F00101BE5126EC64F026D0BFC177
:1083C600EBF0010E0001EC6F000EED6FEB2B03D00E
:1083D600D890EC37ED37EB2FFBD70101AC510001FC
:1083E600EC170101AD510001ED17EC51ED11D8B4B8
:1083F6000CD0BFC1E4F0000EE56FBAC1E6F0BBC118
:10840600E7F00101BE5126EC64F00101BF2BACD7A9
:10841600BE510D0D040EF326000EF4224C0EF3246D
:10842600D96E020EF420DA6EBCC1DEFFBDC1DDFFDF
:10843600010E00019E6FBCC19FF0BDC1A0F00101FD
:10844600BE514CEC5CF00101BE2B4B50BE5DD8B06A
:108456001200C9D6000E0001CA6F5D0E916F230E81
:10846600926F8EEC6EF0000E0001CC6F070ECC659D
:1084760001D01200CC51010D3C0EF324D96E020E30
:10848600F420DA6EDF50CF6F080ECF6115D14B5056
:10849600CF5DD8A010D0CF51030D010EF326000EEC
:1084A600F4226B0EF324D96E010EF420DA6EDE5040
:1084B600DE10D8B401D1CF51030D6B0EF324D96E63
:1084C600010EF420DA6E0101DF380F0B0001CD6FCB
:1084D600CF51030D6B0EF324D96E010EF420DA6E24
:1084E6000101DF500F0B0001CB6FCA51CD19D8B473
:1084F60006D0220E916F1F0E926F8EEC6EF0E70E75
:108506000001916F240E926F8EEC6EF0010E000149
:10851600CF25B86FB96B000EB923010EBA6FADEC5B
:108526006FF0C30E0001916F280E926F8EEC6EF005
:108536000001CA51CD19D8B40AD0CDC0B8F0B96B74
:10854600010EBA6FADEC6FF0CDC0CAF007D0E80EE1
:108556000001916F240E926F8EEC6EF0C30E000137
:10856600916F280E926F8EEC6EF0010E0001CB25F6
:10857600B86FB96B000EB923010EBA6FADEC6FF090
:10858600D70E0001916F280E926F8EEC6EF04C0E96
:108596000001BB6F290EBC6FCB510C0DF328D4EC38
:1085A6006EF0480E0001BB6F290EBC6FCB290C0D77
:1085B600F350D4EC6EF0000E0001CE6F0B0ECE65BC
:1085C60001D074D0CF51030D010EF326000EF42214
:1085D6006B0EF324D96E010EF420DA6EDECFC2F0F4
:1085E600DDCFC3F0CEC0C4F0010EC56F000EC66F5E
:1085F600C42B03D0D890C537C637C42FFBD700018C
:10860600C251C517C351C617C551C611D8B402D039
:10861600010E01D0000EC76F000EC86FCF510C0DB2
:10862600CE51F326000EF422D890F336F436000E1F
:10863600F324D96E060EF420DA6E010EDB5004E147
:10864600C90EDE5CD8A006D04B50CF5DD8B002D0A4
:10865600010EC86FC8C0C9F0C751D8B412D0C951ED
:10866600D8B407D0420E916F290E926F8EEC6EF041
:108676001AD0390E0001916F290E926F8EEC6EF0B2
:1086860012D00001C951D8B407D0360E916F290E09
:10869600926F8EEC6EF007D0E70E0001916F240EFC
:1086A600926F8EEC6EF00001CE2B88D7D20E916FB2
:1086B6001A0E926F8EEC6EF00001CC2BD7D6000E00
:1086C60000019B6F080E9EEC69F055EC70F055ECBE
:1086D60070F0E0EC71F055EC70F055EC70F0400E77
:1086E6000001BC6F040EBD6F000E4EEC67F04BC070
:1086F600E5F0000E4B6E000E0001E46F000EE86F11
:10870600070EE86501D052D0E8510D0D4C0EF3244A
:10871600E66F020EF420E76FE8C0D6F0010ED76FC1
:10872600D62B02D0D890D737D62FFCD70001D751F9
:10873600040140150009D8B404D00001E451D8B4AE
:1087460013D0E6C0D9FFE7C0DAFF0001DF9020EEC4
:108756000BF0E651D926E751DA22000EDE6E000E46
:10876600DD6E010EE46F20D0E851060D710EF32484
:10877600E26F040EF420E36FE6C0D9FFE7C0DAFF2C
:10878600DF8020EE01F0E651D926E751DA2210EE1D
:1087960005F0E251E126E351E222E750D66FD639E1
:1087A6000F0B0F0BDF6E4B2AE82BAAD74B500C0D85
:1087B600F3CF43F0E5514B18D8B402D0010E01D0E7
:1087C600000ED4C0D9FFD5C0DAFFDF6ED4C0D9FF02
:1087D600D5C0DAFFDF50D8B480D04B505FEC25F01F
:1087E600000E0001E86F52D0E8510D0D4C0EF32437
:1087F600E66F020EF420E76F710E916F270E926FEF
:108806008EEC6EF0010E0001E825B86FB96B000E14
:10881600B923010EBA6FADEC6FF0B20E0001916F85
:10882600260E926F8EEC6EF0000120EE0BF0E651F4
:10883600D926E751DA22DE50DE10D8B41ED0460E15
:10884600916F240E926F8EEC6EF0000120EE0BF00D
:10885600E651D926E751DA22DECF90F0DDCF91F04E
:10886600D80E926F000E936FB5EC62F0D80E000131
:10887600916F000E926F8EEC6EF0D20E0001916F2A
:108886001A0E926F8EEC6EF00001E82B4B50E85DED
:10889600D8A0AAD74BC0E8F01AD0710E916F270E58
:1088A600926F8EEC6EF0010E0001E825B86FB96B81
:1088B600000EB923010EBA6FADEC6FF0AA0E0001DF
:1088C600916F240E926F8EEC6EF00001E82BE5514D
:1088D600E85DD8A0E2D7B2EC6BF0000E00019B6F0A
:1088E6004B509EEC69F012003DC0E9F03EC0EAF044
:1088F6000001E91FEA1FE94BEA2B3B50E925906F7F
:108906003C50EA21916F000E936F0D0E926FA0EC12
:108916006DF090C01AF191C01BF101014A514B1143
:10892600D8A4E3D0000E4B6F080E4A6F412A100EF2
:10893600416402D0000E416E41C0E9F0070E00010D
:10894600E917D8A40FD0010118A330D0000E0001FA
:10895600E26F000EE16F000EE46F020EE36FB3EC00
:108966006AF024D04150070B040AD8A40FD00101A5
:1089760018AD1CD0000E0001E26F000EE16F000E74
:10898600E46F400EE36FB3EC6AF010D041A00ED056
:10899600010118A90BD0000E0001E26F000EE16F75
:1089A600000EE46F100EE36FB3EC6AF049A48FD0AB
:1089B600010116511711D8B403D01607D8A017070E
:1089C60016511711D8A411D0FDEC65F001015C51C8
:1089D600D8A45C075C51D8A404D0000E176F300EE3
:1089E60003D0000E176F010E166F41B06AD089ECE6
:1089F60072F00001EE6FEE51D8A41FD013EC56F0C2
:108A0600000E0001C26F00C2B0F001C2B1F002C296
:108A1600B2F003C2B3F0E80EB46F030EB56F000EEA
:108A2600B66F000EB76FBCEC60F0B0C0C3F0B1C05B
:108A3600C4F0000E35EC5AF04AD06DEC55F000014A
:108A4600EE05D8A407D038C1ECF039C1EDF05FC10E
:108A5600EBF01CD0020EEE19D8A407D036C1ECF00C
:108A660037C1EDF05EC1EBF011D0030EEE19D8A4BC
:108A760005D0A7C1ECF0A8C1EDF008D0040EEE19A0
:108A8600D8A404D030C1ECF031C1EDF0320EEC25A3
:108A9600906F000EED21916F000E936F640E926F32
:108AA600A0EC6DF090C0ECF091C0EDF0EBC0C2F020
:108AB600ECC0C3F0EDC0C4F00001EE5135EC5AF045
:108AC60006D0B8EC5DF080EC72F06AEC71F0010152
:108AD60018A50BD0000E0001E26F000EE16F000E2C
:108AE600E46F040EE36FB3EC6AF0010148514911DB
:108AF600D8A41200000E196F000E186F12004AC09B
:108B0600A6F0A1C095F0A2C096F0A3C097F0A4C0AD
:108B160098F0030E0001996F240E9A6FA70E9B6FB3
:108B2600000E9C6FDFEC70F00009D8A4C3D0E3D030
:108B360001016851D8B40FD068C1A6F00001A6A102
:108B460006D0C10E916F220E926F8EEC6EF0000E63
:108B56000101686FC1D04AC068F1000E0001A66F1E
:108B66002B0E916F230E926F8EEC6EF0B5D0A1C0D6
:108B760095F0A2C096F0A3C097F0A4C098F0EE0EB0
:108B86000001996F260E9A6FA70E9B6F000E9C6FC1
:108B9600DFEC70F00009D8B49FD00001A751D8B41B
:108BA60059D07C0E916F1E0E926F8EEC6EF01D0EDC
:108BB6000001916F210E926F8EEC6EF0F40E0001A3
:108BC600916F210E926F8EEC6EF0A50E0001916FE3
:108BD600000E926F2EEC69F00009D8B4F6D70001AA
:108BE600A705D8A40FD0000E916F000E906F000E4F
:108BF600936F000E926F000E956F000E946F020E2B
:108C060023EC51F0020E0001A719D8A40FD0000ED4
:108C1600916F000E906F000E936F000E926F000E14
:108C2600956F000E946F030E23EC51F0030E0001B6
:108C3600A719D8A40FD0000E916F000E906F000EEA
:108C4600936F000E926F000E956F000E946F040ED8
:108C560023EC51F00001A681000E0101686FC10EE0
:108C66000001916F220E926F8EEC6EF035D0000EE1
:108C76000001A66F000E0101686F2B0E0001916FB7
:108C8600230E926F8EEC6EF027D00001A685000EA3
:108C96000101686F6D0E0001916F220E926F8EECCE
:108CA6006EF01AD0A60E0001916F230E926F8EEC15
:108CB6006EF012D00001A751000AD8B439D7010AC4
:108CC600D8B455D7030AD8B452D7010AD8B4CFD7E7
:108CD600070AD8B4DAD7E6D74A500001A619D8B49D
:108CE6001200000E9E6F000E9D6FA6C09FF017EC3F
:108CF6006FF04A6E1200A60E0001916F230E926F5E
:108D06008EEC6EF01200BEC090F0BFC091F0C0C0F5
:108D160092F0C1C093F0A0EC6DF090C0D1F091C07C
:108D2600D2F0D1C097F0D2C098F0C0C099F0C1C0BF
:108D36009AF030EC71F097C0D9F098C0DAF0D9C04B
:108D4600C6F0DAC0C7F00001C61FC71FC64BC72B47
:108D5600BE51C625CE6FBF51C721CF6F000EDB6F48
:108D6600C80ED56F000ED66FD1C0DCF0D2C0DDF0D4
:108D760041D0DCC090F0DDC091F0000E936F0A0E7A
:108D8600926FA0EC6DF090C0D9F091C0DAF0D9C026
:108D960097F0DAC098F0000E00019A6F0A0E996FEC
:108DA60030EC71F00001971F981F974B982BDC5100
:108DB6009725D36FDD519821D46FD9C0DCF0DAC086
:108DC600DDF0DC51DD11D8A407D0D351D411D8A4DD
:108DD60003D0DB51D8A403D0D351300F01D0200EDD
:108DE600D06FD5C0D9FFD6C0DAFFD0C0DFFFD54BD4
:108DF600D62BDB2BDC51DD11D8A4BBD7C251DB5DF2
:108E0600D8A0B7D7C4C0D7F0C5C0D8F010D0D50702
:108E1600D8A0D607D5C0D9FFD6C0DAFFD7C0E1FFA4
:108E2600D8C0E2FFDFCFE7FFD74BD82BDB07DB51FC
:108E3600D8A4EDD7C351D8B461D0D7C0D9FFD8C014
:108E4600DAFF2E0EDF6ED74BD82B000EDB6FC80E67
:108E5600D56F000ED66FCEC0DCF0CFC0DDF032D0BD
:108E6600DCC090F0DDC091F0000E936F0A0E926F99
:108E7600A0EC6DF090C0D9F091C0DAF0D9C097F0AF
:108E8600DAC098F0000E00019A6F0A0E996F30EC66
:108E960071F00001971F981F974B982BDC5197256F
:108EA600D36FDD519821D46FD9C0DCF0DAC0DDF084
:108EB600D351300FD5C0D9FFD6C0DAFFDF6ED54B00
:108EC600D62BDB2BDC51DD11D8A4CAD7C351DB5D11
:108ED600D8B011D0C5D7D507D8A0D607D5C0D9FFE9
:108EE600D6C0DAFFD7C0E1FFD8C0E2FFDFCFE7FF89
:108EF600D74BD82BDB07DB51D8A4EDD7D7C0D9FF8A
:108F0600D8C0DAFF000EDF6E1200010E90EC6FF093
:108F16000D0E0001986FAC0E976F3BEC70F0000ED3
:108F26000001BC6F060EBD6FD40EBE6F000EBF6F84
:108F3600000E8BEC58F0000E0001D86F070ED865B6
:108F460001D051D0000ED66F000ED56FD8510D0D41
:108F56004C0EF324D96E020EF420DA6E0201DFA065
:108F66002FD0000E0001D76F0B0ED76501D028D089
:108F7600D8510C0DF350D725D16FD151020D000EEB
:108F8600F324D96E060EF420DA6E010EDB5004E1EE
:108F9600C90EDE5CD8A012D0D7C0C4F0010EC56FD2
:108FA600000EC66FC42B03D0D890C537C637C42F62
:108FB600FBD70001C551D513C651D613D72BD4D72D
:108FC6000001D8510D0D020EF326000EF4224C0EB0
:108FD600F324D96E020EF420DA6ED5C0DEFFD6C0B9
:108FE600DDFFD82BABD74292000ED86F070ED8659F
:108FF60001D01200D851030D010EF326000EF42203
:109006006B0EF324D96E010EF420DA6EDECFD2F0A9
:10901600DDCFD3F0D8510D0D020EF326000EF4224B
:109026004C0EF324D96E020EF420DA6EDECFD5F0A4
:10903600DDCFD6F0D251D515C46FD351D615C56F35
:10904600D251C41904E1D351C519D8B45BD04282B8
:10905600710E916F270E926F8EEC6EF0010E00016D
:10906600D825B86FB96B000EB923010EBA6FADECF7
:109076006FF0450E0001916F210E926F8EEC6EF02F
:109086004AA439D0090E0001916F290E926F8EEC19
:109096006EF0D2C090F0D3C091F0C70E0001926F6F
:1090A600000E936FB5EC62F0C70E0001916F000ED3
:1090B600926F8EEC6EF00D0E0001916F290E926F7D
:1090C6008EEC6EF0D5C090F0D6C091F0C70E0001C0
:1090D600926F000E936FB5EC62F0C70E0001916FB0
:1090E600000E926F8EEC6EF0480E0001916F290E05
:1090F600926F8EEC6EF0D20E0001916F1A0E926F87
:109106008EEC6EF00001D82B71D70001B16F2A509A
:109116000CE10F0E295CD8B008D0010E29240001FD
:10912600B26F000E2A20B36F05D0000E0001B36F98
:10913600000EB26F2750B2190EE12850B319D8A409
:109146000AD00201C84BC92BD00E0001B76F020E20
:10915600B86F000EC9D029C097F02AC098F0000E4B
:109166009A6F110E996F30EC71F0000E0001972581
:10917600B76F0C0E9821B86F080EB06502D0080EB6
:10918600B06F20EE04F0B751D926B851DA22ACC040
:10919600DFFF20EE05F0B751D926B851DA22ADC06F
:1091A600DFFF20EE06F0B751D926B851DA22B1C05A
:1091B600DFFF20EE07F0B751D926B851DA22ABC04F
:1091C600DFFF20EE08F0B751D926B851DA22B0C039
:1091D600DFFF090EB725B56F000EB821B66FAEC01A
:1091E600D9FFAFC0DAFFB5C0E1FFB6C0E2FFDFCFFF
:1091F600E7FFAE4BAF2BB54BB62BAEC0D9FFAFC01A
:10920600DAFFB5C0E1FFB6C0E2FFDFCFE7FFAE4B46
:10921600AF2BB54BB62BAEC0D9FFAFC0DAFFB5C08A
:10922600E1FFB6C0E2FFDFCFE7FFAE4BAF2BB54B9A
:10923600B62BAEC0D9FFAFC0DAFFB5C0E1FFB6C0EE
:10924600E2FFDFCFE7FFAE4BAF2BB54BB62BAEC081
:10925600D9FFAFC0DAFFB5C0E1FFB6C0E2FFDFCF8E
:10926600E7FFAE4BAF2BB54BB62BAEC0D9FFAFC0A9
:10927600DAFFB5C0E1FFB6C0E2FFDFCFE7FFAE4BD6
:10928600AF2BB54BB62BAEC0D9FFAFC0DAFFB5C01A
:10929600E1FFB6C0E2FFDFCFE7FFAE4BAF2BB54B2A
:1092A600B62BAEC0D9FFAFC0DAFFB5C0E1FFB6C07E
:1092B600E2FFDFCFE7FFAE4BAF2BB54BB62B2A5005
:1092C6000BE10F0E295CD8B007D0010E2924296EB8
:1092D600000E2A202A6E04D0000E2A6E000E296E79
:1092E6006FEC38F0010E0001B46FB4511200000E9D
:1092F6000101DA6F000ED96FD6C195F0D7C196F08D
:10930600D90E0001976F010E986F4E0E996F1B0EC6
:109316009A6FD80E9B6F010E9C6FDFEC70F0000900
:10932600D8A491D0CCD0D6C196F0D7C197F0D90E9B
:109336000001986F010E996F87EC66F01200D6C196
:10934600ECF0D7C1EDF0D90E0001EE6F010EEF6F14
:10935600ABEC14F01200D6C1D2F1D7C1D3F1D90EBD
:109366000101D46F010ED56FC5EC54F01200D6C1C1
:10937600A1F0D7C1A2F0D90E0001A36F010EA46F10
:1093860082EC45F01200D6C1F2F0D7C1F3F0D90E47
:109396000001F46F010EF56FA1EC3FF01200D6C18B
:1093A600F2F0D7C1F3F0D90E0001F46F010EF56F9C
:1093B6004EEC3EF01200D6C1F2F0D7C1F3F0D90E52
:1093C6000001F46F010EF56F30EC4DF01200D6C1BE
:1093D60090F0D7C191F0D90E0001926F010E936FF4
:1093E60092EC72F01200D6C1AEF0D7C1AFF0D90E32
:1093F6000001B06F010EB16FF5EC68F01200D6C136
:1094060096F0D7C197F0D90E0001986F010E996FAB
:10941600E8EC6AF01200D6C1D9F0D7C1DAF0D90E5D
:109426000001DB6F010EDC6F9AEC5EF01200D6C114
:10943600A0F0D7C1A1F0D90E0001A26F010EA36F53
:1094460001EC4EF012000101D851000AD8B4120006
:10945600010AD8B468D7030AD8B465D7010AD8B4C4
:109466006ED7070AD8B46BD7010AD8B474D7030AE3
:10947600D8B471D7010AD8B47AD70F0AD8B477D737
:10948600010AD8B480D7030AD8B47DD7010AD8B464
:1094960086D7070AD8B483D7010AD8B48CD7030A6B
:1094A600D8B495D7010AD8B49ED71F0AD8B4A7D77F
:1094B600010AD8B4B0D7030AD8A41200B8D7440E0C
:1094C6000001916F230E926F8EEC6EF01200000E6B
:1094D60000019B6F080E9EEC69F04B505FEC25F087
:1094E600010E90EC6FF00D0E0001986FAC0E976FA9
:1094F6003BEC70F0000E0001BC6F060EBD6FDE0E79
:10950600BE6F000EBF6F4B508BEC58F010EC72F034
:109516000B0E0001986FB80E976F3BEC70F0280E9B
:109526000001BC6F030EBD6F4B5045EC6AF0F50EA3
:109536000001916F200E926F8EEC6EF0A10E00016D
:10954600916F200E926F8EEC6EF0000E0001DF6FB1
:10955600A9D0DF51060D410EF324D66F040EF42078
:10956600D76FDF51060D710EF324D86F040EF42069
:10957600D96FDF51060D290EF324DC6F030EF4209C
:10958600DD6FDF51060D590EF324DA6F030EF4205A
:10959600DB6FE70E916F240E926F8EEC6EF0010E6C
:1095A6000001DF25B86FB96B000EB923010EBA6F43
:1095B600ADEC6FF07C0E0001916F280E926F8EEC71
:1095C6006EF04B500001DF5DD8B063D0DF510D0D5A
:1095D6000B0EF326000EF4224C0EF324D96E020E67
:1095E600F420DA6EDE50DE10D8A44CD0010EBB6F2C
:1095F600DCC0D9FFDDC0DAFFDECFBCF0DDCFBDF0C9
:10960600DF51E6EC51F0020E0001BB6F20EE02F0D6
:10961600DC51D926DD51DA22DECFBCF0DDCFBDF03C
:10962600DF51E6EC51F0030E0001BB6F20EE04F0B3
:10963600DC51D926DD51DA22DECFBCF0DDCFBDF01C
:10964600DF51E6EC51F0040E0001BB6FDAC0D9FF22
:10965600DBC0DAFFDECFBCF0DDCFBDF0DF51E6ECDC
:1096660051F0050E0001BB6F20EE02F0DA51D9264B
:10967600DB51DA22DECFBCF0DDCFBDF0DF51E6EC08
:1096860051F007D0F00E0001916F280E926F8EEC0C
:109696006EF0D20E0001916F1A0E926F8EEC6EF084
:1096A6000001DF2B4B50DF5DD8B0120052D700010E
:1096B600B36F9EC0CFF39FC0D0F30001B351D8A4BF
:1096C60007D0080EAE6F010EB26F0301CC2B07D088
:1096D600B3C0AEF0020E0001B26F0301CD2B000E37
:1096E6000001B86FC8D08B949EC091F09FC092F0D5
:1096F6001CEC72F0A0C091F0A1C092F01CEC72F0CC
:10970600A4C0ACF0A5C0ADF0A6C0D9FFA7C0DAFFD3
:10971600000EDF6E010E0001B86F000EB96F9DD00E
:10972600ACC0AAF0ADC0ABF0E10EBA6F020EBB6FD3
:10973600000EB16F18D0BAC091F0BBC092F0F2EC37
:109746006CF0AAC0D9FFABC0DAFF000191C0DEFF02
:1097560092C0DDFF020EAA27000EAB23BA4BBB2B2D
:10976600BA4BBB2BB12BA251B15DD8A0E4D7BAC07E
:1097760091F0BBC092F01EEC6DF091C0AFF092C0BC
:10978600B0F00001BA4BBB2BBA4BBB2BE10E906F6E
:10979600020E916FB151020DF3CF92F0F4CF93F018
:1097A60024EC65F090C0B4F091C0B5F00001B5515D
:1097B600BAC0D9FFBBC0DAFFDF6EBA4BBB2BBAC04B
:1097C600D9FFBBC0DAFFB4C0DFFFBA4BBB2BB95120
:1097D600030DD10EF324B66F030EF420B76FAF510D
:1097E600B4191BE1B051B519D8A417D0B9C0A8F067
:1097F600010EA96FA82B02D0D890A937A82FFCD7A5
:10980600A6C0D9FFA7C0DAFF0001A951DF12B6C072
:10981600D9FFB7C0DAFFDF2A19D0AF290EE1B02988
:10982600D8A40BD020EE01F0B651D926B751DA22D2
:10983600DF2AB351D8B40AD007D020EE02F0B651D1
:10984600D926B751DA22DF2A000EB86FA351020DCE
:10985600F350AC27F450AD23B92BAE51B95DD8A067
:109866005FD78B84B207B251D8B405D0B851D8A40B
:1098760002D00301CE2B0001B251D8B41200B85168
:10988600D8A4120030D7000E0001B56FA60EB16F36
:10989600000EB26F9DC0B6F09EC0B7F04DD0B6C0F8
:1098A60090F0B7C091F0000E936F0A0E926FA0EC85
:1098B6006DF090C0AFF091C0B0F0AFC097F0B0C0FF
:1098C60098F0000E00019A6F0A0E996F30EC71F055
:1098D6000001971F981F974B982BB6519725AD6F90
:1098E600B7519821AE6FAFC0B6F0B0C0B7F0B65161
:1098F600B711D8A40BD0AD51AE11D8A407D0B5512D
:10990600D8B404D0020EA019D8A403D0AD51300F9C
:1099160009D0A005D8A402D0200E04D0A051D8A406
:1099260002D0000EAC6FB1C0D9FFB2C0DAFFACC036
:10993600DFFFB14BB22BB52BB651B711D8A4AFD7B9
:10994600B551D8B4ACD7A051D8B404D09F51B55DA9
:10995600D8A0A5D7A4C0B3F0A5C0B4F010D0B10765
:10996600D8A0B207B1C0D9FFB2C0DAFFB3C0E1FFD9
:10997600B4C0E2FFDFCFE7FFB34BB42BB507B55159
:10998600D8A4EDD7A351D8B461D0B3C0D9FFB4C021
:10999600DAFF2E0EDF6EB34BB42B000EB56FA60E9C
:1099A600B16F000EB26FA1C0B6F0A2C0B7F032D050
:1099B600B6C090F0B7C091F0000E936F0A0E926F8A
:1099C600A0EC6DF090C0AFF091C0B0F0AFC097F0D2
:1099D600B0C098F0000E00019A6F0A0E996F30EC35
:1099E60071F00001971F981F974B982BB65197253A
:1099F600AD6FB7519821AE6FAFC0B6F0B0C0B7F03B
:109A0600AD51300FB1C0D9FFB2C0DAFFDF6EB14B36
:109A1600B22BB52BB651B711D8A4CAD7A351B55D91
:109A2600D8B011D0C5D7B107D8A0B207B1C0D9FFF9
:109A3600B2C0DAFFB3C0E1FFB4C0E2FFDFCFE7FF99
:109A4600B34BB42BB507B551D8A4EDD7B3C0D9FFE6
:109A5600B4C0DAFF000EDF6E1200F2C095F0F3C05C
:109A660096F0F4C097F0F5C098F0250E0001996FB6
:109A7600290E9A6FAF0E9B6F010E9C6FDFEC70F094
:109A86000009D8A40BD013D0320E0001916F220E1C
:109A9600926F8EEC6EF043EC5DF012000101AF5157
:109AA600000AD8B4F1D7010AD8A41200EDD7F2C043
:109AB60095F0F3C096F0F4C097F0F5C098F0B20EAA
:109AC6000001996F010E9A6F8DEC71F00009D8B400
:109AD6008DD0F2C095F0F3C096F0F4C097F0F5C0C3
:109AE60098F0B00E0001996F010E9A6F8DEC71F02F
:109AF6000009D8B405D0B2C1AAF1B0C1ABF105D006
:109B0600010E0101AA6FB2C1ABF1ABC198F0B40E60
:109B16000001996F010E9A6FAE0E9B6F010E9C6F3E
:109B26000101AA517DEC64F00009D8B457D00101B7
:109B3600B4510D0D040EF326000EF4224C0EF32440
:109B4600D96E020EF420DA6EDECFACF1DDCFADF1C8
:109B5600AEC1F6F0010E0001F76F000EF86FF62B9E
:109B660003D0D890F737F837F62FFBD70001F75117
:109B76000101AC130001F8510101AD13B4510D0DF3
:109B8600040EF326000EF4224C0EF324D96E020EB8
:109B9600F420DA6EACC1DEFFADC1DDFF010E0001BF
:109BA6009E6FACC19FF0ADC1A0F00101B4514CEC69
:109BB6005CF0030E0101646F1E0E4F6F000E4E6FB8
:109BC600AEC1E4F0010E0001E56F010EE66F000E76
:109BD600E76F0101B45126EC64F01200130E000188
:109BE600916F220E926F8EEC6EF01200EC0E000159
:109BF600916F230E926F8EEC6EF01200A0C095F05E
:109C0600A1C096F0A2C097F0A3C098F0AC0E0001D8
:109C1600996F000E9A6F8DEC71F00009D8B412009E
:109C26000001AC51AD11D8B41200AD5103E1090EDB
:109C3600AC5DD8B01200A0C092F0A1C093F0A2C053
:109C460094F0A3C095F0A4EC52F092C0A7F093C094
:109C5600A8F0010E0101666FFF0E0001AC25976F9B
:109C6600FF0EAD21986F000E9A6F0D0E996F30ECB6
:109C760071F04C0E00019725D96E020E9821DA6E0E
:109C86000201DF80FF0E0001AC25976FFF0EAD21AC
:109C9600986F000E9A6F0D0E996F30EC71F0020EF0
:109CA60000019727000E98234C0E9725D96E020EB9
:109CB6009821DA6EA7C0DEFFA8C0DDFFFF0EAC2537
:109CC600976FFF0EAD21986F000E9A6F0C0E996F6D
:109CD60030EC71F0D890000197379837000E972531
:109CE600A96F050E9821AA6F000EAB6F0B0EAB6520
:109CF60001D037D0ABC0A4F0010EA56F000EA66F41
:109D0600A42B03D0D890A537A637A42FFBD70001E4
:109D1600A751A517A851A617A551A611D8B413D0B7
:109D2600000EA46F800EA56FAB51200DA451F32633
:109D3600A551F422A9C0D9FFAAC0DAFFF3CFDEFFEE
:109D4600F4CFDDFF08D0A9C0D9FFAAC0DAFF000E04
:109D5600DE6E000EDD6E020EA927000EAA23AB2BC7
:109D6600C5D7800E0101A86F300EA76F4B500001BA
:109D7600A46FA56BAC51A45DAD51A559D8B008D060
:109D8600ACC04BF04B500C0DF3CF43F043C0A9F1E0
:109D9600B2EC6BF012006DEC55F0000E0001D16FC5
:109DA6009FC1CBF0A0C1CCF0CB1FCC1FCB4BCC2B93
:109DB600010130510001CB27010131510001CC23B3
:109DC600CB51CC11D8A413D0010130519F250001ED
:109DD600CB6F01013151A0210001CC6FCB1FCC1FED
:109DE600CB4BCC2BCBC0D2F0CCC0D3F012D09FC182
:109DF600CBF0A0C1CCF0CB1FCC1FCB4BCC2B0101A1
:109E060030510001CB25D26F010131510001CC2127
:109E1600D36FD35104E1330ED25DD8A002D0010E28
:109E2600D16F21EEA3F0DECFCBF0DDCFCCF0CB1F90
:109E3600CC1FCB4BCC2B0101A7510001CB27010135
:109E4600A8510001CC23CB51CC11D8A413D00101C9
:109E5600A751A3250001CB6F0101A851A421000140
:109E6600CC6FCB1FCC1FCB4BCC2BCBC0D4F0CCC0F4
:109E7600D5F014D021EEA3F0DECFCBF0DDCFCCF0C1
:109E8600CB1FCC1FCB4BCC2B0101A7510001CB25FF
:109E9600D46F0101A8510001CC21D56FD55104E141
:109EA600330ED45DD8A002D0010ED16F30C19FF120
:109EB60031C1A0F138C1A1F139C1A2F1A7C1A3F105
:109EC600A8C1A4F136C1A5F137C1A6F14C50CB6F9C
:109ED600CC6BCB3BCC3BF00ECC17CB510F0BCC1342
:109EE600F00ECB17F00ECB25CD6FFF0ECC21CE6F2B
:109EF600CF6BCEBFCF07CF51D06F000ECD25B96F38
:109F0600060ECE21BA6FDF0ECF21BB6F010ED02118
:109F1600BC6F9F0EBD6F010EBE6F080EBF6F81EC4A
:109F260068F012000F0130AF12000201CC4BCD2BAE
:109F36002E500BE10F0E2D5CD8B007D0010E2D244C
:109F46000B6E000E2E200C6E04D0000E0C6E000E52
:109F56000B6E2B500B1809E12C500C18D8A405D009
:109F6600D00E0F6E020E106E21D02DC001F02EC045
:109F760002F0000E046E110E036E57EC71F0100E17
:109F860001240F6E0D0E0220106E2E500BE10F0EE7
:109F96002D5CD8B007D0010E2D242D6E000E2E207C
:109FA6002E6E04D0000E2E6E000E2D6E0FC0D9FF41
:109FB60010C0DAFF07C0DEFF08C0DDFF20EE02F0AA
:109FC6000F50D9261050DA2209C0DEFF0AC0DDFF85
:109FD60020EE06F00F50D9261050DA2231CFDFFFDF
:109FE60020EE07F00F50D9261050DA2232CFDFFFCD
:109FF60020EE04F00F50D9261050DA2233CFDFFFBF
:10A0060020EE05F00F50D9261050DA2234CFDFFFAC
:10A0160020EE08F00F50D9261050DA2235CFDFFF98
:10A02600090E0F240D6E000E10200E6E0DC0D9FF06
:10A036000EC0DAFF36CFDFFF0D4A0E2A0DC0D9FF5C
:10A046000EC0DAFF37CFDFFF0D4A0E2A0DC0D9FF4B
:10A056000EC0DAFF38CFDFFF0D4A0E2A0DC0D9FF3A
:10A066000EC0DAFF39CFDFFF0D4A0E2A0DC0D9FF29
:10A076000EC0DAFF3ACFDFFF0D4A0E2A0DC0D9FF18
:10A086000EC0DAFF3BCFDFFF0D4A0E2A0DC0D9FF07
:10A096000EC0DAFF3CCFDFFF0D4A0E2A0DC0D9FFF6
:10A0A6000EC0DAFF3DCFDFFF0D4A0E2A0F01309FAB
:10A0B600120060AE12000201CA4BCB2B2E500BE1F0
:10A0C6000F0E2D5CD8B007D0010E2D240B6E000E9E
:10A0D6002E200C6E04D0000E0C6E000E0B6E2B5054
:10A0E6000B180BE12C500C18D8A407D0CE4BCF2B55
:10A0F600D00E0F6E020E106E21D02DC001F02EC0B4
:10A1060002F0000E046E110E036E57EC71F0100E85
:10A1160001240F6E0D0E0220106E2E500BE10F0E55
:10A126002D5CD8B007D0010E2D242D6E000E2E20EA
:10A136002E6E04D0000E2E6E000E2D6E0FC0D9FFAF
:10A1460010C0DAFF07C0DEFF08C0DDFF20EE02F018
:10A156000F50D9261050DA2209C0DEFF0AC0DDFFF3
:10A1660020EE06F00F50D9261050DA2261CFDFFF1D
:10A1760020EE07F00F50D9261050DA2262CFDFFF0B
:10A1860020EE04F00F50D9261050DA2263CFDFFFFD
:10A1960020EE05F00F50D9261050DA2264CFDFFFEB
:10A1A60020EE08F00F50D9261050DA2265CFDFFFD7
:10A1B600090E0F240D6E000E10200E6E0DC0D9FF75
:10A1C6000EC0DAFF66CFDFFF0D4A0E2A0DC0D9FF9B
:10A1D6000EC0DAFF67CFDFFF0D4A0E2A0DC0D9FF8A
:10A1E6000EC0DAFF68CFDFFF0D4A0E2A0DC0D9FF79
:10A1F6000EC0DAFF69CFDFFF0D4A0E2A0DC0D9FF68
:10A206000EC0DAFF6ACFDFFF0D4A0E2A0DC0D9FF56
:10A216000EC0DAFF6BCFDFFF0D4A0E2A0DC0D9FF45
:10A226000EC0DAFF6CCFDFFF0D4A0E2A0DC0D9FF34
:10A236000EC0DAFF6DCFDFFF0D4A0E2A609E1200B8
:10A246000001986F800E6F6E6E38E832070B040AB5
:10A25600D8A4FAD7000E726E040E00019819D8A47D
:10A2660005D0010E0E01436FE00E10D0020E000164
:10A276009819D8A407D0040E0E01436FB80E446F88
:10A28600050E06D0030E0E01436FA00E446F020E9C
:10A29600456F90C096F091C097F00001D890973323
:10A2A6009633D89097339633D89097339633965102
:10A2B6000E01F86F00019039E846E00B08090E011F
:10A2C600F96F92C096F093C097F00001D89097333B
:10A2D6009633D89097339633D890973396339651D2
:10A2E6000E01E06F00019239E846E00B0E01E16FC6
:10A2F60094C096F095C097F00001D89097339633A6
:10A30600D89097339633D8909733963396510E015B
:10A31600E46F00019439E846E00B0E01E56F000E8C
:10A32600FE6F000EFF6F000EFC6F080EFD6F000E35
:10A33600EA6F000EEB6F000EE86F080EE96F000E75
:10A34600EE6F000EEF6F000EEC6F080EED6F000E55
:10A35600EE6F000EEF6F000EF06F080EF16F000E3D
:10A36600EE6F000EEF6F000EF46F080EF56F708A39
:10A37600000E6F6E6E38E832070B0009D8B4FAD7B4
:10A38600000E606E000E0F01306F000E2E6E000E76
:10A396002D6E000E2C6E000E2B6E000E0101586FF6
:10A3A600000E116F000E106F000E0F6F000E0E6F75
:10A3B600000E2A6E000E296E000E286E000E276E05
:10A3C600070E766E12000001C16FBCC098F0BDC0CA
:10A3D60099F0ACEC59F098C0C3F099C0C4F00001F4
:10A3E600C151010D000EF324D96E010EF420DA6E70
:10A3F600DF50BE6FBBC0BFF0FF0EBF27010EC06FA0
:10A40600BF2B02D0D890C037BF2FFCD70001C05158
:10A41600BE15C26FC32915E1C429D8A412D0C251F2
:10A42600D8B407D0400E916F280E926F8EEC6EF066
:10A4360084D0E30E0001916F240E926F8EEC6EF0C5
:10A446007CD0FD0E0001C31915E1C429D8A412D091
:10A45600C251D8B407D0630E916F280E926F8EEC5E
:10A466006EF06BD0E30E0001916F240E926F8EECAE
:10A476006EF063D00001C251D8B458D0FE0EC31995
:10A486000AE1C429D8A407D04E0E916F280E926F08
:10A496008EEC6EF052D0200E08EC71F00001C4BFB5
:10A4A60006D0C4510BE10A0EC35DD8B007D0E70E43
:10A4B600916F240E926F8EEC6EF00FD00001C4BF28
:10A4C60006D0C4510AE1640EC35DD8B006D0E80ECA
:10A4D600916F240E926F8EEC6EF0C3C0B8F0C4C0BC
:10A4E600B9F0010E0001BA6FADEC6FF0430E08EC47
:10A4F60071F044500001BE6FBF6BC351BE5DBF51CA
:10A50600800AC06FC451800AC059D8B007D04A0E1D
:10A51600916F290E926F8EEC6EF00FD0E80E00014F
:10A52600916F240E926F8EEC6EF007D0390E0001FB
:10A53600916F280E926F8EEC6EF0200E08EC71F083
:10A546001200000E0001986F000E9A6F000E996FB0
:10A5560094C0D9FF95C0DAFFDFCF96F0010EDE2654
:10A56600DFCF97F0000EDD2296519225D96E9751D6
:10A576009321DA6EDF509B6F200E9B19D8B4E8D773
:10A586009B51F6EC6EF000019C6F100E9C6190D012
:10A596009CC099F09A6B94C0D9FF95C0DAFFDFCFC3
:10A5A60096F0010EDE26DFCF97F0000EDD229651E3
:10A5B6009225D96E97519321DA6EDF509B6F9B518E
:10A5C600F6EC6EF000019C6F100E9C6171D099C084
:10A5D60096F09AC097F0963B973BF00E97179651D8
:10A5E6000F0B9713F00E96179C519625996F000E38
:10A5F60097219A6F94C0D9FF95C0DAFFDFCF96F006
:10A60600010EDE26DFCF97F0000EDD229651922551
:10A61600D96E97519321DA6EDF509B6F9B51F6EC02
:10A626006EF000019C6F100E9C6142D099C096F0AE
:10A636009AC097F0963B973BF00E971796510F0BE3
:10A646009713F00E96179C519625996F000E972139
:10A656009A6F94C0D9FF95C0DAFFDFCF96F0010E4E
:10A66600DE26DFCF97F0000EDD2296519225D96EB9
:10A6760097519321DA6EDF509B6F9B51F6EC6EF08B
:10A6860000019C6F100E9C6113D099C096F09AC081
:10A6960097F0963B973BF00E971796510F0B971333
:10A6A600F00E96179C519625996F000E97219A6F7A
:10A6B60099C092F09AC093F01200BBC090F0BCC053
:10A6C60091F0000E0001936F3C0E926FA0EC6DF0BE
:10A6D60090C0C4F091C0C5F0C4C097F0C5C098F052
:10A6E600000E00019A6F3C0E996F30EC71F097C026
:10A6F600CAF098C0CBF0CAC0BFF0CBC0C0F0000112
:10A70600BF1FC01FBF4BC02BBB51BF25C26FBC5163
:10A71600C021C36FBDC0BFF0BEC0C0F0060EC16F82
:10A72600D890C033BF33C12FFBD7BFC0C6F0C0C05F
:10A73600C7F0C6C0BFF0C7C0C0F0060ED890BF377E
:10A74600C037E82EFBD7BFC0CAF0C0C0CBF0CAC026
:10A75600BFF0CBC0C0F0BF1FC01FBF4BC02BBD5149
:10A76600BF25906FBE51C021916F000E936F060EEC
:10A77600926FA0EC6DF090C0C8F091C0C9F00001D6
:10A78600C95104E10A0EC85DD8A004D0000EC96FF5
:10A79600090EC86FC4C0B7F0C5C0B8F0020EB96FD5
:10A7A600020EBA6F9DEC70F0260E0001916F260E18
:10A7B600926F8EEC6EF0C2C0B7F0C3C0B8F0020E56
:10A7C6000001B96F020EBA6F9DEC70F0260E000103
:10A7D600916F260E926F8EEC6EF0C6C0B7F0C7C0B2
:10A7E600B8F0020E0001B96F020EBA6F9DEC70F060
:10A7F600370E0001916F290E926F8EEC6EF0C8C075
:10A80600B7F0C9C0B8F0010E0001B96F020EBA6FF9
:10A816009DEC70F0E70E0001916F240E926F8EECA6
:10A826006EF01200000E0001D16F000EDA6F070EF7
:10A83600DA6501D014D0DA51030D010EF326000EAD
:10A84600F4226B0EF324D96E010EF420DA6EDE507C
:10A85600DE10D8B402D0DA29D16FDA2BE8D7000E91
:10A86600DA6F13D0DA51030D6B0EF324D96E010E95
:10A87600F420DA6EDA51010DD20EF324E16E000EE9
:10A88600F420E26EDFCFE7FFDA2B4B50DA5DD8B06B
:10A8960039D0E8D7DA51030D6B0EF324D96E010EC9
:10A8A600F420DA6E0101DF380F0B0001CB6F080EC2
:10A8B600CB13DA51010DD20EF324D96E000EF4201B
:10A8C600DA6ECB3BDF50CB190F0BCB19DF6EDA51AB
:10A8D600030D6B0EF324D96E010EF420DA6E01011E
:10A8E600DF500F0B0001CB6FDA51010DD20EF324AE
:10A8F600D96E000EF420DA6EDF50CB19F00BCB19AF
:10A90600DF6EDA2BD151DA5DD8A0C4D7070EDA652F
:10A9160001D00CD0DA51010DD20EF324D96E000EFF
:10A92600F420DA6E000EDF6EDA2BF0D74C50CB6FC8
:10A93600CC6BCB3BCC3BF00ECC17CB510F0BCC13D7
:10A94600F00ECB17F00ECB25CD6FFF0ECC21CE6FC0
:10A95600CF6BCEBFCF07CF51D06F000ECD25B96FCD
:10A96600040ECE21BA6FDF0ECF21BB6F010ED021B0
:10A97600BC6FD20EBD6F000EBE6F080EBF6F81ECAE
:10A9860068F01200D2C195F0D3C196F0D4C197F009
:10A99600D5C198F0EB0E0001996F1E0E9A6FF90E55
:10A9A6009B6F000E9C6FDFEC70F00009D8A460D09E
:10A9B60083D068EC1FF087D0980E0001916F240EAB
:10A9C600926F8EEC6EF0040E0001916F280E926F5E
:10A9D6008EEC6EF02D0E0001916F290E926F8EECAB
:10A9E6006EF0FA0E0001916F260E926F8EEC6EF0ED
:10A9F600E80E0001916F240E926F8EEC6EF0870EBA
:10AA06000001916F270E926F8EEC6EF0D20E000150
:10AA1600916F1A0E926F8EEC6EF055D0F0EC34F00A
:10AA260052D07FEC2AF04FD06AEC4AF04CD0D2C11B
:10AA3600F0F0D3C1F1F0D4C1F2F0D5C1F3F0F3ECEC
:10AA460027F041D0D2C1F0F0D3C1F1F0D4C1F2F079
:10AA5600D5C1F3F025EC2FF036D0D2C1BEF0D3C16C
:10AA6600BFF0D4C1C0F0D5C1C1F02DEC42F02BD05F
:10AA76000001F951000AD8B49CD7010AD8B49CD772
:10AA8600030AD8B499D7010AD8B4C8D7070AD8B4E4
:10AA9600C5D7010AD8B4C5D7030AD8B4C5D7010AA1
:10AAA600D8B4C2D70F0AD8B4C2D7010AD8B4CAD705
:10AAB600030AD8B4D2D707D08E0E0001916F230EA9
:10AAC600926F8EEC6EF0000E00019B6F4B509EEC69
:10AAD60069F01200000E0101396F000E386F000E8A
:10AAE600376F000E366F000E00019B6F000E9C6FD5
:10AAF600000E996F050E9A6F000E9F6F3DD099C09C
:10AB0600D9FF9AC0DAFFDECFA1F0DDCFA2F0020EA8
:10AB16009927000E9A23A25104E1C90EA15DD8A07F
:10AB260029D0010138513911D8B409D03851000162
:10AB3600A15D010139510001A259D8B006D0A1C0CA
:10AB460038F1A2C039F19FC09BF00101365137118F
:10AB5600D8B40AD00001A1510101365D0001A2510D
:10AB660001013759D8B006D0A1C036F1A2C037F1DD
:10AB76009FC09CF000019F2B43509F5DD8A0BFD77C
:10AB86009BC090F0916B000E936F0C0E926FCAEC07
:10AB960066F000019051A06FA0510C0DF350000813
:10ABA6009B259E6FA051030D6B0EF324D96E010EEB
:10ABB600F420DA6E0101DF500F0B00019D6F9D51ED
:10ABC6000C0DF3509E25986F982901015F6F9CC06C
:10ABD60090F00001916B000E936F0C0E926FCAEC11
:10ABE60066F000019051A06FA0510C0DF3500008C3
:10ABF6009C259E6FA051030D6B0EF324D96E010E9A
:10AC0600F420DA6E0101DF500F0B00019D6F9D519C
:10AC16000C0DF3509E25986F982901015E6F120066
:10AC2600000E0101616F000E626F000E0001996F48
:10AC3600070E996501D029D09951040D000EF32411
:10AC4600D96E020EF420DA6EDE6ADE6ADE6ADD6A2C
:10AC56009951010D340EF324D96E020EF420DA6EEA
:10AC6600000EDF6E9951030D6B0EF324D96E010EA3
:10AC7600F420DA6E0101DF380F0BE806D8B402D0F3
:10AC8600010E616F0001992BD3D7000E986F67D024
:10AC96009851030D6B0EF324D96E010EF420DA6E73
:10ACA6000101DF380F0B0001976F98510C0DF3CFA0
:10ACB60094F0000E996F0B0E996501D04FD0995103
:10ACC60094C090F0916B9027000E9123D890903706
:10ACD6009137000E9025D96E060E9121DA6EDECFE1
:10ACE60095F0DDCF96F0965104E1C90E955DD8A09A
:10ACF60032D0FC0E906FFF0E916F9751926F936B4F
:10AD0600D89092379337D8909237933790519227AD
:10AD160091519323000E9225D96E020E9321DA6E7D
:10AD26009551DE269651DE22000EDE22DE22FF0E31
:10AD3600906FFF0E916F9751926F936B9051922780
:10AD460091519323340E9225D96E020E9321DA6E19
:10AD5600DF2A0101622B0001992BADD7982B4B50AE
:10AD6600985DD8B0120094D70001946F49B615D0FB
:10AD760035D049A80DD00ED049A802D0898077D009
:10AD8600899075D049A807D0898271D049A802D088
:10AD96008980FAD7899089926AD000019451000A75
:10ADA600D8B4E7D7010AD8B4E4D7030AD8B4E1D7B0
:10ADB600010AD8B4E1D7070AD8B4E4D7010AD8B44F
:10ADC600E5D7030AD8B4E2D7010AD8B4DFD70F0A09
:10ADD600DDD7000E01D0010E936F1CD000019451F7
:10ADE600000AD8B4F6D7010AD8B4F3D7030AD8B400
:10ADF600F0D7010AD8B4EFD7070AD8B4ECD7010ABE
:10AE0600D8B4E9D7030AD8B4E6D7010AD8B4E3D749
:10AE16000F0AE1D749A803D093A107D004D00001B7
:10AE26009351D8A402D08A8222D08A9220D0010ED1
:10AE3600CEEC5CF01200050ECEEC5CF01200040EB7
:10AE4600CEEC5CF01200030ECEEC5CF01200020EAB
:10AE5600CEEC5CF01200060ECEEC5CF01200040E96
:10AE6600CEEC5CF01200060ECEEC5CF01200000197
:10AE76009451000AD8B4DBD7010AD8B4DCD7030A48
:10AE8600D8B4DDD7010AD8B4DED7070AD8B4DFD7DD
:10AE9600010AD8B4E0D7030AD8B4E1D7010AD8B476
:10AEA600DED70F0AE0D70001E36F0001E3510C0D76
:10AEB600D890F336F436000EF324E56F050EF42031
:10AEC600E66F000EE46F020EE46501D01200E5C0E5
:10AED600D9FFE6C0DAFFDECFE7F0DDCFE8F0020EFD
:10AEE600E527000EE623E5C0D9FFE6C0DAFFDECF90
:10AEF600E9F0DDCFEAF0020EE527000EE623E5C015
:10AF0600D9FFE6C0DAFFDECFEBF0DDCFECF0020EC4
:10AF1600E527000EE623E5C0D9FFE6C0DAFFDECF5F
:10AF2600EDF0DDCFEEF0020EE527000EE6234C50E5
:10AF3600CB6FCC6BCB3BCC3BF00ECC17CB510F0B76
:10AF4600CC13F00ECB17F00ECB25CD6FFF0ECC2118
:10AF5600CE6FCF6BCEBFCF07CF51D06FE451D26F3C
:10AF6600D16BD1C0D3F0D2C0D4F0000ED4BFFF0E47
:10AF7600D56FD66FCD51D325D76FCE51D421D86F8B
:10AF8600CF51D521D96FD051D621DA6FE351D725CC
:10AF9600DB6F000ED821DC6F000ED921DD6F000EAD
:10AFA600DA21DE6F000EDB25DF6F090EDC21E06F94
:10AFB600DF0EDD21E16F010EDE21E26FDFC0B9F0A9
:10AFC600E0C0BAF0E1C0BBF0E2C0BCF0E70EBD6F76
:10AFD600000EBE6F080EBF6F81EC68F00001E42B17
:10AFE60072D726C190F027C191F0000E0001936F31
:10AFF6003C0E926FA0EC6DF090C0C0F091C0C1F015
:10B00600C0C097F0C1C098F0000E00019A6F3C0EC8
:10B01600996F30EC71F097C0BCF098C0BDF0BCC021
:10B02600B7F0BDC0B8F00001B71FB81FB74BB82BBB
:10B03600010126510001B725BA6F01012751000110
:10B04600B821BB6F33C0B7F034C0B8F0060EB96F85
:10B05600D890B833B733B92FFBD7B7C0BEF0B8C056
:10B06600BFF0C0C09DF0C1C09EF0050E9F6F000EE0
:10B07600A06F830EA16F010EA26F42EC5BF0830EF0
:10B086000001916F010E926F8EEC6EF0360E00018C
:10B09600916F270E926F8EEC6EF0BAC09DF0BBC01A
:10B0A6009EF0020E00019F6F000EA06F830EA16F2F
:10B0B600010EA26F42EC5BF0830E0001916F010E50
:10B0C600926F8EEC6EF0880E0001916F260E926FD5
:10B0D6008EEC6EF0BEC09DF0BFC09EF0020E000169
:10B0E6009F6F000EA06F830EA16F010EA26F42EC40
:10B0F6005BF0830E0001916F010E926F8EEC6EF085
:10B106006E0E0001916F260E926F8EEC6EF012009D
:10B116000001C26F0001C251D8A402D0000E0CD0AB
:10B12600C2C0C0F0010EC16FC02B02D0D890C1378B
:10B13600C02FFCD70001C105C36F000E9F6F040E20
:10B146009E6F070EA16FC20EA06F030EA26F0C0EAC
:10B15600A36FBCC0A4F0BDC0A5F0BEC0A6F0BFC022
:10B16600A7F0C2515AEC4BF0BEC0D9FFBFC0DAFF00
:10B17600DF500001C315C319D8A419D0000E9F6F64
:10B18600060E9E6F9A0EA16F940EA06F030EA26F0D
:10B196000C0EA36F060EBC25A46F000EBD21A56F75
:10B1A600BEC0A6F0BFC0A7F0C2515AEC4BF0BEC05D
:10B1B600D9FFBFC0DAFFDF500001C315C319D8A4F9
:10B1C60019D0000E9F6F080E9E6F5E0EA16F520E75
:10B1D600A06F030EA26F0C0EA36F0C0EBC25A46FFE
:10B1E600000EBD21A56FBEC0A6F0BFC0A7F0C2511C
:10B1F6005AEC4BF0BEC0D9FFBFC0DAFFDF500001EA
:10B20600C315C319D8A41200000E9F6F0A0E9E6FB5
:10B21600C30EA16F040EA06F030EA26F0C0EA36FD8
:10B22600120EBC25A46F000EBD21A56FBEC0A6F0F0
:10B23600BFC0A7F0C2515AEC4BF0120013EC56F007
:10B2460000C2B0F001C2B1F002C2B2F003C2B3F064
:10B25600E80E0001B46F030EB56F000EB66F000E58
:10B26600B76FBCEC60F0B0C0D1F0B1C0D2F004C290
:10B27600B0F005C2B1F006C2B2F007C2B3F0E80EF4
:10B286000001B46F030EB56F000EB66F000EB76FF8
:10B29600BCEC60F0B0C0D3F0B1C0D4F008C2B0F0DE
:10B2A60009C2B1F00AC2B2F00BC2B3F0E80E000157
:10B2B600B46F030EB56F000EB66F000EB76FBCEC21
:10B2C60060F0B0C0D5F0B1C0D6F00CC2B0F00DC27F
:10B2D600B1F00EC2B2F00FC2B3F0E80E0001B46FC7
:10B2E600030EB56F000EB66F000EB76FBCEC60F0C4
:10B2F600B0C0D7F0B1C0D8F04C500001CB6FCC6BCA
:10B30600CB3BCC3BF00ECC17CB510F0BCC13F00E36
:10B31600CB17F00ECB25CD6FFF0ECC21CE6FCF6BAA
:10B32600CEBFCF07CF51D06F000ECD25B96F0D0E12
:10B33600CE21BA6FDF0ECF21BB6F010ED021BC6FBD
:10B34600D10EBD6F000EBE6F080EBF6F81EC68F0A8
:10B35600120098C090F099C091F0000E0001936F12
:10B36600640E926FCAEC66F090C0A0F091C0A1F096
:10B376000001A1BF06D0A15108E1030EA05DD8B01F
:10B3860004D0FF0E9F6FFD0E64D0A1BF06D0A15161
:10B396000EE1330EA05DD8B00AD0A0C09AF0A1C0CD
:10B3A6009BF09A1F9B1F9A4B9B2B730E41D0A1BFFC
:10B3B60006D0A1511DE1590EA05DD8B019D0A0C08C
:10B3C60090F0A1C091F0000E936F020E926FCAEC3E
:10B3D60066F090C09CF091C09DF09CC09AF09DC014
:10B3E6009BF000019A1F9B1F9A4B9B2B5A0E20D055
:10B3F600A1BF06D0A15122E1E20EA05DD8B01ED0B9
:10B40600A0C090F0A1C091F0000E936F030E926F52
:10B41600CAEC66F090C09CF091C09DF09CC09AF07A
:10B426009DC09BF000019A1F9B1F9A4B9B2B4B0EB6
:10B436009A259E6F000E9B219F6F0FD0A1BF06D04D
:10B44600230EA05D010EA159D8B005D0FF0E9F6F47
:10B45600FE0E9E6F02D09E699F699EC098F09FC0A7
:10B4660099F012000001C56F050E4018D8A412000D
:10B47600C60E0001906F000E916F000E936F080EBE
:10B48600926F1CEC71F00001C697C691C693C695E3
:10B49600C68FC68D01019A979A990001C551D8A405
:10B4A60012D001019A87C3C09DF0C4C09EF0040E5D
:10B4B60000019F6F010EA06FC90EA16F000EA26F53
:10B4C60042EC5BF048D00001C505D8A40FD0C2C03D
:10B4D6009DF09E6B020E9F6F020EA06FC70EA16FAE
:10B4E600000EA26F42EC5BF05F0E12D0020EC51981
:10B4F600D8A410D0C2C09DF09E6B020E9F6F020EA4
:10B50600A06FC70EA16F000EA26F42EC5BF07E0E1D
:10B51600000109D0030EC519D8A407D02D0EC76F98
:10B526002D0EC86F2D0EC96F08D0040EC519D8A4EC
:10B5360004D0730EC76F640EC86FC3C09DF0C4C03D
:10B546009EF0030E9F6F020EA06FCA0EA16F000E33
:10B55600A26F42EC5BF0020E0001BA6F7B0EB96F70
:10B56600C60EBB6F000EBC6F080EBD6F4AEC6DF0C9
:10B57600120090C098F091C099F092C09AF093C0D2
:10B586009BF0000E00019C6F000E9D6F000E9E6FDB
:10B59600000E9F6F000EA06F000EA16F000EA26F2F
:10B5A600400EA36F09D0020E946FD890A333A23336
:10B5B600A133A033942FF9D7A051985DA151995981
:10B5C600A2519A59A3519B59D8B04AD0ECD7A05151
:10B5D6009C25946FA1519D21956FA2519E21966F36
:10B5E600A3519F21976F9451985D95519959965102
:10B5F6009A5997519B59D8A025D0A0519C25946F54
:10B60600A1519D21956FA2519E21966FA3519F2115
:10B61600976F9451985F9551995B96519A5B9751A4
:10B626009B5BD890A035946FA135956FA235966F28
:10B63600A335976F94519C2795519D2396519E2330
:10B6460097519F23D8909F339E339D339C33020E90
:10B65600946FD890A333A233A133A033942FF9D794
:10B66600A051A111A211A311D8A4B1D79CC090F0EA
:10B676009DC091F09EC092F09FC093F01200000E04
:10B686000001B66FA30EB06F000EB16F9DC0B4F08F
:10B696009EC0B5F04DD0B4C090F0B5C091F0000E8C
:10B6A600936F0A0E926FA0EC6DF090C0ACF091C053
:10B6B600ADF0ACC097F0ADC098F0000E00019A6FE7
:10B6C6000A0E996F30EC71F00001971F981F974B87
:10B6D600982BB4519725AE6FB5519821AF6FACC07A
:10B6E600B4F0ADC0B5F0B451B511D8A40BD0AE517D
:10B6F600AF11D8A407D0B651D8B404D0020EA01901
:10B70600D8A403D0AE51300F09D0A005D8A402D0DA
:10B71600200E04D0A051D8A402D0000EAB6FB0C04A
:10B72600D9FFB1C0DAFFABC0DFFFB04BB12BB62BF0
:10B73600B451B511D8A4AFD7B651D8B4ACD7A0512F
:10B74600D8B404D09F51B65DD8A0A5D7A1C0B2F099
:10B75600A2C0B3F010D0B007D8A0B107B0C0D9FFCF
:10B76600B1C0DAFFB2C0E1FFB3C0E2FFDFCFE7FF4F
:10B77600B24BB32BB607B651D8A4EDD7B2C0D9FF9A
:10B78600B3C0DAFF000EDF6E120091EC72F0000E0D
:10B796000001A86F070EA86501D00CD0010E9E6FA0
:10B7A600000EA06F000E9F6FA8514CEC5CF00001DC
:10B7B600A82BF0D7000EA86FA851010DEB0EF324AD
:10B7C600D96E020EF420DA6EFC0EDF6EA82BA8519D
:10B7D600010DEB0EF324D96E020EF420DA6E000E84
:10B7E600DF6EA82BA851010DEB0EF324D96E020EC5
:10B7F600F420DA6E000EDF6EA82BA851010DEB0EB9
:10B80600F324D96E020EF420DA6E000EDF6EA82B3A
:10B81600A851010DEB0EF324D96E020EF420DA6E58
:10B82600000EDF6EA82BA851010DEB0EF324D96E86
:10B83600020EF420DA6E000EDF6EA82BEB0E906F70
:10B84600020E916F000E936F060E926F24EC65F058
:10B8560090C0A6F091C0A7F00001A851010DEB0E13
:10B86600F324D96E020EF420DA6EA751DF6EA82BF0
:10B87600A851010DEB0EF324D96E020EF420DA6EF8
:10B88600A6C0DFFFA82B000E0101596F42EC6CF039
:10B8960012000001A16F0001A151080DF3CFA4F021
:10B8A600A4C0A5F09E51D8B40AD0A551010D890EA9
:10B8B600F324D96E030EF420DA6EFC0E09D0A551DE
:10B8C600010D890EF324D96E030EF420DA6E000EF4
:10B8D600DF6EA52BA551010D890EF324D96E030E3B
:10B8E600F420DA6E000EDF6EA52BA551010D890E30
:10B8F600F324D96E030EF420DA6E000EDF6EA52B4C
:10B90600A551010D890EF324D96E030EF420DA6ECB
:10B91600000EDF6EA52BA551010D890EF324D96EFD
:10B92600030EF420DA6E9FC0DFFFA52BA551010D93
:10B93600890EF324D96E030EF420DA6EA051DF6E61
:10B94600A52BA451010D890EF324906F030EF4204C
:10B95600916F000E936F060E926F24EC65F090C007
:10B96600A2F091C0A3F00001A551010D890EF324A8
:10B97600D96E030EF420DA6EA351DF6EA52BA55106
:10B98600010D890EF324D96E030EF420DA6EA2C0DF
:10B99600DFFFA52B12000001926F000E42EC6EF045
:10B9A600000E6EEC6CF0000E76EC6DF053D0020ECD
:10B9B6000101636F000E216F000E206F000E1F6FD6
:10B9C600000E1E6F1200100E0101636F000E216F34
:10B9D600000E206F000E1F6F010E1E6F1200040E68
:10B9E6000101636F000E216F010E206F000E1F6FA5
:10B9F600000E1E6F020E42EC6EF012000C0E0101DC
:10BA0600636F0F0E216FC00E206F000E1F6F3F0E6B
:10BA16001E6F020E6EEC6CF01200100E0101636FC9
:10BA2600000E216F010E206F000E1F6F010E1E6F9C
:10BA3600010E76EC6DF01200100E0101636F0F0E11
:10BA4600216F2069000E1F6F000E1E6F010E42EC63
:10BA56006EF0120000019251000AD8B4A8D7010A6C
:10BA6600D8B4B1D7030AD8B4BAD7010AD8B4B7D76D
:10BA7600070AD8B4C3D7010AD8B4CFD7030ADCD78C
:10BA8600000E0001F16F070EF16501D066D0F1518D
:10BA96000D0D040EF326000EF4224C0EF324D96E7F
:10BAA600020EF420DA6EDECFEEF0DDCFEFF0EE51CF
:10BAB600EF11D8B436D0000EF06F0B0EF06501D042
:10BAC60030D0F0C0EBF0010EEC6F000EED6FEB2BFB
:10BAD60003D0D890EC37ED37EB2FFBD70001EE51B2
:10BAE600EC17EF51ED17EC51ED11D8B417D0F0C0AB
:10BAF600E4F0000EE56FF1510D0D4C0EF324D96EF6
:10BB0600020EF420DA6E0201000EDFB0010E000113
:10BB1600E66F000EE76FF15126EC64F00001F02BA2
:10BB2600CCD7010E9E6F000EA06F000E9F6FF151D5
:10BB36004CEC5CF00001F1510D0D040EF326000EE5
:10BB4600F4224C0EF324D96E020EF420DA6E000EA7
:10BB5600DE6E000EDD6EF12B96D7000E0101646FCE
:10BB6600000E4F6F000E4E6F1200000E0001C66FE2
:10BB76003DC0BEF03EC0BFF0BE1FBF1FBE4BBF2BB9
:10BB86003B50BE25906F3C50BF21916F000E936FC6
:10BB96000A0E926FA0EC6DF00001901F911F904B62
:10BBA600912B3B509025C26F3C509121C36F9AEC6C
:10BBB6006CF090C0C4F091C0C5F03D500001C45D6A
:10BBC6003E50C559D8A03CD03DC0BEF03EC0BFF0E7
:10BBD600BE1FBF1FBE4BBF2BC451BE27C551BF23BF
:10BBE600BEC0A4F0BFC0A5F0A66BA76B640EA86F7D
:10BBF600000EA96F000EAA6F000EAB6FC6EC6CF0BC
:10BC0600A4C0B0F0A5C0B1F0A6C0B2F0A7C0B3F012
:10BC16003DC0C0F03EC0C1F00001C01FC11FC04BF7
:10BC2600C12BC251C027C351C123C0C0B4F0C1C08B
:10BC3600B5F0B66BB76BBCEC60F00001B051C66FE7
:10BC4600640EC66502D0640EC66FC65112000001AE
:10BC5600BF6F710E0001916F270E926F8EEC6EF022
:10BC6600010E0001BF25B86FB96B000EB923010E96
:10BC7600BA6FADEC6FF0050E0001BB19D8A407D062
:10BC8600E40E916F270E926F8EEC6EF019D03F0E78
:10BC96000001916F290E926F8EEC6EF0010E00017D
:10BCA600BB25B86FB96B000EB923010EBA6FADECA8
:10BCB6006FF0E80E0001916F270E926F8EEC6EF01A
:10BCC6000001BD290AE1BE29D8A407D0B40E916FA0
:10BCD600280E926F8EEC6EF01200FD0E0001BD195B
:10BCE6000AE1BE29D8A407D0BC0E916F270E926F29
:10BCF6008EEC6EF01200BDC0B8F0BEC0B9F0010EF9
:10BD06000001BA6FADEC6FF00001BC51D8B407D09A
:10BD1600CC0E916F240E926F8EEC6EF012007B0E9D
:10BD26000001916F260E926F8EEC6EF01200000EDF
:10BD36000001E06F070EE06501D033D04B50E05DA7
:10BD4600D8B01DD0E0510D0D020EF326000EF422E0
:10BD56004C0EF324D96E020EF420DA6EE051030D78
:10BD6600010EF326000EF4226B0EF324E16E010E93
:10BD7600F420E26EDECFE6FFDDCFE5FF10D0E05126
:10BD8600030D010EF326000EF4226B0EF324D96E7A
:10BD9600010EF420DA6E000EDE6E000EDD6EE02B74
:10BDA600C9D76B0EDD6F010EDE6F0C0EDF6F000E56
:10BDB600E06F170EE06501D011D0DFC09DF09E6BDD
:10BDC600DDC0D9FFDEC0DAFFDF509F6F17EC6FF0E2
:10BDD6000001DF2BDD4BDE2BE02BEBD788EC47F0A9
:10BDE60001016C516D11D8B409D04290BE0E00010C
:10BDF600916F230E926F8EEC6EF01200ED0E000125
:10BE0600916F1F0E926F8EEC6EF01200D30E000132
:10BE1600D16F000ED26FD1C0D9FFD2C0DAFF39C0C0
:10BE2600DEFF3AC0DDFF20EE02F0D151D926D25115
:10BE3600DA2237C0DEFF38C0DDFF20EE04F0D15134
:10BE4600D926D251DA2244C0DFFF20EE05F0D151C7
:10BE5600D926D251DA2267C1DFFF20EE06F0D15192
:10BE6600D926D251DA22DF50F00B0209DF6E20EE1E
:10BE760006F0D151D926D251DA22DF500F0B200914
:10BE8600DF6E20EE07F0D151D926D251DA220E0EFE
:10BE9600DF6E4C50CB6FCC6BCB3BCC3BF00ECC1754
:10BEA600CB510F0BCC13F00ECB17F00ECB25CD6F6D
:10BEB600FF0ECC21CE6FCF6BCEBFCF07CF51D06F49
:10BEC600000ECD25B96F0C0ECE21BA6FDF0ECF2135
:10BED600BB6F010ED021BC6FD30EBD6F000EBE6FBF
:10BEE600080EBF6F81EC68F012000001D16FD1C05F
:10BEF600D3F00001D151010D000EF324D96E010ECD
:10BF0600F420DA6EDF50D46FD151010D440EF324C4
:10BF1600D96E020EF420DA6EDF50D56F000ED26FA6
:10BF2600040ED26501D022D0D151050D000ECB6F83
:10BF3600030ECC6FF350CB27F450CC23D251010D16
:10BF4600F350CB25D96EF450CC21DA6ED251010DC7
:10BF5600030EF326000EF422D30EF324E16E000E38
:10BF6600F420E26EDFCFE7FFD22BDAD74C50CB6F4F
:10BF7600CC6BCB3BCC3BF00ECC17CB510F0BCC1381
:10BF8600F00ECB17F00ECB25CD6FFF0ECC21CE6F6A
:10BF9600CF6BCEBFCF07CF51D06F000ECD25B96F77
:10BFA6000E0ECE21BA6FDF0ECF21BB6F010ED02150
:10BFB600BC6FD30EBD6F000EBE6F080EBF6F81EC57
:10BFC60068F012002B502D5C2C502E58D8A004D0AF
:10BFD6002B5000082D2404D02B5000082D24100FC0
:10BFE6000001966F01015851D8B433D0040E0001F8
:10BFF60096612BD0000E0101586F90C0D9FF91C0F9
:10C00600DAFF010EDF6E0EC194F00FC195F000014C
:10C01600941F951F944B952B0201CE510001942736
:10C026000201CF510001952301011051000194270F
:10C03600010111510001952392C0D9FF93C0DAFF87
:10C0460094C0DEFF95C0DDFF21D00101104B112BFE
:10C056001DD090C0D9FF91C0DAFF000EDF6E92C0EE
:10C06600D9FF93C0DAFF000EDE6E000EDD6E080EFD
:10C07600000196650BD0010E0101586F000E116F7D
:10C08600000E106FCEC20EF1CFC20FF10101585152
:10C09600D8A402D0010E1200000E1200000E0001FC
:10C0A600A36F9BC095F09CC096F09DC097F09EC074
:10C0B60098F0A40E996F000E9A6F8DEC71F000093E
:10C0C600D8B44DD00001A451A511D8B440D0A55183
:10C0D6003EE1090EA45DD8B03AD0A4059FC0D9FFB1
:10C0E600A0C0DAFFDF6E9BC095F09CC096F09DC0A5
:10C0F60097F09EC098F0A40E996F000E9A6F8DEC83
:10C1060071F00009D8B41BD00001A451A511D8B410
:10C116000FD0A5510DE1060EA45DD8B009D0A40537
:10C12600A1C0D9FFA2C0DAFFDF6E010EA36F1ED039
:10C136006B0E916F210E926F8EEC6EF017D0EC0E97
:10C146000001916F230E926F8EEC6EF00FD0110EE0
:10C156000001916F230E926F8EEC6EF007D0EC0EFD
:10C166000001916F230E926F8EEC6EF00001A351C9
:10C176001200000E0001B96FB7AF0AD0B71FB61F85
:10C18600B51FB46D000EB523B623B723010EB96FE4
:10C19600B3AF0AD0B31FB21FB11FB06D000EB123EB
:10C1A600B223B323010EB91B000EBA6F000EBB6F8C
:10C1B600000EBC6F000EBD6FB451B511B611B711AC
:10C1C600D8B42AD0010EB86F06D0D890B437B53798
:10C1D600B637B737B82BB7AFF8D7D890BA37BB371B
:10C1E600BC37BD37B451B05DB551B159B651B2592E
:10C1F600B751B359D8A009D0B451B05FB551B15BAE
:10C20600B651B25BB751B35BBA81D890B733B63388
:10C21600B533B433B82FE1D7B951D8B408D0BD1F60
:10C22600BC1FBB1FBA6D000EBB23BC23BD23BAC007
:10C23600B0F0BBC0B1F0BCC0B2F0BDC0B3F01200EC
:10C246000001E751D8A45FD0DC0E916F270E926FE4
:10C256008EEC6EF0E4C091F0E5C092F08EEC6EF0DC
:10C26600BB0E0001916F240E926F8EEC6EF00001F2
:10C27600E605D8A40BD0E8C0DEF0E9C0DFF0B30EC7
:10C28600E06F280EE16F80EC6BF010D0E80E000135
:10C29600916F240E926F8EEC6EF0E8C0B8F0E9C094
:10C2A600B9F0010E0001BA6FADEC6FF0EB0E0001B4
:10C2B600916F280E926F8EEC6EF00001E605D8A401
:10C2C6000BD0EAC0DEF0EBC0DFF0B30EE06F280E55
:10C2D600E16F80EC6BF010D0E80E0001916F240E38
:10C2E600926F8EEC6EF0EAC0B8F0EBC0B9F0010EBA
:10C2F6000001BA6FADEC6FF0D20E0001916F1A0E0D
:10C30600926F8EEC6EF00001E7511200200E0101D3
:10C31600836F000E0001A26F55D096C0D9FF97C05B
:10C32600DAFFDECFA3F0DECFA4F0DECFA5F0DECFBE
:10C33600A6F0040E9627000E9723000EA3159A6FFB
:10C34600000EA4159B6F000EA5159C6FFF0EA6157B
:10C356009D6F190E05D0D8909D339C339B339A332D
:10C36600E82EF9D79A519E6FA5C09FF0A4C0A0F001
:10C37600A3C0A1F0840E906F010E916F9E5113EC35
:10C386006CF0860E0001906F010E916F9F5113ECB9
:10C396006CF0880E0001906F010E916FA05113ECA6
:10C3A6006CF08A0E0001906F010E916FA15113EC93
:10C3B6006CF0830E0001916F010E926F8EEC6EF0A1
:10C3C6000001A22BA2519A6F9B6B98519A5D9951CD
:10C3D6009B59D8B01200A1D733C008F034C009F079
:10C3E600D89009320832D89009320832D8900932EA
:10C3F600083208C00EF009C00FF0010122510E18D4
:10C4060004E123510F18D8B412000EC001F00FC07A
:10C4160002F063C103F0046ACAEC6DF001C00BF0D0
:10C4260002C00CF0010163510B02F35000080E2408
:10C436000D6E0DC008F0010E096E000E0A6E082A78
:10C4460003D0D89009360A36082EFBD701011E51B3
:10C4560009161F510A1609500A10D8B402D08B8249
:10C4660001D08B920DC008F0010E096E000E0A6E07
:10C47600082A03D0D89009360A36082EFBD70101C0
:10C486002051091621510A1609500A10D8B402D0B3
:10C496008B8001D08B900EC022F10FC023F11200C9
:10C4A60000019A6F00019A51800A7F0FD8B00ED012
:10C4B6009AC096F0976B96BF9707961F971F964B55
:10C4C600972B96C098F097C099F005D09A51986F1F
:10C4D600996B98BF990798C09BF09AAF21D09B5152
:10C4E600800A700FD8A007D0CD0E916F280E926FDC
:10C4F6008EEC6EF0120000019B51800A760FD8A0D8
:10C5060007D0BE0E916F280E926F8EEC6EF0120061
:10C51600E50E0001916F240E926F8EEC6EF0120004
:10C5260000019B51800A700FD8A007D0C80E916FEA
:10C53600280E926F8EEC6EF0120000019B51800A5D
:10C54600760FD8A007D0B90E916F280E926F8EEC99
:10C556006EF01200E50E0001916F240E926F8EECC4
:10C566006EF0120092C09DF093C09EF09DC0D9FF60
:10C576009EC0DAFF300EDF6E00019D4B9E2B9DC0E4
:10C58600D9FF9EC0DAFF780EDF6E9D4B9E2B90C0C2
:10C5960094F091C095F00C0E966FD8909533943325
:10C5A600962FFBD794510F0B976F91510F0B986FE6
:10C5B60090C094F091C095F0040E966FD890953384
:10C5C6009433962FFBD794510F0B996F90510F0B05
:10C5D6009A6F000E9C6F030E9C6501D01BD09C5178
:10C5E600010D970EF324D96E000EF420DA6EDF509B
:10C5F6009B6F090E9B6503D09B51570F02D09B5131
:10C60600300F9DC0D9FF9EC0DAFFDF6E9D4B9E2B7B
:10C616009C2BE1D79DC0D9FF9EC0DAFF000EDF6ECE
:10C6260012000CEE00F012EE20F0EE6AE550E1503A
:10C63600FCE1E250FAE10BEE00F011EE00F0EE6ADA
:10C64600E550E150FCE1E250FAE10AEE00F0C00EDE
:10C65600EE6AE806FDE109EE00F0C00EEE6AE806B5
:10C66600FDE108EE00F0600EEE6AE806FDE107EE79
:10C6760000F0C00EEE6AE806FDE106EE00F0C00E20
:10C68600EE6AE806FDE105EE00F0C00EEE6AE80689
:10C69600FDE104EE00F0E10EEE6AE806FDE103EED0
:10C6A60000F0E90EEE6AE806FDE102EE00F0F30E98
:10C6B600EE6AE806FDE101EE00F0AA0EEE6AE80673
:10C6C600FDE100EE27F0250EEE6AE806FDE14D904D
:10C6D6004D92000EF86E0001F4EF3CF0DB0E000107
:10C6E600916F010E926F2EEC69F00009D8B412001A
:10C6F6007F0E0101DB19D8B404D0080EDB19D8A4CB
:10C706000CD014511511D8B41200DB5108EC71F09D
:10C7160001011407D8A0150712000D0EDB19D8B4B5
:10C7260004D00A0EDB19D8A41DD00D0E08EC71F04A
:10C736000A0E08EC71F0000E01011425D96E0B0EDD
:10C746001521DA6E000EDF6E000ED66F0B0ED76F58
:10C756007AEC49F0000E0101156F000E146F86EC9D
:10C7660070F012000101DB5108EC71F0000E0101BE
:10C776001425D96E0B0E1521DA6EDBC1DFFF144BC3
:10C78600152B1405010E1559D8A01200000E156FB1
:10C79600000E146F120090C0D9FF91C0DAFFDF506F
:10C7A6000001966F000E986F9969000E9B6F070E39
:10C7B6009B6501D037D09B510D0D4C0EF324D96EDD
:10C7C600020EF420DA6E0201DFB011D000019B5197
:10C7D600030D010EF326000EF4226B0EF324D96E20
:10C7E600010EF420DA6EDE50DE10D8B419D0000146
:10C7F6009B51030D6B0EF324D96E010EF420DA6EF5
:10C80600DF509A6F9A51965DD8B00AD099519A5DC9
:10C81600D8B006D09AC099F09BC097F0010E986FD9
:10C826009B2BC5D79851D8B40CD090C0D9FF91C0D6
:10C83600DAFF99C0DFFF92C0D9FF93C0DAFF97C035
:10C84600DFFF985112000001EA6F4AA41200E4C00B
:10C85600BEF00001EA5146EC68F00001EA510C0D09
:10C86600E451F326000EF422D890F336F436000E87
:10C87600F324D96E050EF420DA6EDECFE8F0DDCFB4
:10C88600E9F0E8C0DEF0E9C0DFF00C0EE06F260E3E
:10C89600E16F80EC6BF00001E551D8B407D03C0E97
:10C8A600916F290E926F8EEC6EF007D0150E000177
:10C8B600916F290E926F8EEC6EF00001E651D8B49E
:10C8C6000AD0E751D8B40ED0710E916F250E926F33
:10C8D6008EEC6EF007D0C90E0001916F260E926F96
:10C8E6008EEC6EF0D20E0001916F1A0E926F8EECE6
:10C8F6006EF0120000019E6F000E0001A06F9851AD
:10C90600D8B44BD0FF0E9825906F916BFF0E9123F4
:10C91600000E936F0C0E926FCAEC66F000019051F8
:10C926009F6F9F510C0DF350000898259D6F9D0534
:10C936009BC0D9FF9CC0DAFFDF6E000EA16F27D027
:10C94600A151030D6B0EF324D96E010EF420DA6E9D
:10C956000101DF380F0B00019E19D8A417D0A15191
:10C96600030D6B0EF324D96E010EF420DA6E01016D
:10C97600DF500F0B00019F19D8A408D099C0D9FF2A
:10C986009AC0DAFFA1C0DFFF010EA06FA12B080E2F
:10C99600A16103D0A051D8B4D3D7A0511200000191
:10C9A600966F8B94000E0001926F010E916F1CEC36
:10C9B60072F03D0E0001926F6E0E916F1CEC72F0DC
:10C9C60096C099F0000136D09551D8B41ED0993949
:10C9D600E842F80BF80F976F9951080DF3CF98F0CE
:10C9E60097C09AF00DD09A51010D890EF324D96E95
:10C9F600030EF420DA6EDF5060EC72F000019A2B21
:10CA060098519A5DD8B015D0EED7000E9A6F070EE2
:10CA16009A6501D00ED09A51010DEB0EF324D96E12
:10CA2600020EF420DA6EDF5060EC72F000019A2BF1
:10CA3600EED799079951D8A4C7D78B840301CA2B7F
:10CA46001200000E00019D6F100E9C6F000E9B6F72
:10CA5600000E9A6F34D09CC094F09DC095F0070EDE
:10CA6600966F953595339433962FFBD79A5190252B
:10CA7600D96E9B519121DA6EDF50976F9751941BB7
:10CA8600000E951B9451986F996BD8909835F66E59
:10CA96009935F76EF70EF626110EF7220900F5CF37
:10CAA60094F00900F5CF95F09C51976F966B9451D1
:10CAB60096199C6F955197199D6F9A4B9B2B925186
:10CAC6009A5D9B51800A946F9351800A9459D8A01D
:10CAD600C2D7D8909C35906F9D35916F120000019A
:10CAE600E26F0001E2AF07D04C0E916F290E926FF4
:10CAF6008EEC6EF007D04A0E0001916F290E926FF0
:10CB06008EEC6EF00001E251800A7F0FD8B00ED095
:10CB1600E2C0DEF0DF6BDEBFDF07DE1FDF1FDE4BAE
:10CB2600DF2BDEC0E0F0DFC0E1F005D0E251E06FC0
:10CB3600E16BE0BFE107E0C0BEF0E1C0BFF0000E70
:10CB4600C16F0A0EC06F010EC26F010EC36F830E56
:10CB5600C46F010EC56F86EC46F0830E0001916F1F
:10CB6600010E926F8EEC6EF0120001016451D8A492
:10CB760010D049A01200010E646F020E00019B6FD7
:10CB86004B509EEC69F0000E01014F6F400E4E6F48
:10CB960012006405D8A410D0EFEC40F0010E00019D
:10CBA6009B6F4B509EEC69F0020E0101646F070EFD
:10CBB6004F6F800E4E6F1200030E6419D8A403D077
:10CBC60043EC5DF01200000E0001F26F070EF265F5
:10CBD60001D00CD0010E9E6F000EA06F000E9F6F4D
:10CBE600F2514CEC5CF00001F22BF0D7000E010183
:10CBF600646F1200000E0001966F000E956F000E16
:10CC0600906F050E916F000E926F21D090C0D9FFE4
:10CC160091C0DAFFDECF93F0DDCF94F0020E9027BD
:10CC2600000E9123945104E1C90E935DD8A00ED055
:10CC360095519611D8B406D09551935D9651945955
:10CC4600D8B004D093C095F094C096F0922B435080
:10CC5600925DD8A0DBD701015D2B090E5D6502D080
:10CC6600000E5D6F5D51020D200EF324D96E020E8B
:10CC7600F420DA6E95C0DEFF96C0DDFF12000001DB
:10CC8600CE6FCEC0D0F04C040001D16F42C0D2F0BE
:10CC9600000ED36F4BC0D4F0000ECF6F1ED0CF5115
:10CCA6000D0D0B0EF326000EF4224C0EF324D96E56
:10CCB600020EF420DA6EDE50DE10D8B40DD0CFC0EE
:10CCC600CCF0010ECD6FCC2B02D0D890CD37CC2F27
:10CCD600FCD70001CD51D313CF2B4B50CF5DD8A03D
:10CCE600DED742B2D083010EB96F000EBA6FDD0EE9
:10CCF600BB6F010EBC6FD00EBD6F000EBE6F050E72
:10CD0600BF6F81EC68F012004C0E0001916F180E97
:10CD1600926F8EEC6EF0F70E0001916F130E926F0C
:10CD26008EEC6EF0D50E0001916F1A0E926F8EEC9E
:10CD36006EF0E90E0001916F160E926F8EEC6EF09A
:10CD46000101FFB307D0F40E0001916F1C0E926F24
:10CD56008EEC6EF0870E0001916F1D0E926F8EECB9
:10CD66006EF04A0E0001916F200E926F8EEC6EF0FF
:10CD7600CC0E0001916F200E926F8EEC6EF08B0E32
:10CD86000001916F1F0E926F8EEC6EF01200000E76
:10CD96000001956F93AF06D0926D931FD8B0932B79
:10CDA600010E956F91AF06D0906D911FD8B0912B63
:10CDB600010E951B000E976F000E966F9251931100
:10CDC600D8B41CD0010E946F04D0D8909237933704
:10CDD600942B93AFFAD7D890963797379251905DA8
:10CDE60093519159D8A005D09251905F9351915B80
:10CDF6009681D89093339233942FEDD79551D8B42A
:10CE060004D0966D971FD8B0972B96C090F097C018
:10CE160091F01200000120EE01F09051D9269151B7
:10CE2600DA22DFA007D001015651D8A403D09973A6
:10CE3600010E0CD0000120EE05F09051D92691513B
:10CE4600DA22040EDF6403D0000E0101566F0001E2
:10CE560020EE01F09051D9269151DA22DFA20DD0B1
:10CE660001015751D8A409D0552B040E556502D09F
:10CE7600000E556F010E576F1200000120EE03F0F1
:10CE86009051D9269151DA22040EDF641200000E69
:10CE96000101576F12000001BE6F000E00019F6F67
:10CEA600100E9E6FED0EA16F720EA06F030EA26F95
:10CEB600030EA36F010EBC25A46F000EBD21A56F46
:10CEC600BF0EA66F000EA76FBE515AEC4BF0000EB8
:10CED60000019F6F120E9E6F700EA16F240EA06F41
:10CEE600030EA26F030EA36F310EBC25A46F000EB6
:10CEF600BD21A56FC00EA66F000EA76FBE515AECDE
:10CF06004BF00001BF51C015BCC0D9FFBDC0DAFF50
:10CF1600DF6E1200AECF03F032500BE13F0E315CF4
:10CF2600D8B007D0010E3124016E000E3220026EF9
:10CF360004D0000E026E000E016E2F50011804E19F
:10CF460030500218D8B41CD00350D8B419D0000EF3
:10CF56003124D96E040E3220DA6E03C0DFFF325060
:10CF66000BE13F0E315CD8B007D0010E3124316E93
:10CF7600000E3220326E04D0000E326E000E316E7C
:10CF8600ABA203D0AB98AB92AB88ABA41200AB9428
:10CF96001200000E0001936F23D0D89001011C35BA
:10CFA600D96E1D35DA6E000ED926050EDA22DECFD1
:10CFB60094F0DDCF95F01C4B1D2B000E0001926FF7
:10CFC600F00E945DFF0E9559D8B008D0955104E146
:10CFD600C90E945DD8A002D0010E926F92C093F054
:10CFE600435001011C5D000E1D59D8B004D000014C
:10CFF6009351D8B4D2D790C0D9FF91C0DAFF94C06C
:10D00600DEFF95C0DDFF0001935112003BC0D1F059
:10D016003CC0D2F03DC0D3F03EC0D4F03AC1D5F00A
:10D026003BC1D6F035C0D7F036C0D8F04C50000121
:10D03600CB6FCC6BCB3BCC3BF00ECC17CB510F0B55
:10D04600CC13F00ECB17F00ECB25CD6FFF0ECC21F7
:10D05600CE6FCF6BCEBFCF07CF51D06F000ECD2591
:10D06600B96F030ECE21BA6FDF0ECF21BB6F010E53
:10D07600D021BC6FD10EBD6F000EBE6F080EBF6F04
:10D0860081EC68F012000001C36F0001C351030D6B
:10D096006B0EF324D96E010EF420DA6E0101DF382F
:10D0A6000F0B0001C06FC351030D6B0EF324D96E35
:10D0B600010EF420DA6E0101DF500F0B0001C16F83
:10D0C600C1510C0DF350BE25BF6FBF29C26FC0C042
:10D0D600B8F0B96B010EBA6FADEC6FF04E0E0001F1
:10D0E600916F290E926F8EEC6EF0260E0001BB6FCB
:10D0F600260EBC6FC251D4EC6EF01200BBC0C9F054
:10D10600BCC0CAF0B9C0C7F0BAC0C8F0C9C0C0F048
:10D11600CAC0C1F0050E0001C26FD890C133C0333A
:10D12600C22FFBD7C051C36FC9C0C0F0030EC017D2
:10D13600C9C0C1F01C0EC117D890C137D890C137ED
:10D14600D890C135C0110809C46FC851C56FC7C092
:10D15600C6F0C4C0ABF0C5C0ACF0C6C0ADF0BDC033
:10D16600AEF0BEC0AFF0BFC0B0F0C35188EC48F01F
:10D176001200200E0101836F000E00019E6F28D061
:10D1860096C0D9FF97C0DAFFDECF9FF0DDCFA0F0C3
:10D19600020E9627000E9723A0519C6F9FC09DF00C
:10D1A600840E906F010E916F9C5113EC6CF0860EFD
:10D1B6000001906F010E916F9D5113EC6CF0830E80
:10D1C6000001916F010E926F8EEC6EF000019E2BA6
:10D1D6009E519A6F9B6B98519A5D99519B59D8B005
:10D1E6001200CED7AEC095F0AFC096F0B0C097F0A3
:10D1F600B1C098F0BC0E0001996F260E9A6FB20E60
:10D206009B6F000E9C6FDFEC70F00009D8A40FD066
:10D216001AD0A50E0001916F220E926F8EEC6EF061
:10D2260012008CEC72F0120085EC72F01200000114
:10D23600B251000AD8B4EDD7010AD8B4F2D7030A1E
:10D24600D8A41200F1D78E0E0001916F230E926FB3
:10D256008EEC6EF01200000E0001936F2F50311805
:10D266000FE130503218D8A40BD001015B51D8B46D
:10D2760027D0110E08EC71F0000E01015B6F20D073
:10D28600000E2F24D96E040E3020DA6E91C0E1FF15
:10D2960092C0E2FFDFCFE7FF30500BE13F0E2F5C7D
:10D2A600D8B007D0010E2F242F6E000E3020306E1E
:10D2B60004D0000E306E000E2F6E010E0001936F2B
:10D2C600000193511200320E0001DE25B06F000EF0
:10D2D600DF21B16F000EE021B26F000EE121B36FC6
:10D2E600640EB46F000EB56F000EB66F000EB76F0A
:10D2F600BCEC60F0B0C0BEF0B1C0BFF0000E0001E3
:10D30600C16F640EC06F020EC26F020EC36F830E32
:10D31600C46F010EC56F86EC46F0830E0001916F57
:10D32600010E926F8EEC6EF0E2C091F0E3C092F0C7
:10D336008EEC6EF0120000019C6F55EC70F000014F
:10D346009B05D8A402D0010E06D0020E00019B193F
:10D35600D8A403D0000E0101596F59C195F0000100
:10D366009C51D2EC64F0030E0001986FE80E976FA3
:10D376003BEC70F0000E00019D6F040E9D6501D020
:10D386000FD08B94000E60EC72F08B84030E0001BC
:10D39600986FE80E976F3BEC70F000019D2BEDD770
:10D3A6000301C92B12000001985106E1C80E975DD2
:10D3B600D8B002D0000E2CD097513D5C98513E5803
:10D3C600D8A002D0010E24D03B50975D3C5098590E
:10D3D600D8B01DD03DC099F03EC09AF0991F9A1F53
:10D3E600994B9A2B97519925906F98519A21916F45
:10D3F6001AC192F01BC193F0A0EC6DF000019051A0
:10D40600020F9B6F0E0E9B6504D00E0E01D00F0E01
:10D416009B6F9B51120013EC56F000C2B0F001C294
:10D42600B1F002C2B2F003C2B3F0E80E0001B46F6D
:10D43600030EB56F000EB66F000EB76FBCEC60F052
:10D44600B0C0C2F0B1C0C3F0C2C0C4F00001C35145
:10D45600C56F45C0C6F0000EC76F000EC86F000E40
:10D46600C96F000ECA6F000ECB6F030EBA6F570E50
:10D47600B96FC40EBB6F000EBC6F080EBD6F4AECD1
:10D486006DF012000001BE6F000E00019F6F0C0EC2
:10D496009E6FEF0EA16FCC0EA06F030EA26F030E50
:10D4A600A36F010EBC25A46F000EBD21A56FBCC0E5
:10D4B600A6F0BDC0A7F0BE515AEC4BF0000E00011D
:10D4C6009F6F0E0E9E6F720EA16F9A0EA06F030EC7
:10D4D600A26F030EA36F310EBC25A46F000EBD21F3
:10D4E600A56FBCC0A6F0BDC0A7F0BE515AEC4BF06C
:10D4F600120077EC44F001014C514D11D8A41200F2
:10D506006AB10ED04B50D8B424D0692B4B50695D0C
:10D51600D8A002D0000E696F695178EC5FF019D07F
:10D5260065C1EFF065A106D03E513F11D8B402D0D7
:10D536000001EF91010165A306D040514111D8B415
:10D5460002D00001EF9342C0CBF00001EF5142EC54
:10D5560066F001016A2B000E4D6F200E4C6F120013
:10D566000001E151E211D8B406D0E1C0E7F0E2C013
:10D57600E8F0010E05D0E3C0E7F0E4C0E8F0000EE5
:10D58600E56FE7A50ED0000EE66F07D0E5C0CBF03D
:10D59600E65137EC31F00001E62B4B50E65DD8A0A2
:10D5A600F5D7E7B9CEEC4EF00001E7A304D009ECBD
:10D5B60068F015EC54F00001E7B709EC5FF00001E4
:10D5C600E7AD120021EC59F01200AA0E0001916F8E
:10D5D600190E926F8EEC6EF08B928B90400E0101BD
:10D5E600082500019B6F000E0101092100019C6FB7
:10D5F600000E01010A2100019D6F000E01010B21A1
:10D6060000019E6F9B510101085D00019C510101C3
:10D61600095900019D5101010A590B51800A000167
:10D626009A6F9E51800A9A59D8A0ECD78CEC03F0D9
:10D636001200AF0E0001916F280E926F8EEC6EF005
:10D64600420E0001916F1E0E926F8EEC6EF08F0EE1
:10D656000001916F210E926F8EEC6EF0040E0001A8
:10D66600916F280E926F8EEC6EF0310E0001916F65
:10D676001E0E926F8EEC6EF0080E0001916F1E0E5C
:10D68600926F8EEC6EF0420E0001916F1E0E926F3D
:10D696008EEC6EF01200050E0001DE25906F000E76
:10D6A600DF21916F000E936F0A0E926FA0EC6DF062
:10D6B60090C0E2F091C0E3F0E2C0BEF0E3C0BFF07C
:10D6C600030E0001C16FE80EC06F010EC26F030E9C
:10D6D600C36F830EC46F010EC56F86EC46F0830ED2
:10D6E6000001916F010E926F8EEC6EF0E0C091F02A
:10D6F600E1C092F08EEC6EF01200050E0001DE2500
:10D70600906F000EDF21916F000E936F0A0E926FDD
:10D71600A0EC6DF090C0E2F091C0E3F0E2C0BEF084
:10D72600E3C0BFF0030E0001C16FE80EC06F020E2A
:10D73600C26F030EC36F830EC46F010EC56F86ECF6
:10D7460046F0830E0001916F010E926F8EEC6EF023
:10D75600E0C091F0E1C092F08EEC6EF01200000E87
:10D7660000019D6F010E9C6F000E9F6F070E9F6557
:10D7760001D012009D0E906F000E916F9E0E926F5B
:10D78600000E936FCEEC63F000019C6F9C51D8B4F1
:10D796000BD09F51010D3C0EF324D96E020EF420DE
:10D7A600DA6E9EC0DFFF0AD09F51010D3C0EF324B6
:10D7B600D96E020EF420DA6EFF0EDF6E9F2BD6D7DF
:10D7C6000001BCBF06D0BC510BE10A0EBB5DD8B050
:10D7D60007D0E70E916F240E926F8EEC6EF00FD08D
:10D7E6000001BCBF06D0BC510AE1640EBB5DD8B0D7
:10D7F60006D0E80E916F240E926F8EEC6EF0BBC0D1
:10D80600B8F0BCC0B9F0010E0001BA6FADEC6FF014
:10D81600130E0001916F290E926F8EEC6EF01200BE
:10D826000001926F000192390F0B0F0B936F090ED7
:10D83600936503D09351570F02D09351300F90C088
:10D84600D9FF91C0DAFFDF6E904B912B92510F0BEF
:10D85600936F090E936503D09351570F02D09351DE
:10D86600300F90C0D9FF91C0DAFFDF6E904B912B3D
:10D8760090C0D9FF91C0DAFF000EDF6E1200070ECE
:10D8860000019E6F130E9F6F9E0E906F000E916F9C
:10D89600000E936F020E926F24EC65F090C012F1A9
:10D8A60091C013F1000E0001A06F000E9E6F060ED0
:10D8B6009F6F9E0E906F000E916F000E936F020E7B
:10D8C600926F24EC65F090C012F191C013F1000E36
:10D8D6000001A06F12000001916F00019151D8B4B0
:10D8E60003D0906B902B02D00001906B903B904739
:10D8F600904701019A5100019019BF0B901901013F
:10D906009A6F020E00019119D8A403D0906B902B48
:10D9160002D00001906B903B9047904701019D51CA
:10D9260000019019BF0B901901019D6F1200000EA6
:10D936000001936F000E926F000E966F090E9665AA
:10D9460001D01CD09651020D200EF324D96E020E82
:10D95600F420DA6EDECF94F0DDCF95F09451951178
:10D96600D8B40AD09451925D95519359D8B004D049
:10D9760094C092F095C093F0962BE0D792C090F0A9
:10D9860093C091F01200000E0001AC6F000EAD6F57
:10D99600000EAE6F000EAF6FA4A108D0A851AC2741
:10D9A600A951AD23AA51AE23AB51AF23D890A837C6
:10D9B600A937AA37AB37D890A733A633A533A433F4
:10D9C600A451A511A611A711D8A4E6D7ACC0A4F0FE
:10D9D600ADC0A5F0AEC0A6F0AFC0A7F01200000E15
:10D9E60060EC72F091C0D9FF92C0DAFFDF6E0001E1
:10D9F60020EE01F09151D9269251DA22000E60EC08
:10DA060072F0DF6E91C0D9FF92C0DAFFDF500001DD
:10DA1600936F20EE01F09151D9269251DA22DF5010
:10DA2600946F9451966F956B93519525916F000E57
:10DA36009621926F1200000E60EC72F091C0D9FF31
:10DA460092C0DAFFDF6E000120EE01F09151D92677
:10DA56009251DA22000E60EC72F0DF6E000120EEC9
:10DA660001F09151D9269251DA22DF50936F91C07D
:10DA7600D9FF92C0DAFFDF50946F9451966F956B81
:10DA860093519525916F000E9621926F1200B9C0A1
:10DA9600BEF0BAC0BFF00001D890BF33BE33D890F5
:10DAA600BF33BE33D890BF33BE33BE51C06FB9C08B
:10DAB600BEF0070EBE17050EBF6FD890BE37BF2F3C
:10DAC600FCD7BE51C16FC1C0ABF0000EAC6F000EEB
:10DAD600AD6FBBC0AEF0BCC0AFF0BDC0B0F0C051C2
:10DAE60088EC48F012000001916F00019151D8B402
:10DAF60003D0906B902B02D00001906B9033903343
:10DB060001019A51000190197F0B901901019A6F3A
:10DB1600020E00019119D8A403D0906B902B02D06D
:10DB26000001906B9033903301019D5100019019D3
:10DB36007F0B901901019D6F1200000E0001966F78
:10DB4600000E956F92519311D8B41CD0010E946FAC
:10DB560004D0D89092379337942B93AFFAD7D890B6
:10DB6600953796379251905D93519159D8A005D02B
:10DB76009251905F9351915B9581D89093339233F4
:10DB8600942FEDD795C090F096C091F01200000E3C
:10DB9600066E000E056E03500410D8B41CD0010E9C
:10DBA600076E04D0D89003360436072A04AEFAD797
:10DBB600D890053606360350015C04500258D8A0AA
:10DBC60005D00350015E0450025A0580D8900432F5
:10DBD6000332072EEDD705C001F006C002F0120091
:10DBE60097C090F098C091F0000E0001936F4B0E15
:10DBF600926FA0EC6DF090C099F091C09AF0000180
:10DC06009ABF06D0110E995D010E9A59D8B005D06B
:10DC1600000E9A6F000E996F06D0EF0E9925996F38
:10DC2600FE0E9A219A6F99C097F09AC098F012004A
:10DC3600200E0101836F000E00019C6F16D0840E2A
:10DC4600906F010E916F96C0D9FF97C0DAFFDF5033
:10DC560013EC6CF00001964B972B830E916F010E1F
:10DC6600926F8EEC6EF000019C2B9C519A6F9B6B11
:10DC760098519A5D99519B59D8B01200E0D700018E
:10DC8600916F00019151D8B403D0906B902B02D0C4
:10DC96000001906B0101995100019019FE0B90193A
:10DCA6000101996F020E00019119D8A403D0906B5F
:10DCB600902B02D00001906B01019C51000190193C
:10DCC600FE0B901901019C6F12000001C26FC30E7A
:10DCD6000001906F000E916F000E936F080E926F09
:10DCE6001CEC71F00001C383C3511F0B2009C36FE5
:10DCF600010EC46F200EC56FC2C0C7F0060EBA6F04
:10DD06007B0EB96FC30EBB6F000EBC6F080EBD6FE6
:10DD16004AEC6DF0120004D00001955108EC71F048
:10DD260000019151936F9251946F914B922B93C036
:10DD3600F6FF94C0F7FF000EF86E0E0EF76403D0E0
:10DD46000800F55005D0F6CFE1FFF7CFE2FFE75028
:10DD56000001956F9551D8B41200DED7CBC0D9FF1C
:10DD6600CCC0DAFFDF50406E3F50D8B40FD07F0EE4
:10DD76004018D8A404D03F5068EC6EF01200405012
:10DD8600D8B41200810EE7EC6FF012004050D8B400
:10DD960004D0040E4018D8A41200010EE7EC6FF070
:10DDA60012000001BD6FDF0E0001916F280E926F09
:10DDB6008EEC6EF0BDC0B8F00001B96B010EBA6F03
:10DDC600ADEC6FF00A0E0001BD6106D0E80E916F52
:10DDD600240E926F8EEC6EF0BBC091F0BCC092F038
:10DDE6008EEC6EF012000001916F000190692F0E0B
:10DDF600916506D03A0E916103D09151D00F11D0A2
:10DE0600400E916506D0470E916103D09151C90F1E
:10DE160008D0600E916506D0670E916103D09151CE
:10DE2600A90F906F90511200F2CFA0F0F29E000160
:10DE36009E51030B756E9DC074FF9FC073FF7F9E3E
:10DE46007F9C7F84550E7E6EAA0E7E6E7F827FB289
:10DE5600FED77F940001A0BFF28E9DC090F09EC0B9
:10DE660091F028EC72F012002D0E0101FB6F310EBD
:10DE7600FC6F010EFD6F000EFE6F000E086F000EA8
:10DE8600096F000E0A6F000E0B6F000E346E000E47
:10DE9600336E000E276F000E266F880ED56EF29435
:10DEA600F28A1200A1C09DF0A2C09EF0A3C09FF00E
:10DEB60017EC6FF0010E0001A1259D6F000EA22147
:10DEC6009E6FA4519F6F17EC6FF0A1C092F0A2C095
:10DED60093F0CAEC6FF092C0A1F093C0A2F01200CA
:10DEE600200EF86E000EF76E000EF66E0900F5CFE6
:10DEF600F4F20900F5CFF3F20900F5CFFFF1949A99
:10DF060094968A828B849494899089928A8093903D
:10DF16008B90949094928B9212000001996F00015D
:10DF26009951D8B40BD0030E966F700E956FAF0E45
:10DF3600986F420E976F7CEC71F01200030E000191
:10DF4600966F600E956FF40E986F6C0E976F7CEC63
:10DF560071F01200B8C09DF0B9C09EF0BAC09FF033
:10DF6600010E0001A06F000EA26F000EA16F000E41
:10DF7600A36F830EA46F010EA56F46EC4CF0830EC3
:10DF86000001916F010E926F8EEC6EF0120092C03E
:10DF960090F093C091F028EC72F00001996F010E99
:10DFA6009225906F000E9321916F28EC72F000017C
:10DFB600986F9851946F9951966F94C097F096C048
:10DFC60092F097C093F012000001C26FC30E0001D9
:10DFD600906F000E916F000E936F020E926F1CEC05
:10DFE60071F0C2C0C3F0000E0001BA6F000EB96F27
:10DFF600C30EBB6F000EBC6F020EBD6F4AEC6DF018
:10E006001200080EA76EAC84080EAF6E020E7D6E6F
:10E01600AC98AB8EAB88AB9AAC9CAB9CAC9AAC8AFA
:10E02600000E326E000E316E000E306E000E2F6E38
:10E036009D8A000E01015B6F1200DEC0BEF0DFC0DC
:10E04600BFF0E0C0C0F0E1C0C1F0E2C0C2F0E3C082
:10E05600C3F0830E0001C46F010EC56F86EC46F057
:10E06600830E0001916F010E926F8EEC6EF012001E
:10E07600000ECA6E9E9297C090F098C091F0000E66
:10E086000001936F330E926FA0EC6DF000019029A2
:10E09600CB6E000ECC6E7E0ECA6E9EA2FED7000E12
:10E0A600CA6E12008B94000E60EC72F08B84030E25
:10E0B6000001986FE80E976F3BEC70F08B94000EA2
:10E0C60060EC72F08B84030E0001986FE80E976F78
:10E0D6003BEC70F012000001E451E511D8A407D022
:10E0E600240E916F280E926F8EEC6EF01200E4C033
:10E0F600DEF0E5C0DFF0F50E0001E06F280EE16FFF
:10E1060080EC6BF01200E60E0001916F280E926F04
:10E116008EEC6EF04C04D8B405D04C50ADEC71F0DA
:10E1260008EC71F0300E0001916F290E926F8EECA3
:10E136006EF01200B7C09DF0B8C09EF0B9C09FF057
:10E14600BAC0A0F0830E0001A16F010EA26F42ECCF
:10E156005BF0830E0001916F010E926F8EEC6EF0F4
:10E166001200000E416E000E01014B6F000E4A6F49
:10E17600000E496F000E486F000E196F000E186FE3
:10E18600000E176F000E166F140E5C6F1200000162
:10E19600C16FE0EC71F055EC70F055EC70F055EC99
:10E1A60070F055EC70F0400E0001BC6F040EBD6FB0
:10E1B600C1514EEC67F0120095C060F096C061F058
:10E1C60097C064F098C065F099C062F09AC063F099
:10E1D6009BC070F09CC071F034EC02F000016D51F0
:10E1E6001200970E0001906F010E916F000E936F53
:10E1F600080E926F1CEC71F001019751F80B0209A1
:10E20600976F9787978F9A8712000001906F0CD0AF
:10E21600ABA204D0AC9AAC8AAB98AB88ABA404D0C2
:10E22600AECF5AF1AC9AAC8AACA2F2D790C0ADFF91
:10E23600120009D090C0D9FF91C0DAFF000EDF6E40
:10E246000001904B912B00019207D8A093079229C9
:10E25600F1E19329D8B41200EDD700019751990343
:10E26600F3CF9BF0F4CF9CF097519A03F3509C2781
:10E2760098519903F3509C279BC097F09CC098F047
:10E28600120099C060F09AC061F09BC064F09CC017
:10E2960065F09DC06CF09EC06AF09FC06BF090EC7C
:10E2A60001F000016D51120001500302F3CF05F099
:10E2B600F4CF06F001500402F35006260250030282
:10E2C600F350062605C001F006C002F01200050E46
:10E2D6004018D8A41200020E0001BA6F7B0EB96F67
:10E2E600970EBB6F010EBC6F080EBD6F4AEC6DF04A
:10E2F60012008B9495C091F096C092F01CEC72F0CF
:10E3060097C091F098C092F01CEC72F08B840301D8
:10E31600CB2B120095C060F096C061F097C064F0F8
:10E3260098C065F099C066F09AC067F008EC00F0F6
:10E3360000016D51120001016051D8B407D0090ED9
:10E346000001916F250E926F8EEC6EF0010E0101A9
:10E35600606F12000001916F0A0E0001916103D0F7
:10E366009151300F02D09151570F906F905112007A
:10E376004068000E3F6E000E0101576F000E566F8B
:10E38600000E556FF4EC70F01200050E0001966F4A
:10E396004F0E956F2A0E986F080E976F7CEC71F0F2
:10E3A6001200050E0001966F2F0E956F7B0E986F6B
:10E3B600DE0E976F7CEC71F01200050E0001966F71
:10E3C600680E956F3B0E986FAE0E976F7CEC71F0F2
:10E3D6001200070E0001966F150E956F780E986F56
:10E3E6005E0E976F7CEC71F01200030E0001966FC3
:10E3F600470E956FE50E986FCA0E976F7CEC71F01D
:10E406001200030E0001966F270E956FB40E986FDB
:10E416001C0E976F7CEC71F01200050E0001966FD2
:10E42600600E956FD30E986FA00E976F7CEC71F00F
:10E4360012000001925160EC72F00001936F91514D
:10E4460060EC72F00001946F120000019151030B11
:10E45600756E90C074FF7F9E7F9C7F807350120004
:10E46600000E01012B6F140E2A6F000E296F000E8D
:10E47600286F1200C78CC78EC698C650F00B0209CB
:10E48600C66EC68A1200000E0101236F000E226FAF
:10E49600060ECEEC5CF012003F50D8B41200810E8E
:10E4A600E7EC6FF0000E3F6E12000001C56FC5C0AD
:10E4B6003FF0810EE7EC6FF012000001906F90C004
:10E4C600C9FFC7A0FED7C9501200C90E0001906F40
:10E4D600030E916F1200E10E0001906F020E916F14
:10E4E6001200000E01011D6F000E1C6F1200000EBF
:10E4F6000101156F000E146F12000001906F90C09D
:10E5060098F11200010EB8EC22F0120001015551EB
:10E51600120033EC72F0120040501200120012008A
:020000040020DA
:0800000001010DFFFFFFFFFFEE
:020000040030CA
:0E0000001502567CFF8991FF0F800F800F00C4
:00000001FF
